:020000041000EA
:10000000000002204DF4001089F400108BF4001061
:100010008DF400108FF4001091F400100000000027
:1000200000000000000000000000000093F4001039
:1000300095F400100000000097F40010B5B4001013
:100040009DF400109FF40010A1F4001081CA00106C
:10005000A5F4001045CA001059CA00106DCA00105E
:10006000ADF40010AFF40010B1F40010B3F40010C0
:10007000B5F4001041C10010F5C9001009CA001004
:10008000BDF40010BFF40010C1F40010C3F4001060
:10009000C5F40010C7F40010C9F40010CBF4001030
:1000A000BDBA0010CBBA0010D9BA0010D3F40010BA
:1000B000D5F40010D7F40010D9F40010DBF40010D0
:1000C000DDF40010DFF400101DCA0010E3F400108E
:1000D00055C10010E7F40010E9F40010EBF4001033
:1000E000EDF40010EFF40010F1F40010F3F4001040
:1000F000F5F40010F7F40010F9F40010FBF4001010
:10010000FDF40010FFF4001001F5001003F50010DD
:1001100005F5001007F5001009F500100BF50010AB
:100120000DF500100FF5001011F5001013F500107B
:1001300015F5001017F5001069C100101BF500102F
:100140001DF500101FF5001021F5001023F500101B
:1001500025F5001027F5001029F500102BF50010EB
:100160002DF500102FF5001031F5001033F50010BB
:1001700035F5001037F5001039F500103BF500108B
:100180003DF500103FF5001041F5001043F500105B
:1001900045F5001047F5001049F500104BF500102B
:1001A00031CA00104FF5001051F5001053F5001042
:1001B00055F5001057F5001059F500105BF50010CB
:1001C0005DF500105FF5001061F5001063F500109B
:1001D0000348044B834202D0034B03B118477047D6
:1001E000480B0020480B002000000000054806498D
:1001F000091A891001EBD171491002D0034B03B1E8
:1002000018477047480B0020480B002000000000F2
:1002100010B5064C237843B9FFF7DAFF044B13B14E
:100220000448AFF300800123237010BD000C0020B0
:1002300000000000DC75011008B5044B1BB1044937
:100240000448AFF30080BDE80840CFE7000000009D
:10025000040C0020DC75011080B584B000AF78601C
:10026000124B1B68002B02D1104B114A1A600F4B26
:100270001B68FB600D4B1A687B6813441A460D4BD4
:100280009A4207D90FF060FF02460C2313604FF02B
:10029000FF3306E0054B1A687B681344034A13607A
:1002A000FB6818461037BD4680BD00BF1C0C0020FF
:1002B0000819002000F0012080B485B000AF4FF095
:1002C00080439B6803F46063BB60BB68B3F5006F59
:1002D00026D0BB68B3F5006F0BD8BB68B3F5806F51
:1002E00017D0BB68B3F5C06F16D0BB68002B1AD00F
:1002F00024E0BB68B3F5406F1CD0BB68B3F5606FFA
:1003000004D0BB68B3F5206F10D017E0164BFB602C
:1003100017E0164BFB6014E04FF4FA53FB6010E05B
:10032000134BFB600DE0134BFB600AE04FF4E1035D
:10033000FB6006E04FF40043FB6002E00C4BFB6007
:1003400000BF4FF080439B689B0903F007037B606D
:10035000FA687B6822FA03F3074A136000BF143778
:10036000BD465DF8047B7047C06878040048E8012A
:1003700000E1F505008793030000002080B483B0FE
:1003800000AF4FF080439B6803F4E0737B604FF055
:1003900080439B684FF0804243F4E073936000BF5A
:1003A000124B1B6C03F00103002BF9D000BF0F4B65
:1003B0001B6C03F00203002BF9D000BF0B4B1B6C2E
:1003C00003F00403002BF9D04FF080439B6823F423
:1003D000E0724FF080417B6813438B600023184626
:1003E0000C37BD465DF8047B704700BF00440040F9
:1003F00080B400AF00BFBD465DF8047B70470000CD
:1004000080B500AF1F4B204A9A6062B61F4802F0C9
:10041000DBF81C4BD3F888301A4A43F47003C2F857
:100420008830BFF34F8FBFF36F8F40F2D66002F07A
:10043000C7F900BF02F0EEF90346002BFAD140F2F3
:100440004C4002F0CBF900BF02F0EEF90346002B5E
:10045000FAD140F24C4002F0CFF900BF02F0EEF9C1
:100460000346002BFAD1042004F01CF8002004F00D
:1004700021F9FFF721FF0CF03BF9FFF7B9FF00BFAF
:1004800080BD00BF00ED00E00000001000A00240B1
:1004900080B500AF1A2004F03BF9172003F034FFB9
:1004A000024800F071F80346184680BD0040034042
:1004B00080B584B000AF78607B689B02FB60FB680E
:1004C0001C4A934202D96FF002032EE01A4B1B68BC
:1004D0005A08FB68B2FBF3F3FB72FB7A0F2B02D8CE
:1004E000FB7A012B02D86FF002031EE0134B1B684E
:1004F000124A23F4006313604FF080439B694FF06E
:10050000804223F4705393614FF080439B69FA7AE1
:10051000920211464FF080420B439361796807487D
:1005200000F08DF800F00CF8034618461037BD4671
:1005300080BD00BF00127A00000000200040034090
:1005400080B582B000AF4FF080439B699B0ADBB25D
:1005500003F00F03FB71FB79184600F083F80346A4
:1005600018460837BD4680BD80B582B000AF03464F
:10057000FB71FB791946034800F08AF800BF083781
:10058000BD4680BD0040034080B584B000AF7860B8
:1005900041F2D760FFF78CFFB8604FF40031786804
:1005A00000F038F87B681B6843F002027B681A6031
:1005B0007B681B6843F008027B681A6000BF7B6899
:1005C000DB6803F40033002BF9D04FF40031786876
:1005D00000F020F80C4B00221A600023FB7307E0A8
:1005E000FB7B0A4A002142F82310FB7B0133FB739B
:1005F000FB7B032BF4D9064B00221A60002318461C
:100600001037BD4680BD00BF300C0020200C0020FC
:10061000340C002080B483B000AF786039607B6810
:10062000DB6803F01F023B6803F4F8131A437B688E
:10063000DA6000BF0C37BD465DF8047B704780B4BC
:1006400083B000AF786039607B681B6843F4006258
:100650007B681A60002318460C37BD465DF8047BA2
:100660007047000080B485B000AF0346FB71074BB4
:100670001B685A08FB79B2FBF3F3FB60FB689B0A2B
:1006800018461437BD465DF8047B70470000002013
:1006900080B483B000AF78600B46FB707B681B684A
:1006A00023F4C0227B681A60FB78062B00F2858059
:1006B00001A252F823F000BFD5060010EF0600108B
:1006C0000907001023070010490700106F070010EA
:1006D000950700107B681B6843F480727B681A6082
:1006E0007B681B6823F400727B681A6072E07B6889
:1006F0001B6823F480727B681A607B681B6823F494
:1007000000727B681A6065E07B681B6823F4807266
:100710007B681A607B681B6843F400727B681A6010
:1007200058E07B681B6823F480727B681A607B68E2
:100730001B6823F400727B681A607B681B6843F4B3
:1007400080227B681A6045E07B681B6823F4807216
:100750007B681A607B681B6843F400727B681A60D0
:100760007B681B6843F400327B681A6032E07B6868
:100770001B6823F480727B681A607B681B6843F4F3
:1007800000727B681A607B681B6843F480227B6878
:100790001A601FE07B681B6823F480727B681A6014
:1007A0007B681B6843F400727B681A607B681B6877
:1007B00043F4C0227B681A600CE07B681B6823F45A
:1007C00080727B681A607B681B6823F400727B6808
:1007D0001A6000BF00BF0C37BD465DF8047B704750
:1007E00080B582B000AF78607B68002B43DB7B680C
:1007F000032B40DC23497A6813469B0013449B007B
:100800000B441B68002B36D001211F4803F0B4FCB9
:100810000346002B02D06FF005032EE019497A68D9
:1008200013469B0013449B000B4400221A60154999
:100830007A6813469B0013449B000B440C331B68DF
:1008400000221A600F497A6813469B0013449B00EC
:100850000B440C3319680B487A6813469B00134409
:100860009B0003440C331B684A685A60064803F037
:10087000A9FC002301E06FF0020318460837BD46CB
:1008800080BD00BF380C0020880C002080B485B0EB
:1008900000AF7860134B1B78002B1CD10023FB604A
:1008A00013E00023BB600AE00F49FB685A01BB68F4
:1008B0001344002241F82320BB680133BB60BB68AE
:1008C0001F2BF1DDFB680133FB60FB68032BE8DDC8
:1008D000044B01221A70002318461437BD465DF8F8
:1008E000047B70478C1000208C0C002080B487B0F3
:1008F00000AFF860B9607A60FB685B687B610023D9
:100900003B6154E07B6903F00103002B49D0FB6895
:100910001B682B4A934217D0FB681B68294A9342F5
:1009200010D0FB681B68284A934209D0FB681B68FB
:10093000264A934201D1032307E04FF0FF3304E03E
:10094000022302E0012300E0002321495A013B6910
:100950001344BA6841F82320FB681B68184A934285
:1009600017D0FB681B68174A934210D0FB681B68BE
:10097000154A934209D0FB681B68144A934201D17F
:10098000032307E04FF0FF3304E0022302E00123DA
:1009900000E000230F495A013B6913447A6841F88B
:1009A00023203B6901333B617B695B087B617B6989
:1009B000002BA7D100BF1C37BD465DF8047B7047F4
:1009C00000800040009000400004084000060840FD
:1009D0008C0C00208C0E002080B586B000AF7860B3
:1009E0007B68002B10D07B68012B0BD07B68022B1F
:1009F00006D07B68032B01D11F4B06E0002304E0E7
:100A00001E4B02E01E4B00E01E4BFB60F86800F03E
:100A1000FCFA78617969F86800F0EAFA00233B6132
:100A200023E07B6903F00103002B18D016497B6893
:100A30005A013B69134451F82330002B0FD012495F
:100A40007B685A013B69134451F823300F487A6898
:100A500051013A690A4450F82220104698473B69F0
:100A600001333B617B695B087B617B69002BD8D1DB
:100A700000BF1837BD4680BD00060840000408408E
:100A800000900040008000408C0C00208C0E002064
:100A900080B582B000AF78607B6803F00103002B63
:100AA00002D0002003F030FC7B6803F00203002B2F
:100AB00002D0012003F028FC7868FFF7E7FE034628
:100AC00018460837BD4680BD80B586B000AF786057
:100AD0007B681B687B617B681B68994A934217D0CF
:100AE0007B681B68974A934210D07B681B68964AC4
:100AF000934209D07B681B68944A934201D1032337
:100B000007E04FF0FF3304E0022302E0012300E09E
:100B100000233B617B681B688C4A93426FD17B68E2
:100B20005B6803F00103002B2FD07B681B7A002B3E
:100B300002D0012B07D00DE0854B1B6A844A23F0BD
:100B40000203136209E0824B1B6A814A43F00203ED
:100B5000136202E06FF0100305E17B685B7A002B03
:100B600002D0012B07D00DE0794B1B6A784A23F0A5
:100B7000040313620AE0764B1B6A754A43F00403D0
:100B8000136203E06FF01003EDE000BF7B685B6869
:100B900003F00203002B2FD07B681B7A002B02D0BE
:100BA000012B07D00DE06A4B1B6A694A23F0200332
:100BB000136209E0664B1B6A654A43F02003136227
:100BC00002E06FF01003CEE07B685B7A002B02D06E
:100BD000012B07D00DE05E4B1B6A5D4A23F04003FA
:100BE00013620AE05A4B1B6A594A43F040031362EE
:100BF00003E06FF01003B6E000BF0023B3E0012272
:100C00003B6902FA03F31846FFF742FF7B68197A43
:100C10007B685B681A46786900F044FBF860FB6803
:100C2000002B01D0FB689EE07B685B7A042B00F20E
:100C3000848001A252F823F04D0C0010A30C001088
:100C4000090D00106F0C0010D50C00107B691A6E96
:100C50007B685B68DB431A407B691A667B695A6E66
:100C60007B685B68DB431A407B695A6672E07B698C
:100C70001A6E7B685B681A437B691A667B695A6ED9
:100C80007B685B68DB431A407B695A667B69D3F8F3
:100C9000B8207B685B68DB431A407B69C3F8B820E7
:100CA00058E07B691A6E7B685B681A437B691A6639
:100CB0007B695A6E7B685B68DB431A407B695A66C6
:100CC0007B69D3F8B8207B685B681A437B69C3F8FB
:100CD000B8203FE07B691A6E7B685B68DB431A4093
:100CE0007B691A667B695A6E7B685B681A437B690D
:100CF0005A667B69D3F8B8207B685B68DB431A408F
:100D00007B69C3F8B82025E07B691A6E7B685B6855
:100D1000DB431A407B691A667B695A6E7B685B68A5
:100D20001A437B695A667B69D3F8B8207B685B6895
:100D30001A437B69C3F8B8200CE06FF0020312E09D
:100D40000080004000900040000408400006084079
:100D5000006C00407B68997A7B685B681A4678690A
:100D600000F05FF9034618461837BD4680BD00BF46
:100D700080B584B000AF786039607B68234A9342C5
:100D80003BD13B6803F00103002B22D03B6803F00A
:100D90000203002B1DD00023FB601D4B1B6A03F0D8
:100DA0000803002B14BF01230023DBB21A46FB68A3
:100DB0001343FB60164B1B6A03F08003002B01D02A
:100DC000022300E000231A46FB681343FB60FB6824
:100DD00018E03B6803F00103002B04D00C4B1B6AA6
:100DE00003F008030EE03B6803F00203002B04D07D
:100DF000074B1B6A03F0800304E03968786800F051
:100E000022F9034618461037BD4680BD000608404B
:100E1000006C004080B582B000AF786039607B68BC
:100E2000114A934216D13B6803F00103002B05D011
:100E30000E4B1B6A0D4A43F0010313623B6803F03B
:100E40000203002B0BD0094B1B6A084A43F0100326
:100E5000136204E03968786800F004F900E000BF2C
:100E60000837BD4680BD00BF00060840006C00404A
:100E700080B582B000AF786039607B68114A9342D8
:100E800016D13B6803F00103002B05D00E4B1B6A03
:100E90000D4A23F0010313623B6803F00203002BA9
:100EA0000BD0094B1B6A084A23F01003136204E0BD
:100EB0003968786800F0E4F800E000BF0837BD4604
:100EC00080BD00BF00060840006C004080B584B0C3
:100ED00000AF786039607B68214A934236D13B6825
:100EE00003F00303002B1DD00023FB601D4B1B6A86
:100EF00003F00103002B14BF01230023DBB21A46C9
:100F0000FB681343FB60174B1B6A03F01003002BB5
:100F100001D0022300E000231A46FB681343FB6064
:100F2000FB6818E03B6803F00103002B04D00D4B75
:100F30001B6A03F001030EE03B6803F00203002B81
:100F400004D0084B1B6A03F0100304E0396878688A
:100F500000F0A4F8034618461037BD4680BD00BF18
:100F600000060840006C004080B582B000AF786099
:100F70000B46FB70FB781946786800F09FF8034633
:100F800018460837BD4680BD80B582B000AF786096
:100F900039603968786800F025F900BF0837BD4628
:100FA00080BD80B582B000AF7860396039687868FC
:100FB00000F026F900BF0837BD4680BD80B584B07B
:100FC00000AFF860B9607A607A68B968F868FFF7CE
:100FD0008DFC00BF1037BD4680BD80B582B000AF2C
:100FE00078607868FFF7F8FC00BF0837BD4680BD21
:100FF00080B582B000AF786039603968786800F0F9
:101000000DF900BF0837BD4680BD80B582B000AF86
:101010007860786800F010F9034618460837BD4636
:1010200080BD80B584B000AFF8600B467A60FB727B
:10103000FB7A7A681946F86800F00AF90346184600
:101040001037BD4680BD80B483B000AF7860396092
:101050007B685A6A3B68134018460C37BD465DF8FA
:10106000047B704780B483B000AF786039607B68E0
:101070003A68DA6100BF0C37BD465DF8047B704703
:1010800080B483B000AF786039607B683A681A62D8
:1010900000BF0C37BD465DF8047B704780B483B059
:1010A00000AF786039607B689A693B6813401846E6
:1010B0000C37BD465DF8047B7047000080B485B0F6
:1010C00000AF78600B46FB707B681B68FB60FB78A9
:1010D000042B7CD801A252F823F000BF231100108A
:1010E000F11000108311001053110010B111001005
:1010F000FB68DA6A7B685B68DB431A40FB68DA628C
:10110000FB68DA6D7B685B68DB431A40FB68DA6575
:10111000FB689A6A7B685B68DB431A40FB689A62EB
:1011200058E0FB68DA6A7B685B68DB431A40FB685F
:10113000DA62FB68DA6D7B685B68DB431A40FB6848
:10114000DA65FB689A6A7B685B681A43FB689A6297
:1011500040E0FB68DA6A7B685B681A43FB68DA6226
:10116000FB68DA6D7B685B68DB431A40FB68DA6515
:10117000FB689A6A7B685B68DB431A40FB689A628B
:1011800028E0FB68DA6A7B685B681A43FB68DA620E
:10119000FB68DA6D7B685B68DB431A40FB68DA65E5
:1011A000FB689A6A7B685B681A43FB689A6211E085
:1011B000FB68DA6D7B685B681A43FB68DA65FB687D
:1011C0009A6A7B685B681A43FB689A6202E06FF078
:1011D000020300E0002318461437BD465DF8047B87
:1011E000704700BF80B483B000AF786039607B681F
:1011F0003A689A6300BF0C37BD465DF8047B7047C0
:1012000080B483B000AF786039607B683A68DA6395
:1012100000BF0C37BD465DF8047B704780B483B0D7
:1012200000AF786039607B683A689A6400BF0C3719
:10123000BD465DF8047B704780B483B000AF786032
:101240007B681B6C18460C37BD465DF8047B704705
:1012500080B485B000AFF8600B467A60FB72FB7A11
:10126000002B02D0012B0AD012E0FB68D3F8C0207B
:101270007B68DB431A40FB68C3F8C0200BE0FB68C7
:10128000D3F8C0207B681A43FB68C3F8C02002E093
:101290006FF0020300E0002318461437BD465DF8E6
:1012A000047B704780B485B000AFF8600B467A606D
:1012B000FB72FB681A6B7B681A43FB681A63FB7A44
:1012C000052B69D801A252F823F000BFE5120010E7
:1012D00007130010291300104513001061130010AC
:1012E0007D130010FB687A685A61FB687A685A605F
:1012F000FB687A681A67FB687A68DA67FB687A685D
:10130000C3F888204BE0FB687A681A61FB687A684A
:101310005A60FB687A681A67FB687A68DA67FB6864
:101320007A68C3F888203AE0FB687A68DA67FB6875
:101330007A681A67FB687A689A60FB687A68C3F80B
:1013400088202CE0FB687A68DA67FB687A68DA66DE
:10135000FB687A689A60FB687A68C3F888201EE0A8
:10136000FB687A689A67FB687A681A67FB687A682C
:101370009A60FB687A68C3F8882010E0FB687A6896
:101380009A67FB687A68DA66FB687A689A60FB6835
:101390007A68C3F8882002E06FF0020300E00023BF
:1013A00018461437BD465DF8047B704780B584B09D
:1013B00000AFF860B9607A60FB68002B02D14FF093
:1013C000FF332CE0F86800F04BF8FB68164A9342B4
:1013D00006D10D2002F098FF1448FFF775FB18E0C6
:1013E000FB68134A934206D11C2002F08DFF11487E
:1013F000FFF76AFB0DE0FB680F4A934206D13820E5
:1014000002F082FF0D48FFF75FFB02E06FF001037F
:1014100005E07A68B968F86800F01EF903461846D6
:101420001037BD4680BD00BF00D00140506501109F
:1014300000E001405C65011000F0014068650110AA
:1014400080B584B000AFF860B9607A607A68B96836
:10145000F86800F081F9034618461037BD4680BD94
:1014600080B582B000AF78607B68144A934206D1A1
:101470000D2002F00BFF102003F04AF918E07B6802
:101480000F4A934206D11C2002F000FF202003F0F7
:101490003FF90DE07B680B4A934206D1382002F0F9
:1014A000F5FE342003F034F902E06FF0010300E0B0
:1014B000002318460837BD4680BD00BF00D001405C
:1014C00000E0014000F0014080B582B000AF7860DC
:1014D00039603B68074A934202D96FF0100304E079
:1014E0003968786800F068F9034618460837BD4641
:1014F00080BD00BF40420F0080B582B000AF786071
:10150000786800F0BDF9034618460837BD4680BD2F
:1015100080B582B000AF7860786800F0CFF90346FC
:1015200018460837BD4680BD80B582B000AF7860F0
:10153000786800F0E7F9034618460837BD4680BDD5
:1015400080B584B000AFF860B9607A607A68B96835
:10155000F86800F0F5F9034618461037BD4680BD1F
:1015600080B584B000AFF860B9607A607A68B96815
:10157000F86800F010FA034618461037BD4680BDE3
:1015800080B582B000AF7860786800F030FA00BFB4
:101590000837BD4680BD80B582B000AF78607868FE
:1015A00000F03CFA00BF0837BD4680BD80B584B06E
:1015B00000AFF860B9607A607A68B968F86800F0DE
:1015C00044FA00BF1037BD4680BD80B582B000AF81
:1015D000786039603968786800F049FA034618463F
:1015E0000837BD4680BD80B582B000AF78607868AE
:1015F00000F0E0FA034618460837BD4680BD80B5C6
:1016000082B000AF786039603968786800F008FC13
:10161000034618460837BD4680BD80B582B000AF8E
:10162000786039603968786800F01AFC034618461B
:101630000837BD4680BD000080B582B000AF78603D
:10164000044B1B681946786800F07AFF00BF083722
:10165000BD4680BD0400002080B586B000AFF860B4
:10166000B9607A60FB68002B02D14FF0FF3367E06E
:101670001021F868FFF7A9FF78617B69002B01D082
:101680007B695DE0FB681B6843F00102FB681A6040
:10169000F868FFF775FFF868FFF77DFF0221F8682B
:1016A000FFF7BBFF0621F868FFF7A9FFBB68002B17
:1016B00022D100227968F868FFF7C2FEFB68224A4F
:1016C00093420ED0FB68214A934208D0FB68204A1F
:1016D000934201D1022205E04FF0FF3202E00122E5
:1016E00000E000221B4913465B001344DB000B445F
:1016F000043300221A6022E0FB681B6843F00202F8
:10170000FB681A60FB68104A93420ED0FB680F4AD0
:10171000934208D0FB680E4A934201D1022205E0B1
:101720004FF0FF3202E0012200E000220949134697
:101730005B001344DB000B44043301221A600023D6
:1017400018461837BD4680BD00D0014000E001407A
:1017500000F001409010002080B485B000AFF86028
:10176000B9607A60FB68002B02D14FF0FF331DE0B7
:101770007B68002B02D06FF0100317E0BB68B3F555
:10178000806F02D36FF0020310E0FB680022DA647E
:10179000BB687F2B03D9FB684FF40042DA64FB6817
:1017A000DA6CBB681A43FB68DA6400231846143706
:1017B000BD465DF8047B704780B588B000AF7860A7
:1017C00039607B68002B02D14FF0FF334BE03B6860
:1017D000274A934220D9274B1B685A083B68B2FB23
:1017E000F3F3FB61FB695B00234AA2FB03235B0865
:1017F000013BBB61FB69204AA2FB03235B08013B61
:101800007B617B690F2B02DCBB690F2B02DD6FF064
:10181000020328E0194B3B60164B1B685A083B68D3
:10182000B2FBF3F3FB61FB695B08013B3B61FB69C6
:101830005B08013BFB603B69B3F5007F02D2FB68AC
:10184000002B02D16FF002030DE0FB68C3F3080226
:101850007B685A633B69C3F308027B689A637868C4
:10186000FFF74AFE034618462037BD4680BD00BF3D
:1018700040420F0000000020ABAAAAAA801A06006E
:1018800080B485B000AF78600023FB607B685B6B41
:10189000C3F308027B689B6BC3F308031344FB602C
:1018A000054B1B685A08FB68B2FBF3F31846143764
:1018B000BD465DF8047B70470000002080B483B013
:1018C00000AF78607B68002B02D14FF0FF3313E04C
:1018D0007B681B6B03F00103002B06D07B681B6B3E
:1018E00043F002027B681A6305E07B681B6B43F0E0
:1018F00001027B681A63002318460C37BD465DF869
:10190000047B704780B483B000AF78607B68002BA5
:1019100002D14FF0FF330DE07B681B6B43F00402F4
:101920007B681A6300BF7B681B6B03F00403002B0A
:10193000F9D1002318460C37BD465DF8047B70478B
:1019400080B487B000AFF860B9607A6000237B6133
:10195000FB68002B02D0BB68002B0BD14FF0FF338C
:1019600013E0FB68D96A7B695A1C7A61BA68134430
:10197000CAB21A707A687B699A4205D9FB685B68BB
:1019800003F00203002BECD07B6918461C37BD46E0
:101990005DF8047B704780B487B000AFF860B96031
:1019A0007A6000237B61FB68002B02D0BB68002BB0
:1019B0000CD14FF0FF3314E07B695A1C7A61BA688E
:1019C00013441B78DBB21A46FB68DA627A687B69DB
:1019D0009A4205D9FB685B6803F01003002BEBD03B
:1019E0007B6918461C37BD465DF8047B704780B4A0
:1019F00083B000AF78607B68DB6943F080027B686E
:101A0000DA6100BF7B68DB6903F08003002BF9D14A
:101A100000BF0C37BD465DF8047B704780B483B0CF
:101A200000AF78607B685B6A43F080027B685A6233
:101A300000BF7B685B6A03F08003002BF9D100BF15
:101A40000C37BD465DF8047B704780B485B000AFAD
:101A5000F860B9607A60FB68BA689A60FB687A6877
:101A60001A6100BF1437BD465DF8047B704780B52E
:101A700086B000AF786039607B68002B02D14FF0F0
:101A8000FF3393E06FF008037B617B681B6843F0D2
:101A900001027B681A607B681B6803F48063FB604B
:101AA0007B68002B02D14FF0FF337FE07B681B681F
:101AB00043F480627B681A6000233B6162E00A2085
:101AC00002F022FB7B681B6823F040027B681A60EF
:101AD0000A2002F019FB7B681B6803F48073002B5B
:101AE00006D07B681B6843F0C0027B681A6046E042
:101AF0000A2002F009FB7B681B6823F080027B68E8
:101B00001A600A2002F000FB7B681B6803F4007374
:101B1000002B06D07B681B6843F0C0027B681A600C
:101B20002DE00A2002F0F0FA7B681B6843F0800287
:101B30007B681A600A2002F0E7FA7B681B6803F4EE
:101B40000073002B06D17B681B6843F0C0027B68E2
:101B50001A6014E00A2002F0D7FA7B681B6843F091
:101B600040027B681A600A2002F0CEFA7B681B688C
:101B700003F48073002B02D000237B6106E03B69F5
:101B800001333B613A693B689A4298D3FB68002B6A
:101B900005D17B681B6823F480627B681A607B68D0
:101BA0001B6823F001027B681A607B6918461837AE
:101BB000BD4680BD80B586B000AF78607B681B688D
:101BC000FB6000237B6100233B617B685B687F2BAC
:101BD00002D96FF0100319E1FB688E4A93420AD0D4
:101BE000FB688D4A934206D0FB688C4A934202D030
:101BF0006FF002030AE1FB681B6803F00203002B8D
:101C000002D16FF0060301E107226FF07F41F8680F
:101C1000FFF7CCFCF868FFF7BEFCF868FFF7B0FCF4
:101C2000FB680022DA60FB6800225A617B685B690E
:101C3000002B03D07B68DB68002B34D07B685B68AB
:101C40005A00FB68DA62FB681B6B43F00102FB6819
:101C50001A6328E0FB689B6803F02003002B13D075
:101C60007B689A687B69D1187B68DA687B69D31ACC
:101C70001A46F868FFF774FC03461A467B6913445A
:101C80007B61FB6820229A60FB689B6803F4FE433B
:101C9000002B08D07B687A69DA60F868FFF744FCAB
:101CA0006FF00803B2E07B68DB687A699A42D1D3AF
:101CB00000221121F868FFF779FC7B685B69002B33
:101CC00073D07B685B69B3F5807F03D9FB68002222
:101CD0001A6203E07B685A69FB681A62F868FFF7CA
:101CE00017FC00BFFB681B6B03F00203002BF9D14C
:101CF0007B685B685B0043F00102FB68DA6254E0DA
:101D0000FB689B6803F01103002B13D07B681A69F2
:101D10003B69D1187B685A693B69D31A1A46F8683F
:101D2000FFF70EFC03461A463B6913443B61FB6810
:101D300010229A60FB689B6803F4FE43002B08D0D6
:101D40007B683A695A61F868FFF7EEFB6FF00803A9
:101D50005CE0FB689B6803F00103002B25D07B68E7
:101D60005B693A699A4220D97B685A693B69D31A00
:101D7000B3F5807F03D9FB6800221A6205E07B6817
:101D80005A693B69D21AFB681A62FB681B6B43F005
:101D90000202FB681A63FB6801229A607B685B6839
:101DA0005B0043F00102FB68DA627B685B693A69B9
:101DB0009A42A5D37B689B69002B06D0FB681B6BFE
:101DC00043F00202FB681A6305E0FB681B6B43F0FB
:101DD0000402FB681A6300BFFB689B6803F04003C2
:101DE000002BF9D000BFFB689B6803F00103002BB8
:101DF000F9D0FB6841229A60FB689B6803F4FE43BC
:101E0000002B02D06FF0080300E0002318461837BB
:101E1000BD4680BD00D0014000E0014000F001401F
:101E200080B485B000AF786039607B689B69DBB2B5
:101E3000FB603A68FB689A4202D96FF0020309E03E
:101E40007B68DB6923F470623B681B021A437B6882
:101E5000DA61002318461437BD465DF8047B7047ED
:101E600080B485B000AF786039607B689B691B0ADD
:101E7000DBB2FB603A68FB689A4202D96FF002035A
:101E800009E07B685B6A23F470623B681B021A43BB
:101E90007B685A62002318461437BD465DF8047B00
:101EA0007047000080B584B000AF786039607B680F
:101EB000114A93420ED07B68104A934208D07B6847
:101EC0000F4A934201D1022305E04FF0FF3302E0B5
:101ED000012300E000230B4A52F82330FB60FB682B
:101EE000DB69002B04D0FB68DB693968F868984728
:101EF00000BF1037BD4680BD00D0014000E001406A
:101F000000F001405018002080B483B000AF78602A
:101F10007B680022DA607B6800225A617B689A68DD
:101F20007B689A607B681A697B681A617B680E4AD5
:101F300093420ED07B680D4A934208D07B680C4ACE
:101F4000934201D1022305E04FF0FF3302E0012369
:101F500000E00023074A002142F8231000BF0C379D
:101F6000BD465DF8047B704700D0014000E00140B1
:101F700000F001405018002080B586B000AF7860B6
:101F8000984A7B6852F823307B61974A7B6852F805
:101F900023303B617B68002B0BD07B68012B06D084
:101FA0007B68022B01D1914B04E0002302E0904BAF
:101FB00000E0904BFB60904A7B6852F82330BB6096
:101FC000FB689B6803F4FE43002B19D0FB689A68FA
:101FD000FB689A60FB681A69FB681A61FB6800225B
:101FE000DA60FB6800225A61F868FFF79DFA6FF02B
:101FF0000801F868FFF756FFF868FFF785FFEEE085
:10200000BB68DB687A699A4243D2FB689B6803F03D
:102010002003002B13D0BB689A687B69D118BB687A
:10202000DA687B69D31A1A46F868FFF799FA03460B
:102030001A467B6913447B61FB6820229A60BB6867
:10204000DB687A699A4206D2FB68DB6843F02002BB
:10205000FB68DA6005E0FB68DB6823F02002FB68C0
:10206000DA60BB68DB687A699A4212D1BB685B6947
:10207000002B0ED0FB681B6B43F00202FB681A6357
:10208000FB6801229A60FB68DB6843F00102FB6891
:10209000DA60BB685B693A699A4219D2FB689B684F
:1020A00003F01103002B13D0BB681A693B69D118E8
:1020B000BB685A693B69D31A1A46F868FFF740FAB9
:1020C00003461A463B6913443B61FB6810229A6041
:1020D000BB68DB687A699A423AD1BB685B693A6946
:1020E0009A4235D0FB689B6803F00103002B2FD088
:1020F000FB6801229A603B69002B06D1BB685B68D4
:102100005B0043F00102FB68DA62BB685A693B6915
:10211000D31AB3F5807F03D9FB6800221A6205E069
:10212000BB685A693B69D21AFB681A62BB685B6973
:102130003A699A4206D2FB68DB6843F01102FB68F9
:10214000DA6005E0FB68DB6823F01102FB68DA6007
:10215000BB68DB687A699A4237D1BB685B693A69C8
:102160009A4232D1FB680022DA60FB6800225A6191
:10217000FB689A68FB689A60FB681A69FB681A61D9
:10218000BB689B69002B06D0FB681B6B43F0020207
:10219000FB681A6305E0FB681B6B43F00402FB68F5
:1021A0001A63FB689B6803F4FE43002B05D06FF0B5
:1021B0000801F868FFF776FE03E00021F868FFF7F2
:1021C00071FEF868FFF7A0FE09E006497B687A69AE
:1021D00041F8232004497B683A6941F823201837E5
:1021E000BD4680BD5C1800206818002000F001404A
:1021F00000E0014000D001405018002080B586B0BA
:1022000000AFF860B9607A603B60FB689B687B61F7
:102210003B6800221A60FB681B6803F400633B61A3
:102220007A68A04B1340002B40F0DF807B6903F4F9
:10223000FE43002B31D03B686FF008021A60BB6888
:10224000002B04D0BB683A680421F868984707223D
:102250006FF07F41F868FFF7A9F9F868FFF79BF97D
:10226000F868FFF78DF900237B60FB688E4A934284
:102270000ED0FB688D4A934208D0FB688C4A93428B
:1022800001D1022305E04FF0FF3302E0012300E01B
:102290000023884A002142F823107B6803F01103D1
:1022A000002B20D07B6903F01003002B0AD0BB6801
:1022B000002B04D0BB6800220221F8689847FB6815
:1022C00010229A60FB681B6903F00103002B0AD0FF
:1022D000BB68002B04D0BB6800220621F868984731
:1022E000FB6801221A617A6848F222031340002B2E
:1022F0004ED07B6903F02003002B0AD0BB68002B73
:1023000004D0BB6800220321F8689847FB682022AC
:102310009A60FB681B6903F00203002B0AD0BB68BC
:10232000002B04D0BB6800220521F8689847FB68A1
:1023300002221A617B6903F40043002B28D03B681A
:1023400000221A60BB68002B04D0BB683A680421E5
:10235000F8689847FB684FF400429A6000237B605E
:10236000FB68514A93420ED0FB68504A934208D012
:10237000FB684F4A934201D1022305E04FF0FF333F
:1023800002E0012300E000234A4A002142F8231022
:102390007B6903F04003002B27D03B6800221A60C2
:1023A000BB68002B04D0BB683A680421F8689847E2
:1023B000FB6840229A6000237B60FB683A4A9342A4
:1023C0000ED0FB68394A934208D0FB68384A9342E2
:1023D00001D1022305E04FF0FF3302E0012300E0CA
:1023E0000023344A002142F823107B6903F4800360
:1023F000002B11D0BB68002B04D0BB680022002149
:10240000F8689847FB684FF480029A60FB680822DE
:102410009A6047F611737B607B6903F40003002B1D
:1024200011D0BB68002B04D0BB6800220121F868E2
:102430009847FB684FF400029A60FB6808229A6094
:102440004FF622737B607B6903F00803002B33D0C7
:102450003B6903F40063002B11D0BB68002B04D050
:10246000BB6800220121F8689847FB6808229A603F
:10247000FB6808229A604FF622737B6053E0BB68CA
:10248000002B04D0BB6800220021F8689847FB6845
:1024900008229A60FB6808229A6047F611737B60F5
:1024A00041E000BF0800C00000D0014000E0014052
:1024B00000F00140501800207B6903F4FE43002B1C
:1024C00031D03B686FF008021A60BB68002B04D063
:1024D000BB683A680421F868984707226FF07F418B
:1024E000F868FFF7B2FAF868FFF798FAF868FFF7AC
:1024F0007EFA00237B60FB680D4A93420ED0FB6896
:102500000C4A934208D0FB680B4A934201D1022344
:1025100005E04FF0FF3302E0012300E00023074A0B
:10252000002142F823107B6818461837BD4680BD4D
:1025300000D0014000E0014000F0014050180020B0
:1025400080B586B000AF786039607B681A4A9342E4
:102550000ED07B68194A934208D07B68184A934290
:1025600001D1022305E04FF0FF3302E0012300E038
:1025700000237B617B69002B1ADB7B681B6803F0FF
:102580000203002B03D07869FFF7F6FC11E00D4A37
:102590007B6952F823303B617B68DA6807F10C03F2
:1025A00039697868FFF72AFE02467B68DA6000E046
:1025B00000BF1837BD4680BD00D0014000E001409B
:1025C00000F001405018002080B582B000AF786064
:1025D000786800F013F800BF0837BD4680BD80B4AE
:1025E00083B000AF78607B68D3F8003103F48033A8
:1025F00018460C37BD465DF8047B704780B582B045
:1026000000AF78607B68D3F8003123F001027B686B
:10261000C3F800217B680122C3F8002700BF786857
:10262000FFF7DDFF0346002BF9D07B68D3F80031BC
:1026300043F001027B68C3F8002100BF7868FFF710
:10264000CEFF0346002BF9D000BF0837BD4680BD42
:1026500080B582B000AF78607968044800F042F835
:10266000034618460837BD4680BD00BF00600040E5
:1026700080B582B000AF78607968044800F057F800
:10268000034618460837BD4680BD00BF00600040C5
:1026900080B500AF024800F070F80346184680BDD0
:1026A0000060004080B582B000AF7860796804486F
:1026B00000F071F8034618460837BD4680BD00BFDC
:1026C0000060004080B400AF00BF054B1B6903F001
:1026D0000803002BF9D100BFBD465DF8047B7047AD
:1026E0000060004080B582B000AF786039603B6820
:1026F00003F026033B603B68002B02D16FF002031E
:1027000011E0FFF7DFFF7B681A693B681A437B68BB
:102710001A613B6823F020033B603B68002B01D02B
:10272000FFF7D0FF002318460837BD4680BD80B5AF
:1027300082B000AF786039603B6803F026033B60ED
:102740003B68002B02D16FF0020312E0FFF7BAFFE3
:102750007B681A693B68DB431A407B681A613B68F7
:1027600023F020033B603B68002B01D0FFF7AAFF5A
:10277000002318460837BD4680BD80B483B000AF43
:1027800078607B681B6903F0D00318460C37BD46A0
:102790005DF8047B704780B483B000AF7860396027
:1027A0007B681B693A6802F0D002D2431A407B680A
:1027B0001A61002318460C37BD465DF8047B70474C
:1027C00080B582B000AF78607968034800F040F8C7
:1027D00000BF0837BD4680BD0044004080B582B0D0
:1027E00000AF78607968034800F066F800BF0837EA
:1027F000BD4680BD0044004080B582B000AF786027
:102800007968034800F08CF800BF0837BD4680BDEA
:102810000044004080B500AF024800F0B5F8034620
:10282000184680BD0044004080B500AF024800F06B
:10283000BFF80346184680BD0044004080B500AF95
:10284000024800F0C9F80346184680BD0044004025
:1028500080B487B000AF7860396000237B617B680B
:102860005B6803F08003002B03D04FF416737B6189
:1028700002E04FF4FA737B613A687B69D31A0D4A20
:10288000A2FB0323DB083B617B685B6823F07F02CC
:102890003B6903F07F031343FB607B68FA685A606F
:1028A0007B68FA685A6000BF1C37BD465DF8047B40
:1028B000704700BFCDCCCCCC80B487B000AF78607F
:1028C000396000237B617B689B6803F08003002BE9
:1028D00003D04FF416737B6102E04FF4FA737B610F
:1028E0003A687B69D31A0D4AA2FB0323DB083B61DC
:1028F0007B689B6823F07F023B6903F07F031343EF
:10290000FB607B68FA689A607B68FA689A6000BF2F
:102910001C37BD465DF8047B704700BFCDCCCCCCE6
:1029200080B487B000AF7860396000237B617B683A
:10293000DB6803F08003002B03D04FF416737B6138
:1029400002E04FF4FA737B613A687B69D31A0D4A4F
:10295000A2FB0323DB083B617B68DB6823F07F027B
:102960003B6903F07F031343FB607B68FA68DA601E
:102970007B68FA68DA6000BF1C37BD465DF8047BEF
:10298000704700BFCDCCCCCC80B483B000AF7860B2
:102990007B681B6C03F00103002B01D0002301E0D6
:1029A0006FF0060318460C37BD465DF8047B704790
:1029B00080B483B000AF78607B681B6C03F00203C7
:1029C000002B01D0002301E06FF0060318460C37FE
:1029D000BD465DF8047B704780B483B000AF78607B
:1029E0007B681B6C03F00403002B01D0002301E083
:1029F0006FF0060318460C37BD465DF8047B704740
:102A000080B58AB002AFF860B9607A603B60FB685D
:102A1000824A934208D0FB68814A934201D1012344
:102A200003E04FF0FF3300E00023FB613B68042B21
:102A300002DD6FF00203ECE0FB69002B08D1794B5B
:102A40001B685B08FA6A9A4202D96FF00203E0E061
:102A5000FB69012B07D1734B1B68FA6A9A4202D9B2
:102A60006FF00203D5E000237B766F4B3B6197F854
:102A70003830002B02D00123BB7601E00023BB7667
:102A8000FB68664A934256D10D2001F041FE0620B4
:102A900001F03AFC97F83230002B09D04FF08063F8
:102AA0007B6103233B7607F110031846FEF70CF811
:102AB00097F83330002B09D003233B764FF00063A7
:102AC0007B6107F110031846FDF7FEFF00237B61D1
:102AD00097F83030002B03D07B6943F400037B610F
:102AE00097F83430002B03D07B6943F480037B617B
:102AF00097F83530002B03D07B6943F400137B61DA
:102B000097F83630002B03D07B6943F080737B61EC
:102B100097F83730002B03D07B6943F000737B615B
:102B200097F83130002B03D07B6943F480137B612D
:102B300002233B765DE0FB68394A934256D12B2055
:102B400001F0E6FD302001F0DFFB97F83230002B7A
:102B500009D04FF400637B6103233B7607F1100338
:102B60001846FDF7B1FF97F83330002B09D0032347
:102B70003B764FF480637B6107F110031846FDF745
:102B8000A3FF00237B6197F83030002B03D07B69D3
:102B900043F080037B6197F83430002B03D07B69CE
:102BA00043F040037B6197F83530002B03D07B69FD
:102BB00043F020037B6197F83630002B03D07B690C
:102BC00043F480737B6197F83730002B03D07B6927
:102BD00043F400737B6197F83130002B03D07B699D
:102BE00043F010037B6102233B7602E06FF00103A8
:102BF0000FE007F110031846FDF766FFFB6A01932B
:102C0000BB6A00933B687A68B968F86800F080F99D
:102C1000034618462037BD4680BD00BF0060044013
:102C200000E00B40000000200080004080B584B030
:102C300000AF78607B68144A934208D07B68134ADF
:102C4000934201D1012303E04FF0FF3300E0002362
:102C5000FB60786800F028FA7B680B4A934203D146
:102C6000062001F013FB0AE07B68084A934203D177
:102C7000302001F00BFB02E06FF0010300E00023C5
:102C800018461037BD4680BD0060044000E00B4090
:102C900080B485B000AF78607B68294A934204D144
:102CA000284B1B685B08FB603EE07B68264A93422A
:102CB00037D14FF080439B685B0A03F00703BB608A
:102CC000BB68072B2AD801A252F823F0FB2C001076
:102CD0001D2D0010172D0010012D0010ED2C0010DF
:102CE000F32C0010092D0010112D0010174BFB6064
:102CF0001AE04FF4E103FB6016E0154BFB6013E0B4
:102D00004FF4FA53FB600FE04FF40043FB600BE01D
:102D1000104BFB6008E0104BFB6005E06FF0060312
:102D200008E06FF0020305E0FB68DA0F13445B1064
:102D3000FB60FB6818461437BD465DF8047B70479E
:102D4000006004400000002000E00B4000E1F505B9
:102D500000879303C06878040048E80180B582B01A
:102D600000AF786039603968786800F063FA03462C
:102D700018460837BD4680BD80B582B000AF786088
:102D800039603968786800F0BDFA0346184608379C
:102D9000BD4680BD80B582B000AF7860786800F035
:102DA0001BFB034618460837BD4680BD80B582B080
:102DB00000AF786039603968786800F037FB034607
:102DC00018460837BD4680BD80B582B000AF786038
:102DD0000B46FB70FB781946786800F06BFB0346E6
:102DE00018460837BD4680BD80B582B000AF786018
:102DF000786800F0AFFB034618460837BD4680BD33
:102E000080B582B000AF78600B46FB70FB78194646
:102E1000786800F0C3FB034618460837BD4680BDFE
:102E200080B582B000AF7860786800F01BFC034684
:102E300018460837BD4680BD80B582B000AF7860C7
:102E4000786800F03BFC034618460837BD4680BD55
:102E500080B584B000AFF860B9607A607A68B9680C
:102E6000F86800F03FFC034618461037BD4680BDA9
:102E700080B582B000AF7860786800F09DFC0346B2
:102E800018460837BD4680BD80B584B000AFF860F5
:102E9000B9607A607A68B968F86800F09CFC03460B
:102EA00018461037BD4680BD80B582B000AF78604F
:102EB000786800F0EEFC034618460837BD4680BD32
:102EC00080B582B000AF786039603968786800F00A
:102ED000F1FC034618460837BD4680BD80B582B078
:102EE00000AF786039603968786800F000FD03460B
:102EF00018460837BD4680BD80B582B000AF786007
:102F0000786800F0B3FF034618460837BD4680BD19
:102F100080B586B000AFF860B9607A603B60FB684E
:102F20005D4A934208D0FB685C4A934201D1012379
:102F300003E04FF0FF3300E000237B6158497A69DA
:102F400013469B001344DB000B4400221A605449D3
:102F50007A6913469B001344DB000B4408330022BC
:102F60001A604F497A6913469B001344DB000B44F7
:102F70000C3301221A604A497A6913469B001344B4
:102F8000DB000B44103300221A6045497A6913466E
:102F90009B001344DB000B441C3300221A604049A1
:102FA0007A6913469B001344DB000B442033002254
:102FB0001A603B497A6913469B001344DB000B44BB
:102FC00014336FF001021A6035497A6913469B0089
:102FD0001344DB000B4418336FF001021A60FB68E6
:102FE00001225A60FB682F4A1A61BB68002B06D089
:102FF000FB685B6843F00202FB685A6005E0FB680F
:103000005B6823F00202FB685A60796AF868FFF790
:10301000A5FE3B6AFF2B02D96FF0020338E0FB6884
:10302000DA683B6A1B041A43FB68DA60FB681A6AB9
:10303000FB681A623B68012B05D1FB685B6843F4AF
:103040008032FB685A603B68022B05D1FB685B68E5
:1030500043F44032FB685A603B68032B05D1FB68A0
:103060005B6843F4E022FB685A603B68042B05D19F
:10307000FB685B6843F47022FB685A607B68002B36
:1030800005D0FB68DB6843F40052FB68DA6000237C
:1030900018461837BD4680BD0060044000E00B4074
:1030A000D81000200101010080B584B000AF786025
:1030B0007B685D4A934208D07B685C4A934201D1A9
:1030C000012303E04FF0FF3300E00023FB607B6847
:1030D00000225A627B681A6A7B681A627B685B68A6
:1030E00023F001027B685A607B68DB6923F04012A1
:1030F0007B68DA617B684C4A934208D07B684B4A14
:10310000934201D1012303E04FF0FF3300E000239D
:10311000FB604749FA6813469B001344DB000B44ED
:103120001B68002B2AD04249FA6813469B001344BF
:10313000DB000B441B68BB60FA6813469B0013441A
:10314000DB003B4A1344184601F03CF83849FA6862
:1031500013469B001344DB000B441B685B6A002B87
:103160000CD03349FA6813469B001344DB000B4430
:103170001B685B6A6FF00E01B86898477B68002295
:103180005A607B6800229A607B680022DA607B6864
:1031900000221A612649FA6813469B001344DB009B
:1031A0000B4414331B68002B16DB2149FA681346C5
:1031B0009B001344DB000B4414331B681846FDF7D7
:1031C0000FFB1B49FA6813469B001344DB000B44BA
:1031D00014336FF001021A601549FA6813469B0018
:1031E0001344DB000B4418331B68002B16DB10491B
:1031F000FA6813469B001344DB000B4418331B682A
:103200001846FDF7EDFA0A49FA6813469B00134485
:10321000DB000B4418336FF001021A6000231846DC
:103220001037BD4680BD00BF0060044000E00B4089
:10323000D810002080B586B000AF78603960304B80
:103240001B685B083A689A4202D96FF0020353E0A8
:103250007868FFF71DFD0346BB60BA683B68B2FBA8
:10326000F3F3BB60BB685B087B61BB685B083B61D9
:103270000023FB60BB6803F00103002B10D07B69C7
:1032800001337B610CE07B69DA0F13445B107B61D7
:103290003B69DA0F13445B103B61FB680133FB6051
:1032A0007B690F2B02DDFB68072BECDDFB68082B2D
:1032B00003D10F233B610F237B617B685B6923F0A4
:1032C000FF023B69DBB21A437B685A617B685B692A
:1032D00023F47F427B691B029BB21A437B685A61CD
:1032E0007B685B6923F47022FB681B0403F4702382
:1032F0001A437B685A61002318461837BD4680BDC3
:103300000000002080B485B000AF786039603B6871
:10331000012B02D03B68102B02DD6FF002034EE060
:103320007B682A4A934208D07B68294A934201D19C
:10333000012303E04FF0FF3300E00023FB607B68D4
:103340001B6B03F00103002B37D12249FA681346A7
:103350009B001344DB000B440C331B68012B2CD166
:103360007B685B6823F001027B685A603968194802
:10337000FA6813469B001344DB00034408331960CA
:103380003B680F2B0BDC7B68DB6823F470623B68C7
:103390001B0203F470631A437B68DA6005E07B6804
:1033A000DB6823F470627B68DA607B685B6843F0FB
:1033B00001027B685A60002301E06FF006031846A3
:1033C0001437BD465DF8047B704700BF00600440C1
:1033D00000E00B40D810002080B485B000AF7860CA
:1033E0007B68104A934208D07B680F4A934201D110
:1033F000012303E04FF0FF3300E00023FB607B6814
:10340000DB6803F47063002B01D1102304E07B68B8
:10341000DB681B0A03F00F0318461437BD465DF83E
:10342000047B70470060044000E00B4080B485B02E
:1034300000AF786039603B68032B02DD6FF0020358
:103440002EE07B685B6803F00203002B02D16FF073
:10345000060325E07B68154A934208D07B68144A2E
:10346000934201D1012303E04FF0FF3300E000233A
:10347000FB607B685B6801213A6801FA02F2120482
:103480001A437B685A607B685A6801213B6801FADD
:1034900003F31B0463F470231A407B685A60002313
:1034A00018461437BD465DF8047B70470060044041
:1034B00000E00B4080B485B000AF78600B46FB7035
:1034C0007B68224A934208D07B68214A934201D10B
:1034D000012303E04FF0FF3300E00023FB607B6833
:1034E000DB6823F430427B68DA60FB78032B25D855
:1034F00001A252F823F000BF093500101735001063
:10350000213500102F3500107B68DB6843F4004242
:103510007B68DA6012E07B68DA687B68DA600DE06D
:103520007B68DB6843F480527B68DA6006E07B6886
:10353000DB6843F400527B68DA6000BF0023184662
:103540001437BD465DF8047B704700BF006004403F
:1035500000E00B4080B483B000AF78607B68DB682C
:1035600003F40043002B01D0002310E07B68DB68EC
:1035700003F48053002B01D0022308E07B68DB6852
:1035800003F40053002B01D0032300E0012318466D
:103590000C37BD465DF8047B7047000080B485B0F1
:1035A00000AF78600B46FB707B682C4A934208D0D2
:1035B0007B682B4A934201D1012303E04FF0FF3394
:1035C00000E00023FB60FB78032B3FD801A252F8F8
:1035D00023F000BFE5350010FF350010193600104C
:1035E000333600107B68DB6823F001027B68DA6009
:1035F0007B68DB6823F002027B68DA6027E07B6887
:10360000DB6823F001027B68DA607B68DB6843F0EB
:1036100002027B68DA601AE07B68DB6843F0010233
:103620007B68DA607B68DB6823F002027B68DA6023
:103630000DE07B68DB6843F001027B68DA607B6841
:10364000DB6843F002027B68DA6000E000BF002321
:1036500018461437BD465DF8047B7047006004408F
:1036600000E00B4080B584B000AF78607B68114A01
:10367000934208D07B68104A934201D1012303E0B2
:103680004FF0FF3300E00023FB607868FFF7D4FBC6
:10369000034613F1060F02D16FF0050306E07B68C5
:1036A0005B6843F020027B685A600023184610379D
:1036B000BD4680BD0060044000E00B4080B483B094
:1036C00000AF78607B681B6B03F00103002B02D016
:1036D0006FF0050300E0002318460C37BD465DF887
:1036E000047B704780B588B000AFF860B9607A603D
:1036F000BB68002B02D07B68002B01D1002357E070
:10370000F868FFF7B5FBB861F868FFF743FB0346BD
:103710007B617A68BB699A4201D9BB697B607B692E
:10372000082B03D97B6823F001037B600023FB6136
:103730007B69082B36D97B68012B38D932E07B684E
:10374000032B0CD9BA68FB691344FA6812681A6033
:103750007B68043B7B60FB690433FB611CE07B6896
:10376000012B0DD9BA68FB691344FA68128892B22A
:103770001A807B68023B7B60FB690233FB610BE0D4
:10378000FB695A1CFA61BA681344FA681278D2B21B
:103790001A707B68013B7B607B68012B02D17B69DF
:1037A000082B03D87B68002BC9D100E000BFFB6960
:1037B00018462037BD4680BD80B483B000AF786026
:1037C0007B68DB691B0E03F03F0318460C37BD46D0
:1037D0005DF8047B704780B588B000AFF860B960D1
:1037E0007A60BB68002B02D07B68002B01D10023DC
:1037F0004BE0F868FFF758FBB861F868FFF7CAFAC2
:1038000003467B617A68BB699A4201D9BB697B60D8
:103810007B69082B03D97B6823F001037B600023BD
:10382000FB612EE07B68032B0CD9FB68B968FA6951
:103830000A4412681A607B68043B7B60FB690433AE
:10384000FB611EE07B68012B0DD9FB68B968FA6942
:103850000A44128892B21A807B68023B7B60FB6943
:103860000233FB610DE07B69082B0AD8FB695A1C07
:10387000FA61BA6813441A78FB681A707B68013BD6
:103880007B607B68002BCDD1FB6918462037BD4695
:1038900080BD80B483B000AF78607B68DB691B0AB1
:1038A00003F03F03C3F1200318460C37BD465DF813
:1038B000047B704780B483B000AF786039603B68A8
:1038C000202B02D96FF002030BE07B68DB6923F445
:1038D000F8123B681B0403F4F8131A437B68DA619F
:1038E000002318460C37BD465DF8047B704780B452
:1038F00083B000AF786039603B68202B02D96FF04D
:1039000002030AE07B68DB6923F01F023B6803F0D7
:103910001F031A437B68DA61002318460C37BD4643
:103920005DF8047B7047000080B584B000AF78601C
:103930007B681B68994A934209D07B681B68984A48
:10394000934201D1012303E04FF0FF3300E0002355
:10395000FB607B68002B07D07B68DB68002B06D1FF
:103960007B681B69002B02D16FF0020312E17B68B8
:103970005B69B3F5803F02D36FF002030AE17B6815
:103980001B681846FFF706FA0346FB727B680022A5
:10399000DA617B6800221A628249FA6813469B004A
:1039A0001344DB000B447A681A607E49FA681346B8
:1039B0009B001344DB000B44043300221A60794956
:1039C000FA6813469B001344DB000B4425330022A6
:1039D0001A707B681B685B6803F00203002B07D03A
:1039E0007B681A687B685B6819461046FFF7DEF94A
:1039F0007B681B69002B17D07B689B69002B13D059
:103A00007B681B689B6899B27B689B691A047B681A
:103A10001B680A439A607B681B68DA697B681B68CD
:103A200042F48002DA610EE07B681B689A687B686A
:103A30001B6892B29A607B681B68DA697B681B68B6
:103A400022F48002DA617B681B681846FFF7CCF924
:103A50000346012B2AD17B681B68DB6803F4004313
:103A6000002B23D17B68DB68002B1FD17B68186992
:103A70004C49FA6813469B001344DB000B44103397
:103A80001B681946FB7A082B03D97B689B695B008E
:103A900001E07B689B691A460CF0F6FE7B681A69A8
:103AA0007B68DA607B689A697B685A617B68DB684F
:103AB000002B18D07B685B69002B14D07B681B68D7
:103AC0009B681B0C1B047A68526991B27A68126871
:103AD0000B4393607B681B68DA697B681B6842F064
:103AE0004002DA610FE07B681B689B687A681268A5
:103AF0001B0C1B0493607B681B68DA697B681B687E
:103B000022F04002DA617B68DB68002B16D07B680C
:103B10005B69002B12D07B681B69002B0ED07B6881
:103B20009B69002B0AD01F49FA6813469B00134477
:103B3000DB000B44243301221A7009E01949FA68AA
:103B400013469B001344DB000B44243300221A70FD
:103B50007B681B68DA697B681B6842F08012DA6157
:103B60007B681B685A687B681B6842F001025A60D8
:103B70007B689B6818460B49FA6813469B00134400
:103B8000DB000B440C3318607B681B684FF4006249
:103B90001A62002318461037BD4680BD00600440FD
:103BA00000E00B40D810002080B584B000AF7860F2
:103BB00039607B68214A934208D07B68204A93424F
:103BC00001D1012303E04FF0FF3300E00023FB604D
:103BD0003B689B68002B05D17B685B6843F480726F
:103BE0007B685A603968786800F02EF8B86015492B
:103BF000FA6813469B001344DB000B4404331B6834
:103C0000002B0CD17868FFF70BF90E49FA681346C0
:103C10009B001344DB000B44043301221A603B6811
:103C20009B68002B05D07B685B6823F480727B68FF
:103C30005A60BB6818461037BD4680BD006004401E
:103C400000E00B40D810002080B588B000AF78604D
:103C500039600023FB610023BB6100237B617B682B
:103C60007E4A934208D07B687D4A934201D101236A
:103C700003E04FF0FF3300E000233B613B681B682B
:103C80001846FFF787F80346FB73FB7B082B08D920
:103C90003B685B695B00BB613B689B695B007B6168
:103CA00005E03B685B69BB613B689B697B613B6886
:103CB000DB68002B12D03B68DA683B68DB69D118FF
:103CC0003B68DB69BA69D31A1A467868FFF7DCF8F3
:103CD00002463B68DB691A443B68DA613B68DB6992
:103CE000BA69D31ABB60BB68002B10D0BB68202B0D
:103CF00004DD20217868FFF7F1F804E0BB6819467D
:103D00007868FFF7EBF8FB6943F00103FB613B6860
:103D10001B69002B20D13B68DB69BA699A421BD131
:103D20007B6800225A620023FB613A6913469B00BC
:103D30001344DB004B4A1344184600F043FA4A4B45
:103D40001B78002B08D03B685B6A002B04D03B68D3
:103D50005B6A0021386898473B681B69002B51D08B
:103D60003B681A693B681B6AD1183B681B6A7A6911
:103D7000D31A1A467868FFF76BF802463B681B6A4D
:103D80001A443B681A623B681B6A7A69D31ABB60A3
:103D9000BB68002B11D0BB68202B04DD02217868A2
:103DA000FFF78EF805E0BB68013B19467868FFF71E
:103DB00087F8FB6943F00403FB613B68DB68002B79
:103DC00020D13B681B6A7A699A421BD17B6800222A
:103DD0005A620023FB613A6913469B001344DB00DF
:103DE000204A1344184600F0EDF91F4B1B78002BB6
:103DF00008D03B685B6A002B04D03B685B6A0021FB
:103E0000386898473B681B6A7A699A4220D13B68B8
:103E1000DB69BA699A421BD17B6800225A6200238F
:103E2000FB613A6913469B001344DB000D4A1344BF
:103E3000184600F0C7F90C4B1B78002B08D03B68E4
:103E40005B6A002B04D03B685B6A002138689847A6
:103E5000FB6918462037BD4680BD00BF00600440A6
:103E600000E00B40D81000207418002080B584B00A
:103E700000AF78607868FFF757FDF860FB68002BAB
:103E800001D0FB6815E00D4B00221A7000BF7B6863
:103E90001B6879681846FFF787FE0346002BF6D1AA
:103EA00000BF7B681B681B6A03F40063002BF8D01B
:103EB000002318461037BD4680BD00BF741800208F
:103EC00080B500AF0F4B1B6803F48033002B16D076
:103ED0000D4B1B68002B05DD0B4B1B68013B0A4A91
:103EE00013600CE000F0F0F8084B1B68002B06D0C4
:103EF000064B1B6800209847044B00221A6000BF45
:103F000080BD00BF10E000E008000020301100205C
:103F1000B0B586B000AF7860334B9B687B61324BA5
:103F20001B6823F48033314A13602F4B1B6803F066
:103F30000103002B11D12C4B6FF07F425A602A4BAA
:103F40006FF07F429A60284B05221A606FF07F4322
:103F50007B614FF080733B6103E0234B5B6801336F
:103F60003B617B6819464FF00002214B1B684FF004
:103F7000000403FB02F501FB04F00544A1FB03016F
:103F80006B1819461B4A4FF000030BF01DFF034648
:103F90000C46FB60FA683B69B2FBF3F31A46164B1A
:103FA0001A60FB683A69B3FBF2F2396901FB02F26D
:103FB0009B1ABB60BA687B699A420CD30E4B1B6894
:103FC00001330D4A13607A69BB68D21A3B69134406
:103FD0000A4A136004E07A69BB68D31A074A13607F
:103FE00000BF1837BD46B0BD10E000E02C11002026
:103FF0000000002040420F0008000020281100208F
:1040000080B582B000AF78603960104A3B681360B9
:104010000F4B1B68002B02DD6FF0050312E07B687D
:10402000002B01D100230DE07868FFF771FF084BEA
:104030001B68002B05DD074B1B68064A43F0020393
:104040001360002318460837BD4680BD301100209C
:104050000800002010E000E080B500AF164B1B68A0
:10406000002B0CDA154B1B68002B06D0134B1B687A
:1040700000209847114B00221A6000231AE00E4BD3
:104080001B68002B14D10E4B9A680E4B1B689A428A
:104090000ED800F019F8094B1B68002B06D0074B0F
:1040A0001B6800209847054B00221A60002301E09E
:1040B0006FF00503184680BD080000203011002075
:1040C00010E000E02811002080B500AF0A4B1B680B
:1040D000002B07D0084B1B686FF00F009847064B6A
:1040E00000221A60054A064B1B681360054B4FF00F
:1040F000FF321A6000BF80BD3011002010E000E0E8
:104100002C1100200800002080B582B000AF78603C
:10411000164B1B68002B02DD6FF0050321E07B6866
:10412000002B01D100231CE07868FFF7F1FE0AE0C4
:104130000F4B1B6803F48033002B04D00B4B1B6820
:10414000013B0A4A1360094B1B68002BF0DC00BFDF
:10415000074B9A68074B1B689A42F9D8FFF7B4FFE0
:10416000002318460837BD4680BD00BF0800002068
:1041700010E000E02811002080B489B000AF786022
:1041800039607B68FB61FB6953E8003FBB61BB6939
:10419000002B02D06FF005030EE03B687B617B686B
:1041A0003B6139697A6941E80023FB60FB68002BB9
:1041B000E7D1BFF35F8F002318462437BD465DF873
:1041C000047B704780B483B000AF7860BFF35F8F2B
:1041D0007B6800221A6000BF0C37BD465DF8047B87
:1041E0007047000080B483B000AF0346FB71FB79D9
:1041F00003F01F03012202FA03F1064A97F9073080
:104200005B0942F8231000BF0C37BD465DF8047B04
:10421000704700BF00E100E080B500AF064A074BE1
:10422000104619464FF4F0731A460CF093FA044BFB
:10423000014A9A6000BF80BD0012002000000010FB
:1042400000ED00E080B584B000AF03463960FB713B
:1042500097F907301033FB600A4B9B680A4A934278
:1042600001D0FFF7D9FF0849FB683A6841F82320DD
:1042700097F907301846FFF7B5FF00BF1037BD4666
:1042800080BD00BF00ED00E00012002080B483B0CC
:1042900000AF0346FB71FB793F2B0DD9FB79403B07
:1042A000FB71184BDB68FA79012101FA02F2114621
:1042B000144A0B43D3601EE0FB791F2B0FD9FB7907
:1042C000203BFB714FF080439B6CFA79012101FA8E
:1042D00002F211464FF080420B4393640BE04FF023
:1042E00080435B6AFA79012101FA02F211464FF02C
:1042F00080420B43536200BF0C37BD465DF8047B20
:10430000704700BF0000084080B483B000AF034690
:10431000FB71FB793F2B0ED9FB79403BFB71194BAD
:10432000DB68FA79012101FA02F2D2431146154AFB
:104330000B40D36020E0FB791F2B10D9FB79203B89
:10434000FB714FF080439B6CFA79012101FA02F274
:10435000D24311464FF080420B4093640CE04FF083
:1043600080435B6AFA79012101FA02F2D2431146D5
:104370004FF080420B40536200BF0C37BD465DF8E2
:10438000047B70470000084080B582B000AF034650
:10439000FB71FB79023B052B5BD801A252F823F09D
:1043A00003440010F7430010B9430010D543001038
:1043B00037440010F14300104FF080439B684FF0EA
:1043C000804243F4002393604FF0006000F04AF80D
:1043D000034640E04FF080439B684FF0804243F437
:1043E000801393604FF0805000F03CF8034632E0B9
:1043F0006FF010032FE04FF0005000F033F8034649
:1044000029E04FF080435B6F4FF0804243F011038F
:104410005367134B42F288129A614FF080439B68B6
:104420004FF0804243F4803393604FF0807000F08F
:1044300019F803460FE04FF080439B684FF080422D
:1044400043F4003393604FF0007000F00BF8034624
:1044500001E06FF0020318460837BD4680BD00BF7B
:104460000008004080B582B000AF786000214FF4B2
:104470007A70FFF7C5FD4FF080439A687B68134060
:10448000002B03D0FFF720FE002307E0FFF7E4FD39
:10449000034613F1060FEED06FF0090318460837F4
:1044A000BD4680BD80B584B000AF0346FB714FF0C0
:1044B00080439B6803F46063FB60FB79072B00F289
:1044C000D98001A252F823F0E9440010754600108B
:1044D000CF450010174600102D45001075450010FF
:1044E0002D460010BD4500104FF080439B6803F43B
:1044F0008023002B11D14FF080439B684FF0804206
:1045000043F4802393604FF08060FFF7ABFF0346D6
:10451000002B02D06FF00903C8E04FF080439B6886
:104520004FF0804223F460639360A6E04FF0804335
:104530009B6803F40023002B11D14FF080439B684C
:104540004FF0804243F4002393604FF00060FFF788
:1045500089FF0346002B02D06FF00903A6E04FF05D
:1045600080439B6823F460634FF0804243F4006310
:10457000936082E04FF080439B6803F48013002B2C
:1045800011D14FF080439B684FF0804243F4801379
:1045900093604FF08050FFF765FF0346002B02D079
:1045A0006FF0090382E04FF080439B6823F460635F
:1045B0004FF0804243F4206393605EE04FF080430D
:1045C0009B684FF0804243F46063936055E04FF086
:1045D00080439B6803F48033002B11D14FF080435C
:1045E0009B684FF0804243F4803393604FF08070BB
:1045F000FFF738FF0346002B02D06FF0090355E0A8
:104600004FF080439B6823F460634FF0804243F493
:104610008063936031E04FF080439B6823F46063D4
:104620004FF0804243F4C063936026E04FF0804334
:104630009B6803F40033002B11D14FF080439B683B
:104640004FF0804243F4003393604FF00070FFF767
:1046500009FF0346002B02D06FF0090326E04FF05C
:1046600080439B6823F460634FF0804243F44063CF
:10467000936002E06FF0020318E04FF40050FFF780
:10468000F1FE0346002B0ED04FF080439B6823F4CD
:104690006062FB6803F460634FF0804113438B60FA
:1046A0006FF0090302E0FBF707FE002318461037FE
:1046B000BD4680BD80B582B000AF0346FB8000F0F0
:1046C00018F803461A46FB8893420ED04FF08043F9
:1046D0009B6823F4E072FB8803F4E0734FF08041A1
:1046E00013438B60FBF7E8FD00E000BF0837BD46D1
:1046F00080BD80B400AF4FF080439B689BB203F451
:10470000E0739BB21846BD465DF8047B704700001D
:1047100080B483B000AF0346FB71FB793F2B12D905
:10472000FB79403BFB71FB7901229A401D4B9A605B
:1047300000BF1C4B9B68FA79012101FA02F2134079
:10474000002BF6D128E0FB791F2B14D9FB79203BF5
:10475000FB71FB7901229A404FF080435A6400BFFD
:104760004FF080435B6CFA79012101FA02F21340A9
:10477000002BF5D110E0FB7901229A404FF08043E5
:104780005A6000BF4FF080435B68FA79012101FA5B
:1047900002F21340002BF5D100BF0C37BD465DF887
:1047A000047B70470000084080B586B000AFF86019
:1047B000B9601346FB71FB687D4A934220D0FB68C9
:1047C0007C4A93421AD0FB687B4A934214D0FB6820
:1047D0007A4A93420ED0FB68794A934208D0FB682C
:1047E000784A934201D105230BE04FF0FF3308E0F4
:1047F000042306E0032304E0022302E0012300E097
:1048000000233B610023FB75BB68002B02D14FF0F6
:10481000FF33C9E0BB68DB78023B032B41D801A220
:1048200052F823F0354800104D480010654800103C
:104830008B4800103B69032B02DD6FF01003B3E0DF
:104840000123FB750220FFF79FFD2BE03B69032B43
:1048500002DD6FF01003A7E00223FB750520FFF7D0
:1048600093FD1FE03B69042B02D10123FB7508E097
:104870003B69032B02DC0323FB7502E06FF010039E
:1048800092E00620FFF780FD0CE03B69032B02DC81
:104890006FF0100388E00223FB750320FFF774FD1F
:1048A00000E000BF3B69052B77D801A252F823F046
:1048B000C9480010F34800101D4900104749001076
:1048C000714900107F4900100520FFF721FF0F20DC
:1048D000FFF71AFDFB79002B58D0BB689B78022BA1
:1048E00003D03948FCF7F0F850E03848FCF7ECF812
:1048F0004CE00620FFF70CFF1020FFF705FDFB79C9
:10490000002B45D0BB689B78022B03D03048FCF7C6
:10491000DBF83DE02F48FCF7D7F839E00720FFF738
:10492000F7FE1120FFF7F0FCFB79002B32D0BB68BB
:104930009B78022B03D02848FCF7C6F82AE02748CA
:10494000FCF7C2F826E00820FFF7E2FE1220FFF78E
:10495000DBFCFB79002B1FD0BB689B78022B03D0BC
:104960001F48FCF7B1F817E01E48FCF7ADF813E05C
:104970004220FFF7CDFE4220FFF7C6FC0DE04320AA
:10498000FFF7C6FE4320FFF7BFFC06E000BF04E0D0
:1049900000BF02E000BF00E000BFFB7D1A46B9681F
:1049A000F86800F0B5F8034618461837BD4680BDD4
:1049B0000000014000100140002001400030014093
:1049C000000C084000100840EC650110F86501106B
:1049D00004660110106601101C66011028660110A3
:1049E000346601104066011080B582B000AF786077
:1049F000786800F01BFA7B68164A934202D10F20B8
:104A0000FFF744FC7B68144A934202D11020FFF761
:104A10003DFC7B68114A934202D11120FFF736FC1E
:104A20007B680F4A934202D11220FFF72FFC7B686C
:104A30000C4A934202D14220FFF728FC7B680A4AC5
:104A4000934202D14320FFF721FC00BF0837BD4647
:104A500080BD00BF00000140001001400020014067
:104A600000300140000C08400010084080B582B0C2
:104A700000AF7860786800F021FA00BF0837BD46C3
:104A800080BD80B582B000AF7860786800F060FAD1
:104A900000BF0837BD4680BD80B582B000AF7860EA
:104AA00039603968786800F097FA03461846083785
:104AB000BD4680BD80B582B000AF7860786800F0F8
:104AC000E3FA00BF0837BD4680BD80B582B000AFB5
:104AD0007860786800F01CFB00BF0837BD4680BDD9
:104AE00080B582B000AF7860786800F055FB00BFF9
:104AF0000837BD4680BD80B582B000AF78603960B0
:104B00003968786800F08CFB00BF0837BD4680BD6F
:104B100080B586B000AFF860B9601346FB71FB68E2
:104B2000644A934220D0FB68634A93421AD0FB68E0
:104B3000624A934214D0FB68614A93420ED0FB68EC
:104B4000604A934208D0FB685F4A934201D1052333
:104B50000BE04FF0FF3308E0042306E0032304E0FA
:104B6000022302E0012300E000233B61BB68002B2D
:104B700002D14FF0FF3399E0BB689B78022B02D142
:104B800010237B6101E000237B61BB689B7803F00D
:104B90000303002B06D0FB689B6923F00042FB68EF
:104BA0009A6105E0FB689B6943F00042FB689A61EB
:104BB000FB68DB6843F00112FB68DA60FB681B6985
:104BC000BA68127811467A6901FA02F21A43FB6850
:104BD0001A61FB689B69F9797A6901FA02F21A4352
:104BE000FB689A61BB685B78072B5ED801A252F81C
:104BF00023F000BF154C00101F4C0010294C001072
:104C0000934C0010414C0010594C0010634C0010A4
:104C10007B4C0010B968F86800F058F845E0B968B6
:104C2000F86800F053F840E0BB689B78022B02D193
:104C30006FF010033AE0B968F86800F047F834E024
:104C4000BB689B78022B02D16FF010032EE0B9688D
:104C5000F86800F03BF828E0B968F86800F036F82A
:104C600023E0BB689B78022B02D16FF010031DE09C
:104C7000B968F86800F02AF817E0BB689B78022B47
:104C800002D16FF0100311E0B968F86800F01EF867
:104C90000BE0BB689B78022B02D16FF0100305E09C
:104CA000B968F86800F012F800BF002318461837FA
:104CB000BD4680BD000001400010014000200140C1
:104CC00000300140000C08400010084080B485B05E
:104CD00000AF786039607B684E4A934220D07B6891
:104CE0004D4A93421AD07B684C4A934214D07B6859
:104CF0004B4A93420ED07B684A4A934208D07B6865
:104D0000494A934201D105230BE04FF0FF3308E0FD
:104D1000042306E0032304E0022302E0012300E071
:104D20000023BB603B68002B6DD03B689B78022B57
:104D300002D11023FB6001E00023FB607B681A694D
:104D40004FF48041FB6801FA03F31A437B681A6150
:104D500000BF7B689A690821FB6801FA03F31340DE
:104D6000002BF6D07B681B693A6852781146FA68C6
:104D700001FA02F21A437B681A617B681A693B6880
:104D80009B681902FB6801FA03F31A437B681A61F6
:104D90000122FB6802FA03F31A467B681A6000BF1F
:104DA0007B68DA684FF48071FB6801FA03F3134003
:104DB000002BF5D03B685A68FB689A407B685A60C4
:104DC0007B689A694FF40051FB6801FA03F3DB43F7
:104DD0001A407B689A613B689B78022B14D17B68F0
:104DE0009B6943F080727B689A617B681B6943F022
:104DF00000427B681A6100BF7B689B6903F48023D3
:104E0000002BF9D000E000BF1437BD465DF8047BED
:104E1000704700BF00000140001001400020014029
:104E200000300140000C08400010084080B485B0FC
:104E300000AF78607B681B4A934220D07B681A4A97
:104E400093421AD07B68194A934214D07B68184A5F
:104E500093420ED07B68174A934208D07B68164A6B
:104E6000934201D105230BE04FF0FF3308E0042308
:104E700006E0032304E0022302E0012300E0002314
:104E8000FB607B6800221A6100BF7B689B6903F0AE
:104E90000803002BF9D100BF1437BD465DF8047B31
:104EA000704700BF00000140001001400020014099
:104EB00000300140000C08400010084080B485B06C
:104EC00000AF78607B681C4A934220D07B681B4A05
:104ED00093421AD07B681A4A934214D07B68194ACD
:104EE00093420ED07B68184A934208D07B68174AD9
:104EF000934201D105230BE04FF0FF3308E0042378
:104F000006E0032304E0022302E0012300E0002383
:104F1000FB607B681B6943F400427B681A6100BF39
:104F20007B689B6903F00403002BF9D000BF1437A2
:104F3000BD465DF8047B7047000001400010014051
:104F40000020014000300140000C084000100840E3
:104F500080B485B000AF78607B68194A934220D056
:104F60007B68184A93421AD07B68174A934214D040
:104F70007B68164A93420ED07B68154A934208D04C
:104F80007B68144A934201D105230BE04FF0FF33B5
:104F900008E0042306E0032304E0022302E00123E7
:104FA00000E00023FB607B681B6923F400427B6800
:104FB0001A6100BF1437BD465DF8047B704700BF1F
:104FC000000001400010014000200140003001407D
:104FD000000C08400010084080B485B000AF786035
:104FE00039607B68224A934220D07B68214A9342F1
:104FF0001AD07B68204A934214D07B681F4A9342A0
:105000000ED07B681E4A934208D07B681D4A9342AB
:1050100001D105230BE04FF0FF3308E0042306E045
:10502000032304E0022302E0012300E00023FB60ED
:105030007B685B683A689A4202D96FF0020310E01D
:1050400000BF7B681B683A689A42FAD97B683A6865
:105050009A6000BF7B68DB6803F48073002BF9D093
:10506000002318461437BD465DF8047B704700BF27
:1050700000000140001001400020014000300140CC
:10508000000C08400010084080B485B000AF786084
:105090007B68194A934220D07B68184A93421AD001
:1050A0007B68174A934214D07B68164A93420ED00D
:1050B0007B68154A934208D07B68144A934201D119
:1050C00005230BE04FF0FF3308E0042306E0032341
:1050D00004E0022302E0012300E00023FB607B6880
:1050E000DB6843F001127B68DA6000BF1437BD460D
:1050F0005DF8047B704700BF0000014000100140D4
:105100000020014000300140000C08400010084021
:1051100080B485B000AF78607B68194A934220D094
:105120007B68184A93421AD07B68174A934214D07E
:105130007B68164A93420ED07B68154A934208D08A
:105140007B68144A934201D105230BE04FF0FF33F3
:1051500008E0042306E0032304E0022302E0012325
:1051600000E00023FB607B689B6943F001227B68C1
:105170009A6100BF1437BD465DF8047B704700BFDD
:1051800000000140001001400020014000300140BB
:10519000000C08400010084080B485B000AF786073
:1051A0007B68194A934220D07B68184A93421AD0F0
:1051B0007B68174A934214D07B68164A93420ED0FC
:1051C0007B68154A934208D07B68144A934201D108
:1051D00005230BE04FF0FF3308E0042306E0032330
:1051E00004E0022302E0012300E00023FB607B686F
:1051F0009B6923F001227B689A6100BF1437BD468A
:105200005DF8047B704700BF0000014000100140C2
:105210000020014000300140000C08400010084010
:1052200080B485B000AF786039607B681A4A9342D9
:1052300020D07B68194A93421AD07B68184A93425F
:1052400014D07B68174A93420ED07B68164A93426B
:1052500008D07B68154A934201D105230BE04FF03B
:10526000FF3308E0042306E0032304E0022302E006
:10527000012300E00023FB607B683A681A6000BFEE
:105280007B68DB6803F48073002BF9D000BF143710
:10529000BD465DF8047B70470000014000100140EE
:1052A0000020014000300140000C08400010084080
:1052B00080B582B000AF786000BF786800F0F2FB84
:1052C0000346002BF9D0786800F084FB03461846AB
:1052D0000837BD4680BD80B582B000AF78600B4610
:1052E000FB7000BF786800F0F9FB0346002BF9D093
:1052F000FB781946786800F079FB034618460837B2
:10530000BD4680BD80B582B000AF78603960396835
:10531000786801F0C3FA034618460837BD4680BDD9
:1053200080B582B000AF7860786801F051FB034629
:1053300018460837BD4680BD80B586B000AFF8601E
:10534000B9601346FB71F86800F076F878617B6904
:10535000002B01D07B695BE0FB79022B05D0042B8D
:1053600007D10620FFF710F804E00520FFF70CF83E
:1053700000E000BFFB68284A934214D0FB68274A2C
:1053800093420ED0FB68264A934208D0FB68254A18
:10539000934201D1032307E04FF0FF3304E00223DF
:1053A00002E0012300E00023032B27D801A252F8DA
:1053B00023F000BFC5530010D3530010E153001079
:1053C000EF5300101848FBF77FFB0920FEF79CFF06
:1053D00017E01648FBF778FB0A20FEF795FF10E070
:1053E0001348FBF771FB2120FEF78EFF09E01148FF
:1053F000FBF76AFB4420FEF787FF02E06FF0020331
:1054000006E0FB791A46B968F86800F019FC034613
:1054100018461837BD4680BD0020044000300440C7
:1054200000400440001408407465011098650110A4
:10543000BC650110E065011080B582B000AF7860F6
:105440007B68254A934214D07B68244A93420ED04D
:105450007B68234A934208D07B68224A934201D159
:10546000032307E04FF0FF3304E0022302E00123AF
:1054700000E00023032B27D801A252F823F000BF3D
:10548000915400109F540010AD540010BB540010F4
:105490000B20FFF73DF90920FEF7F8FE17E00C207E
:1054A000FFF736F90A20FEF7F1FE10E01C20FFF7A7
:1054B0002FF92120FEF7EAFE09E04420FFF728F942
:1054C0004420FEF7E3FE02E06FF0020300E0002359
:1054D00018460837BD4680BD002004400030044017
:1054E000004004400014084080B588B000AFF86068
:1054F000B9601346FB710023BB6100237B61FB682D
:105500008A4A93420ED0FB68894A93420AD0FB68CC
:10551000884A934206D0FB68874A934202D06FF0D4
:105520000203FFE0FB68844A934267D1FB680522CF
:105530005A61FB79022B02D0042B11D048E04FF4C2
:10554000E102BB68B2FBF3F37B614FF4E103BA689D
:10555000B3FBF2F2B96801FB02F29B1ABB613AE0BD
:10556000BB68B3F5165F02D96FF01003DAE0FB6891
:105570001B6843F48032FB681A60FB681B6843F4C5
:105580000012FB681A60BB68B3F5165F04D10723ED
:105590007B610023BB610FE04FF48032BB68B2FB3C
:1055A000F3F37B614FF48033BA68B3FBF2F2B9686E
:1055B00001FB02F29B1ABB61BB68B3F5166F03D9FE
:1055C000FB6800225A6106E0FB6801225A6102E092
:1055D0006FF00203A6E07B69002B04D0BB685B0878
:1055E000BA699A4202D97B6901337B61FB687A69A7
:1055F0001A61F86800F0A6F8F86182E000237B6188
:105600000023BB61FB68494A93420ED0FB68484ABD
:1056100093420AD0FB68474A934206D0FB68464A49
:10562000934202D06FF002037CE0FB6805225A61CE
:10563000FB79032B50D801A252F823F04D560010ED
:105640007356001081560010AF5600103B4B1B687C
:105650005A08BB68B2FBF3F37B61384B1B685B08ED
:10566000BA68B3FBF2F2B96801FB02F29B1ABB61A4
:1056700035E0FB681B6843F48032FB681A602EE05B
:105680004FF4E102BB68B2FBF3F37B614FF4E1033B
:10569000BA68B3FBF2F2B96801FB02F29B1ABB6174
:1056A000FB681B6843F40032FB681A6017E0244A69
:1056B000BB68B2FBF3F37B61214BBA68B3FBF2F238
:1056C000B96801FB02F29B1ABB61FB681B6843F4DB
:1056D0004032FB681A6002E06FF0020322E07B694F
:1056E000002B04D0BB685B08BA699A4202D97B6977
:1056F00001337B61FB687A691A61F86800F022F86F
:10570000F861FB69002B0CDDFB681B6843F4004269
:10571000FB681A6000BFFB681B6803F40023002BC2
:10572000F9D0FB6918462037BD4680BD00200440F3
:1057300000300440004004400014084000000020F5
:105740000048E80180B485B000AF78600023FB60BA
:105750007B683F4A93420ED07B683E4A93420AD010
:105760007B683D4A934206D07B683C4A934202D014
:105770006FF0020366E07B68384A93421DD17B6874
:105780001B6803F44033B3F5803F03D14FF48033FB
:10579000FB600CE07B681B6803F44033002B03D1F3
:1057A0004FF4E103FB6002E06FF002034AE0FA68A5
:1057B0007B681B69B2FBF3F344E07B68244A9342A5
:1057C0000ED07B68234A93420AD07B68224A9342D8
:1057D00006D07B68214A934202D06FF0020331E089
:1057E0007B681B6803F44033B3F5803F02D16FF050
:1057F000100327E07B681B6803F44033002B04D1BF
:10580000174B1B685B08FB6017E07B681B6803F4A1
:105810004033B3F5003F03D14FF4E103FB600CE0EC
:105820007B681B6803F44033B3F5403F02D10D4B56
:10583000FB6002E06FF0020304E0FA687B681B691A
:10584000B2FBF3F318461437BD465DF8047B70478E
:105850000020044000300440004004400014084090
:10586000000000200048E80180B582B000AF7860F9
:1058700039603968786800F03FFA034618460837FF
:10588000BD4680BD80B582B000AF78600B46FB702E
:10589000FB781946786800F06DFA03461846083719
:1058A000BD4680BD80B582B000AF78600B46FB700E
:1058B000FB781946786800F09DFA034618460837C9
:1058C000BD4680BD80B584B000AFF8600B467A60FD
:1058D000FB72FB7A012B2ED1FB68344A934214D021
:1058E000FB68334A93420ED0FB68324A934208D099
:1058F000FB68314A934201D1032307E04FF0FF33A5
:1059000004E0022302E0012300E00023012B07D082
:10591000022B09D0002B0BD12848FBF7D5F839E032
:105920002748FBF7D1F835E02648FBF7CDF831E002
:105930006FF0020335E0FB681C4A934214D0FB6809
:105940001B4A93420ED0FB681A4A934208D0FB6868
:10595000194A934201D1032307E04FF0FF3304E0DB
:10596000022302E0012300E00023012B07D0022BD9
:1059700009D0002B0BD11448FBF7A6F80AE0134816
:10598000FBF7A2F806E01248FBF79EF802E06FF082
:10599000020306E0FB7A7A681946F86800F0BAFA62
:1059A000034618461037BD4680BD00BF00200440A6
:1059B000003004400040044000140840806501109D
:1059C000A4650110C86501108C650110B065011057
:1059D000D465011080B582B000AF7860786800F0BF
:1059E000D9FA034618460837BD4680BD80B582B057
:1059F00000AF78600B46FB70FB781946786800F0C2
:105A0000F9FA034618460837BD4680BD80B582B016
:105A100000AF78607868FFF74BFC034618460837FC
:105A2000BD4680BD80B582B000AF78600B46FB708C
:105A3000FB7819467868FFF74EFC0346184608378E
:105A4000BD4680BD80B584B000AFF860B9607A60B3
:105A50007A68B968F86800F001FB03461846103709
:105A6000BD4680BD80B584B000AFF860B9607A6093
:105A70007A68B968F86800F043FB034618461037A7
:105A8000BD4680BD80B584B000AFF860B9607A6073
:105A90007A68B968F86800F083FB03461846103747
:105AA000BD4680BD80B582B000AF7860786800F0F8
:105AB0009DFB034618460837BD4680BD80B584B0BF
:105AC00000AFF860B9607A607A68B968F86800F089
:105AD0009CFB034618461037BD4680BD80B582B09A
:105AE00000AF7860786800F0B6FB034618460837C8
:105AF000BD4680BD80B582B000AF7860786800F0A8
:105B0000BDFB034618460837BD4680BD80B582B050
:105B100000AF786039603968786800F0E3FB0346CD
:105B200018460837BD4680BD80B582B000AF7860AA
:105B3000786800F011FC034618460837BD4680BD62
:105B400080B582B000AF7860786800F013FC03463F
:105B500018460837BD4680BD80B582B000AF78607A
:105B600039603968786800F011FC03461846083738
:105B7000BD4680BD80B582B000AF786039603968BD
:105B8000786800F02DFC034618460837BD4680BDF6
:105B900080B582B000AF786039603968786800F00D
:105BA0004DFC034618460837BD4680BD80B582B01F
:105BB00000AF7860786800F06FFC0346184608373D
:105BC000BD4680BD80B582B000AF7860786800F0D7
:105BD0006FFC034618460837BD4680BD80B582B0CD
:105BE00000AF7860786800F01DFF0346184608375C
:105BF000BD4680BD80B582B000AF7860786800F0A7
:105C00003DFF034618460837BD4680BD80B483B0CB
:105C100000AF0346FB71FB7903F01F03012202FA78
:105C200003F1064A97F907305B09403342F8231025
:105C300000BF0C37BD465DF8047B704700E100E013
:105C400080B586B000AFF860B9601346FB71FB68A1
:105C5000254A93420ED0FB68244A93420AD0FB683F
:105C6000234A934206D0FB68224A934202D06FF047
:105C7000020334E00121F868FFF748FF78617B698F
:105C8000002B01D07B692AE00821F868FFF7ECFDC2
:105C900078617B69002B01D07B6920E00021F868E6
:105CA000FFF700FE78617B69002B01D07B6916E06D
:105CB0000021F868FFF7E6FD78617B69002B01D0D1
:105CC0007B690CE0FB791A46B968F868FFF70CFCB1
:105CD00078617B69002B01DA7B6900E000231846BC
:105CE0001837BD4680BD00BF00200440003004408E
:105CF000004004400014084080B483B000AF7860D6
:105D000039607B68174A93420ED07B68164A9342EB
:105D10000AD07B68154A934206D07B68144A9342A6
:105D200002D06FF0020317E03B68042B02DD3B68F2
:105D3000082B02DD6FF002030EE03B68053B9B027F
:105D40003B607B681B6823F440623B6803F440635C
:105D50001A437B681A60002318460C37BD465DF86D
:105D6000047B7047002004400030044000400440A1
:105D70000014084080B483B000AF78600B46FB701D
:105D80007B68184A93420ED07B68174A93420AD028
:105D90007B68164A934206D07B68154A934202D02C
:105DA0006FF0020317E0FB78002B02D0012B07D025
:105DB0000DE07B681B6823F480527B681A6009E061
:105DC0007B681B6843F480527B681A6002E06FF0C6
:105DD000020300E0002318460C37BD465DF8047B43
:105DE000704700BF002004400030044000400440E1
:105DF0000014084080B483B000AF78600B46FB709D
:105E00007B68404A93420ED07B683F4A93420AD057
:105E10007B683E4A934206D07B683D4A934202D05B
:105E20006FF0020367E0FB78042B60D801A252F800
:105E300023F000BF495E0010575E00107D5E001029
:105E4000A35E0010C95E00107B681B6823F010027F
:105E50007B681A604EE07B681B6843F010027B6829
:105E60001A607B681B6823F020027B681A607B68DD
:105E70001B6823F040027B681A603BE07B681B686C
:105E800043F010027B681A607B681B6823F02002D5
:105E90007B681A607B681B6843F040027B681A606D
:105EA00028E07B681B6843F010027B681A607B68FF
:105EB0001B6843F020027B681A607B681B6823F034
:105EC00040027B681A6015E07B681B6843F0100293
:105ED0007B681A607B681B6843F020027B681A604D
:105EE0007B681B6843F040027B681A6002E06FF039
:105EF000020300E0002318460C37BD465DF8047B22
:105F0000704700BF002004400030044000400440BF
:105F10000014084080B485B000AFF8600B467A608A
:105F2000FB72FB68174A93420ED0FB68164A9342F5
:105F30000AD0FB68154A934206D0FB68144A934284
:105F400002D06FF0020317E0FB7A002B02D0012B86
:105F500007D00DE0FB681B6823F40052FB681A6051
:105F600009E0FB681B6843F40052FB681A6002E01A
:105F70006FF0020300E0002318461437BD465DF8B9
:105F8000047B70470020044000300440004004407F
:105F90000014084080B483B000AF78607B68114A79
:105FA00093420ED07B68104A93420AD07B680F4A16
:105FB000934206D07B680E4A934202D06FF00203F0
:105FC0000AE07B685B6803F01003002B02D06FF0DF
:105FD0000C0301E07B681B6A18460C37BD465DF870
:105FE000047B70470020044000300440004004401F
:105FF0000014084080B483B000AF78600B46FB709B
:106000007B68124A93420ED07B68114A93420AD0B1
:106010007B68104A934206D07B680F4A934202D0B5
:106020006FF002030CE07B685B6803F08003002BD9
:1060300002D06FF00B0303E0FA787B681A6200234A
:1060400018460C37BD465DF8047B704700200440BD
:1060500000300440004004400014084080B586B081
:1060600000AFF860B9607A6000237B61FB68204A6A
:1060700093420ED0FB681F4A93420AD0FB681E4A27
:10608000934206D0FB681D4A934202D06FF0020390
:1060900029E0BB68002B02D14FF0FF3323E07B687F
:1060A000002B17D14FF0FF331DE0F868FFF7AEFC6F
:1060B00038613B69002B04DA7B687A691A603B69B6
:1060C00011E07B69BA6813443A69D2B21A707B69ED
:1060D00001337B617B681B687A699A42E5DB7B68E8
:1060E0007A691A60002318461837BD4680BD00BF84
:1060F00000200440003004400040044000140840E8
:1061000080B586B000AFF860B9607A6000237B612B
:10611000FB681F4A93420ED0FB681E4A93420AD086
:10612000FB681D4A934206D0FB681C4A934202D08A
:106130006FF0020328E0BB68002B02D14FF0FF3361
:1061400022E07B68002B16D14FF0FF331CE07B6907
:10615000BA6813441B781946F868FFF763FC386186
:106160003B69002B04D07B687A691A603B690BE0BD
:106170007B6901337B617B681B687A699A42E6DB45
:106180007B687A691A60002318461837BD4680BDBF
:106190000020044000300440004004400014084047
:1061A00080B487B000AFF860B9607A6000237B618B
:1061B0000FE0FB685B6803F01003002B0ED1FB6857
:1061C000196ABA687B691344CAB21A707B690133D1
:1061D0007B617A697B689A42EBD300E000BF7B6900
:1061E00018461C37BD465DF8047B704780B483B009
:1061F00000AF78607B685B681B0A03F00F031846EA
:106200000C37BD465DF8047B704780B487B000AFA3
:10621000F860B9607A6000237B610FE0FB685B681F
:1062200003F08003002B0ED1BA687B6913441B78FE
:106230001A46FB681A627B6901337B617A697B6865
:106240009A42EBD300E000BF7B6918461C37BD467D
:106250005DF8047B704780B485B000AF78607B68E0
:106260005B681B0B03F00F03FB60FB68C3F10803C3
:1062700018461437BD465DF8047B704780B483B080
:1062800000AF78607B68134A93420ED07B68124A55
:1062900093420AD07B68114A934206D07B68104A29
:1062A000934202D06FF002030DE07B681B6843F459
:1062B00080727B681A6000BF7B681B6803F4807380
:1062C000002BF9D1002318460C37BD465DF8047B3E
:1062D000704700BF002004400030044000400440EC
:1062E0000014084080B483B000AF786039607B68E8
:1062F000154A93420ED07B68144A93420AD07B68B9
:10630000134A934206D07B68124A934202D06FF040
:10631000020313E03B68002B02D03B68082B02D934
:106320006FF002030AE07B681B6823F00F023B68F2
:1063300003F00F031A437B681A60002318460C37DA
:10634000BD465DF8047B70470020044000300440E7
:10635000004004400014084080B483B000AF78606F
:106360007B681B6803F00F0318460C37BD465DF8C9
:10637000047B704780B483B000AF78607B68DB68D3
:1063800018460C37BD465DF8047B704780B483B077
:1063900000AF786039607B680D4A93420ED07B680D
:1063A0000C4A93420AD07B680B4A934206D07B6822
:1063B0000A4A934202D06FF0020303E07B683A6816
:1063C000DA60002318460C37BD465DF8047B704741
:1063D0000020044000300440004004400014084005
:1063E00080B483B000AF786039607B680F4A934215
:1063F0000ED07B680E4A93420AD07B680D4A9342C6
:1064000006D07B680C4A934202D06FF0020306E08C
:106410007B689A683B681A437B689A600023184639
:106420000C37BD465DF8047B704700BF0020044078
:1064300000300440004004400014084080B483B0A1
:1064400000AF786039607B680F4A93420ED07B685A
:106450000E4A93420AD07B680D4A934206D07B686D
:106460000C4A934202D06FF0020307E07B689A68FF
:106470003B68DB431A407B689A60002318460C3760
:10648000BD465DF8047B70470020044000300440A6
:10649000004004400014084080B483B000AF78602E
:1064A0007B685B6818460C37BD465DF8047B704717
:1064B00080B586B000AF78607B681B689F4A9342C6
:1064C00017D07B681B689E4A934210D07B681B687C
:1064D0009C4A934209D07B681B689B4A934201D136
:1064E000032307E04FF0FF3304E0022302E001231F
:1064F00000E000237B617B69002B02DA6FF003036D
:106500002EE1924A7B6952F82330002B14D1904A35
:106510007B6952F82330002B0ED17B681B684FF04B
:10652000FF311846FFF734FB7B681B684FF0FF31E3
:106530001846FFF711FB19E0854A7B6952F82330B2
:10654000002B06D07B681B69002B02D06FF005037F
:1065500006E17E4A7B6952F82330002B06D07B6827
:10656000DB68002B02D06FF00503F9E07B680022A6
:106570005A617B6800229A617B68DB68002B75D0CA
:106580007B685B68002B02D16FF00203E8E07B6858
:106590001B6840211846FFF7EDFA7B681B68184618
:1065A000FFF79CFA38617B68DA687B685B69D31A0D
:1065B0003A69934228BF13463B617B6818687B6841
:1065C0005A687B685B6913443A691946FFF776FAA3
:1065D00002467B685B691A447B685A617B681B686A
:1065E0001846FFF77BFA0346032B1DD97B685A69CF
:1065F0007B68DB689A4217D17B69002B10D07B69DE
:10660000012B0BD07B69022B06D07B69032B01D1B8
:10661000582306E0002304E0222302E00F2300E0D9
:106620000E231846FFF7F2FA7B681B68434A934231
:1066300017D07B681B68424A934210D07B681B6866
:10664000404A934209D07B681B683F4A934201D17C
:10665000032307E04FF0FF3304E0022302E00123AD
:1066600000E0002339497A6841F823207B681B69E0
:10667000002B74D07B681B680B211846FFF77AFA51
:106680007B689B68002B0ED17B681B684FF0FF3145
:106690001846FFF77DFA7B681B681846FFF72AFA51
:1066A0006FF002035CE07B681B6810211846FFF75F
:1066B00061FA7B681B681846FFF7F4F9F8607B689D
:1066C0001A697B689B69D31AFA68934228BF1346FC
:1066D000FB607B6818687B689A687B689B691344D9
:1066E000FA681946FFF7CEF902467B689B691A449F
:1066F0007B689A617B681B6810211846FFF72CFAAB
:106700007B681B680D4A934224D07B681B680C4A47
:10671000934210D07B681B680A4A934209D07B6879
:106720001B68094A934201D1032314E04FF0FF3361
:1067300011E002230FE001230DE000BF0020044020
:10674000003004400040044000140840E0130020E2
:10675000F0130020002304497A6841F82320002325
:1067600018461837BD4680BDF013002080B584B0B0
:1067700000AF786039607B681D4A934214D07B6813
:106780001C4A93420ED07B681B4A934208D07B6818
:106790001A4A934201D1032307E04FF0FF3304E08C
:1067A000022302E0012300E00023FB60FB68002BD2
:1067B00002DA6FF0020316E0114AFB6852F8233048
:1067C000BB60BB68002B0DD0BB68DB69002B09D018
:1067D0000B4AFB68002142F82310BB68DB6939686B
:1067E000B8689847002318461037BD4680BD00BFE3
:1067F00000200440003004400040044000140840E1
:10680000E013002080B584B000AF786039607B6809
:106810001D4A934214D07B681C4A93420ED07B6879
:106820001B4A934208D07B681A4A934201D1032342
:1068300007E04FF0FF3304E0022302E0012300E011
:106840000023FB60FB68002B02DA6FF0020316E006
:10685000114AFB6852F82330BB60BB68002B0DD097
:10686000BB68DB69002B09D00B4AFB68002142F8AA
:106870002310BB68DB693968B8689847002318465D
:106880001037BD4680BD00BF0020044000300440EA
:106890000040044000140840F013002080B584B08C
:1068A00000AF786039607B681B4A934214D07B68E4
:1068B0001A4A93420ED07B68194A934208D07B68EB
:1068C000184A934201D1032307E04FF0FF3304E05D
:1068D000022302E0012300E00023FB60FB68002BA1
:1068E00002DA6FF0020312E039687868FFF73EFFC2
:1068F0000D4AFB6852F823200C49FB6851F82330FD
:106900009A4203D039687868FFF77CFF0023184665
:106910001037BD4680BD00BF002004400030044059
:106920000040044000140840F0130020E013002051
:1069300080B582B000AF78607B680D4A93420ED07C
:106940007B680C4A93420AD07B680B4A934206D07C
:106950007B680A4A934202D06FF0020304E04021B0
:106960007868FFF715F9002318460837BD4680BD43
:10697000002004400030044000400440001408405F
:1069800080B582B000AF78607B680D4A93420ED02C
:106990007B680C4A93420AD07B680B4A934206D02C
:1069A0007B680A4A934202D06FF0020304E00B2195
:1069B0007868FFF7EDF8002318460837BD4680BD1C
:1069C000002004400030044000400440001408400F
:1069D00080B582B000AF78607B680E4A93420ED0DB
:1069E0007B680D4A93420AD07B680C4A934206D0DA
:1069F0007B680B4A934202D06FF0020305E04FF030
:106A0000FF317868FFF7C4F8002318460837BD4601
:106A100080BD00BF0020044000300440004004401E
:106A20000014084080B582B000AF78607B680F4AE0
:106A300093420ED07B680E4A93420AD07B680D4A7F
:106A4000934206D07B680C4A934202D06FF0020357
:106A500008E07868FEF764FC6FF00F017868FEF7D5
:106A600051FC002318460837BD4680BD0020044075
:106A700000300440004004400014084090B589B044
:106A800000AF78607B68974A934214D07B68964A3F
:106A900093420ED07B68954A934208D07B68944A13
:106AA000934201D1032307E04FF0FF3304E00223B8
:106AB00002E0012300E00023FB61FB69002B02DA06
:106AC0006FF003030AE17868FFF73AF8B861894A82
:106AD000FB6952F82330002B0ED1874AFB6952F82C
:106AE0002330002B08D17B68DB6819467868FFF7F4
:106AF00033F86FF00303F1E07B689A68BB691340D9
:106B000003F00B03002B0AD07868FEF709FC6FF046
:106B100008017868FEF7F6FB6FF00303DEE0754AC4
:106B2000FB6952F823307B617B69002B30D07B6995
:106B3000DB68002B2CD07B691B681846FEF7CEFF64
:106B400038617B69DA687B695B69D31A3A699A4272
:106B500005D97B69DA687B695B69D31A00E03B6918
:106B60003B617B6918687B695A687B695B69134480
:106B70003A691946FEF7A2FF02467B695B691A442F
:106B80007B695A617B691B6840211846FEF7E4FF68
:106B9000594AFB6952F823307B617B69002B4CD04A
:106BA000BB6903F01003002B47D07B691B69002BE6
:106BB00043D07B691B681846FEF774FFF8607B6959
:106BC0001A697B699B69D31AFA689A4205D97B696D
:106BD0001A697B699B69D31A00E0FB68FB607B69DB
:106BE00018687B699A687B699B691344FA6819463F
:106BF000FEF748FF02467B699B691A447B699A61EC
:106C00007B691A697B699B69D41A7B691B68184682
:106C1000FEF78AFF03469C4209D27B6918687B69AC
:106C20001A697B699B69D31A1946FEF76FFF7B6966
:106C30001B6810211846FEF78FFF2F4AFB6952F898
:106C400023202C49FB6951F823309A4217D17B69E4
:106C5000002B12D07B699A697B691B699A420CD11F
:106C60007B695A697B69DB689A4206D17868FEF7CE
:106C700057FB00217868FEF745FB00232EE01E4AF3
:106C8000FB6952F823307B617B69002B0ED07B6956
:106C90009A697B691B699A4208D17868FFF770FE90
:106CA00000217868FFF7AEFD002317E0114AFB6969
:106CB00052F823307B617B69002B0ED07B695A69C7
:106CC0007B69DB689A4208D17868FFF731FE0021C2
:106CD0007868FFF74BFD002300E0002318462437B7
:106CE000BD4690BD002004400030044000400440F8
:106CF00000140840E0130020F0130020B0B598B055
:106D000000AF78600023FB652A4B07F108041D469D
:106D10000FCD0FC42B682360274B07F11C041D46C1
:106D20000FCD0FC42B682360244B07F130041D46A0
:106D30000FCD0FC42B682360214B07F144041D467F
:106D40000FCD0FC42B6823600023BB652AE0BB6D09
:106D50009B007A68D01807F10801BA6D13469B00B2
:106D600013449B000B44194603F0BFF8F865FB6D14
:106D7000002B01D0FB6D19E07B681B68002B0ED047
:106D8000BB6D9B007A6813441B680021184603F012
:106D900027F9F865FB6D002B01D0FB6D06E0BB6D9C
:106DA0000133BB65BB6D032BD1D9FB6D1846603732
:106DB000BD46B0BD9800002070000020FC000020FF
:106DC0001001002080B582B000AF786001217868A2
:106DD00003F02CF9034618460837BD4680BD80B540
:106DE00082B000AF78600021786803F01FF9034695
:106DF00018460837BD4680BD80B584B000AF7860C6
:106E000007F10B031946786803F036F9F860FB6860
:106E1000002B01D0FB680DE0FB7A002B02D101238F
:106E2000FB7201E00023FB72FB7A1946786803F0DD
:106E3000FDF8034618461037BD4680BD80B582B0C8
:106E400000AF78607B681B7E082B40F0D0807B68A9
:106E500093F84830032B04D07B6893F84830042B18
:106E600014D17B689B681846FFF7ACFF7B68DB6832
:106E70001846FFF7B4FF7B681B691846FFF7AFFFA2
:106E80007B685B691846FFF7B7FFFAE07B6893F809
:106E90004830062B14D17B689B681846FFF7ACFF7F
:106EA0007B68DB681846FFF7A7FF7B681B691846FD
:106EB000FFF7A2FF7B685B691846FFF79DFFE0E0E4
:106EC0007B6893F84830052B14D17B689B68184683
:106ED000FFF785FF7B68DB681846FFF78DFF7B684F
:106EE0001B691846FFF788FF7B685B691846FFF748
:106EF00076FFC6E07B6893F84830072B14D17B6897
:106F00009B681846FFF76BFF7B68DB681846FFF746
:106F100073FF7B681B691846FFF76EFF7B685B6930
:106F20001846FFF769FFACE07B6893F84830082B00
:106F300014D17B689B681846FFF75EFF7B68DB68AF
:106F40001846FFF74CFF7B681B691846FFF747FFA1
:106F50007B685B691846FFF742FF92E07B6893F815
:106F60004830012B14D17B689B681846FFF744FF1B
:106F70007B68DB681846FFF732FF7B681B691846A1
:106F8000FFF720FF7B685B691846FFF728FF78E072
:106F90007B6893F848300A2B14D17B689B681846AD
:106FA000FFF72AFF7B68DB681846FFF725FF7B6841
:106FB0001B691846FFF713FF7B685B691846FFF7EC
:106FC0000EFF5EE07B689B681846FFF7FBFE7B6860
:106FD000DB681846FFF703FF7B681B691846FFF75D
:106FE000FEFE7B685B691846FFF7ECFE49E07B68B4
:106FF0001B7E042B03D07B681B7E052B14D17B6882
:107000009B681846FFF7DEFE7B68DB681846FFF7D3
:10701000E6FE7B681B691846FFF7EEFE7B685B693E
:107020001846FFF7DCFE2CE07B681B7E032B14D197
:107030007B689B681846FFF7C5FE7B68DB681846CF
:10704000FFF7C0FE7B681B691846FFF7C8FE7B6828
:107050005B691846FFF7C3FE13E07B689B68184620
:10706000FFF7B0FE7B68DB681846FFF7B8FE7B6869
:107070001B691846FFF7B3FE7B685B691846FFF78C
:10708000AEFE002318460837BD4680BD80B586B0E9
:1070900000AF6FF015037B612D4B2E4A1A602C4B0D
:1070A0002D4A5A602A4B2D4A9A6005F00BFB7861F5
:1070B0007B69002B01D07B6946E007F108030022C1
:1070C0001A605A609A60264BFB6007F10803194664
:1070D000244803F03DF978617B69002B01D07B697E
:1070E00032E0204B1B6801221821184603F02EFACB
:1070F00078617B69002B01D07B6925E0194B1B6807
:107100001821184603F0DEF978617B69002B01D065
:107110007B6919E03B1D1449184603F063FB786155
:107120007B69002B01D07B690EE07B68184607F075
:107130002FF901F095F878617B69002B03D07B680B
:10714000184603F093FB7B6918461837BD4680BD8F
:107150000014002028000020480000205C000020CF
:1071600084710110781800200C00002080B483B0D6
:1071700000AF0346FB71FB7903F01F03012202FA03
:1071800003F1064A97F907305B0942F8231000BF64
:107190000C37BD465DF8047B704700BF00E100E09E
:1071A00080B483B000AF0346FB71FB7903F01F038B
:1071B000012202FA03F1064A97F907305B092033EE
:1071C00042F8231000BF0C37BD465DF8047B7047C2
:1071D00000E100E080B500AF1820FFF7E1FF0A4BA7
:1071E0009B680A4A1360084B1B68074A43F0010377
:1071F00013600748FDF73AFC0648FDF75BFC1820D2
:10720000FFF7B4FF00BF80BD004003401C14002006
:10721000001001400000014080B500AF1820FFF7CA
:10722000BFFF114B9B68114A13600F4B1B680E4A3E
:1072300043F0010313600E48FDF73CFC0C48FDF7DA
:1072400020FC01210A48FDF756FC0A4B1B6801335C
:10725000084A1360084B1B680133074A1360182063
:10726000FFF784FF00BF80BD0040034020140020D2
:1072700000100140141400201814002080B400AF46
:10728000034B1B681846BD465DF8047B704700BF82
:107290001414002080B400AF034B1B681846BD4691
:1072A0005DF8047B704700BF1C14002080B400AF61
:1072B000034B1B681846BD465DF8047B704700BF52
:1072C0002014002080B400AF034B00221A6000BFDE
:1072D000BD465DF8047B70471414002080B584B06F
:1072E00000AF786000F0ECF8F860FB68002B01D08C
:1072F000FB681DE0104B1B687968184600F082F8A7
:10730000F860FB68002B01D0FB6811E00B4809F026
:1073100067FB40F2E73000F015F8094B1B68084A9C
:1073200023F4F8331360064B054A1B6813600023EF
:1073300018461037BD4680BD7818002058660110E9
:107340000040034080B58AB000AF7860264B1B68D0
:10735000264AA2FB0323DB097B627B6A7A6802FB75
:1073600003F3234AA2FB03235B093B622148FDF799
:107370003BFB00233B7503237B757B6ABB610123C9
:10738000FB6107F11403012219461A48FDF70CFAB4
:10739000396A1848FDF780FB17490520FCF752FFB2
:1073A0001448FDF792FB1348FDF760FB1348FDF707
:1073B0001BFB00233B7201237B727B6A5B08FB6033
:1073C00001233B6107F10803002219460B48FDF732
:1073D000EBF90B490620FCF735FF0848FDF775FB74
:1073E00000BF2837BD4680BD00000020D34D62108D
:1073F0001F85EB5100000140D571001000100140C5
:107400001972001080B584B000AF78603960052132
:10741000786803F057F8F860FB68002B01D0FB6830
:107420000AE00621786803F04DF8F860FB68002B4D
:1074300001D0FB6800E0002318461037BD4680BD30
:1074400080B584B000AF786039601A4B1B681A4A67
:10745000A2FB0323DB09FB60FB683A6802FB03F332
:10746000154AA2FB03239B09BB603B6840F2E7324D
:10747000934207D17B68012283F834207B68C822BD
:10748000DA860FE07B68002283F834203B68A62B65
:1074900004D17B6842F60412DA8603E07B6844F28A
:1074A0007402DA86B9680548FDF7F6FA00BF1037AE
:1074B000BD4680BD00000020D34D62100000014099
:1074C00080B582B000AF4020FCF71EFFF8F7E0FF68
:1074D00078607B68002B04D0074809F081FA7B684C
:1074E00006E00220F9F740F80448F9F7EDFA002326
:1074F00018460837BD4680BD746601104C66011001
:1075000080B483B000AF78607B6840F6881202FBDD
:1075100003F2064BA3FB0213D21A520813445B0A70
:1075200018460C37BD465DF8047B704705104000D7
:1075300080B586B000AF0346FB7100237B610A2350
:10754000FB6000233B6114E0FB79002B07D0114A5C
:107550003B6952F823307A6913447B6106E00E4A96
:107560003B6952F823307A6913447B613B690133EC
:107570003B613A69FB689A42E6D37A69FB68B2FBE1
:10758000F3F37B617869FFF7BBFF034618461837B2
:10759000BD4680BD241400204C14002080B582B06C
:1075A00000AF78600120FFF7C3FF02467B681A62D4
:1075B0000020FFF7BDFF02467B68DA610023184612
:1075C0000837BD4680BD000080B483B000AF0923FA
:1075D0007B600BE07B68013B164A52F8232015497B
:1075E0007B6841F823207B68013B7B607B68002B34
:1075F000F0D1114B1B680F4A136009233B600BE06D
:107600003B68013B0D4A52F823200C493B6841F886
:1076100023203B68013B3B603B68002BF0D1084BCB
:107620001B68064A136000BF0C37BD465DF8047B3B
:10763000704700BF24140020201400204C140020A8
:107640001C14002080B400AF034B1B681846BD46D5
:107650005DF8047B704700BF1814002080B400AFB1
:10766000034B00221A6000BFBD465DF8047B7047E3
:107670001814002080B483B000AF7860054B1B68FD
:107680000133044A136000BF0C37BD465DF8047B2C
:10769000704700BF7814002080B400AF034B1B6814
:1076A0001846BD465DF8047B704700BF7814002083
:1076B00080B400AF034B00221A6000BFBD465DF8E6
:1076C000047B70477814002080B58AB000AFF86062
:1076D000B9607A603B60594B7B610023BB6100233A
:1076E0003B7700237B7700233B625549B86802F063
:1076F000FCFB78627B6A002B01D07B6A99E0BB6857
:10770000002B0BD0BB681B680121184602F068FCF7
:1077100078627B6A002B01D07B6A8AE0494938682D
:1077200002F0E3FB78627B6A002B01D07B6A80E089
:107730003B68002B0AD03B681B68184602F02EFC01
:1077400078627B6A002B01D07B6A72E007F1140338
:107750001A461B21F86802F048FE78627B6A002B0B
:1077600001D07B6A65E003221B21F86802F085FEE8
:1077700078627B6A002B01D07B6A5AE001221B21D0
:10778000F86802F0E3FE78627B6A002B01D07B6A26
:107790004FE01B21F86802F095FE78627B6A002BAF
:1077A00001D07B6A45E02849786802F09EFB786248
:1077B0007B6A002B01D07B6A3BE07B68002B0AD000
:1077C0007B681B68184602F0E9FB78627B6A002B35
:1077D00001D07B6A2DE007F114031A461A21F868DC
:1077E00002F003FE78627B6A002B01D07B6A20E006
:1077F00003221A21F86802F040FE78627B6A002BAF
:1078000001D07B6A15E001221A21F86802F09EFE81
:1078100078627B6A002B01D07B6A0AE01A21F86843
:1078200002F050FE78627B6A002B01D07B6A00E098
:10783000002318462837BD4680BD00BF757600106E
:10784000C0000020D4000020E800002080B584B0F3
:1078500000AF78600E49786802F047FBF860FB687B
:10786000002B01D0FB680FE07B68002B0BD07B68FE
:107870001B680021184602F0B3FBF860FB68002B80
:1078800001D0FB6800E0002318461037BD4680BDDC
:107890008400002080B582B000AF78600021786855
:1078A00002F09EFB034618460837BD4680BD80B5F2
:1078B00082B000AF78600121786802F091FB034646
:1078C00018460837BD4680BD80B582B000AF7860ED
:1078D00039603968786802F0CFFB034618460837EC
:1078E000BD4680BD80B400AF034B01221A7000BFBB
:1078F000BD465DF8047B70477C14002080B400AF67
:10790000034B00221A7000BFBD465DF8047B704730
:107910007C14002090B58FB000AF78600123FB721B
:1079200000237B6300233B630023FB620AE000BF6C
:1079300002F07CF80346002BFAD002F083F8FB6AD1
:107940000133FB62FB6A052BF1D90023FB624FE098
:107950007B681B6807F114020021184603F05EFBE8
:10796000B862BB6A002B01D0BB6AA8E17B681B68C8
:1079700007F110020121184603F050FBB862BB6A00
:10798000002B01D0BB6A9AE17B681B6807F10C02EF
:107990000221184603F042FBB862BB6A002B01D0FB
:1079A000BB6A8CE13B69184602F0DAF903464FEAFC
:1079B000E374C7E90834FB68184602F01DFA034671
:1079C0004FEAE374C7E906343B6A7A6B9342B8BF67
:1079D00013467B63BB693A6B9342B8BF13463B6364
:1079E00002F024F80346002BB2D0FB6A0133FB629D
:1079F000FB6A052BF4D90023FB62796BB24808F0CF
:107A0000A7FF7B6893F84830032B18D07B6BAF4AF5
:107A1000934208DD7B6BAE4A934204DC7B68002214
:107A200083F835200BE07B6BAA4A934203DC7B6B27
:107A3000A94A934203DC7B68012283F835207B68E6
:107A400093F83530002B09D07B6BA44A934240F366
:107A500024817B6BA24A93420ADD1EE17B6BA14A23
:107A6000934240F31C817B6B9F4A934200F3178142
:107A70009E4808F0B5FF7B685B681846FFF717FF64
:107A8000B862BB6A002B40F00E81994808F0A8FF4D
:107A90004FF4967003F02BFD00237B6300233B63C0
:107AA00000BF01F0C3FF0346002BFAD001F0CAFF6C
:107AB0004FE07B681B6807F114020021184603F0B1
:107AC000ADFAB862BB6A002B01D0BB6AF7E07B68F5
:107AD0001B6807F110020121184603F09FFAB862F3
:107AE000BB6A002B01D0BB6AE9E07B681B6807F129
:107AF0000C020221184603F091FAB862BB6A002B0F
:107B000001D0BB6ADBE03B69184602F029F9034665
:107B10004FEAE374C7E90834FB68184602F06CF9D1
:107B200003464FEAE374C7E906343B6A7A6B934233
:107B3000B8BF13467B63BB693A6B9342B8BF134629
:107B40003B6301F073FF0346002BB2D0FB6A0133A5
:107B5000FB62FB6A052BF4D90023FB62396B786862
:107B600000F0ACFAB862BB6A002B40F09E800023A4
:107B70007B6300233B637B685B681846FFF78AFEE4
:107B8000B862BB6A002B40F092804FF4967003F00D
:107B9000AEFC00BF01F04AFF0346002BFAD001F013
:107BA00051FF4FE07B681B6807F114020021184663
:107BB00003F034FAB862BB6A002B01D0BB6A7EE0E6
:107BC0007B681B6807F110020121184603F026FAB2
:107BD000B862BB6A002B01D0BB6A70E07B681B688F
:107BE00007F10C020221184603F018FAB862BB6ACA
:107BF000002B01D0BB6A62E03B69184602F0B0F886
:107C000003464FEAE374C7E90834FB68184602F0FC
:107C1000F3F803464FEAE374C7E906343B6A7A6B2C
:107C20009342B8BF13467B63BB693A6B9342B8BFBC
:107C300013463B6301F0FAFE0346002BB2D0FB6A09
:107C40000133FB62FB6A052BF4D90023FB62294850
:107C500008F0C6FE7B685B6807F10B021146184608
:107C6000FFF732FEB862BB6A002B22D1FB7A002BF1
:107C700021D13B6BB3F5FA6F03DB3B6B1A4A93429E
:107C800003DD1D4808F0ACFE16E0194808F0A8FE18
:107C90001A4808F0A5FE002311E000BF00E000BF75
:107CA0000223BB6208E000BF06E000BF04E000BFA3
:107CB00002E000BF00E000BF0123BB62BB6A1846C0
:107CC0003C37BD4690BD00BF98660110B8F9020070
:107CD0003F070400708E01000F1B02006F8E010031
:107CE000101B0200B7F9020040070400B86601103B
:107CF000D8660110E86601101067011028670110AE
:107D000080B584B000AF78600023FB720023BB72A3
:107D10007B681B68DB691B21184602F0F5FBF860E5
:107D2000FB68002B01D0FB68C0E07B681B68DB6947
:107D30001A21184602F0E8FBF860FB68002B01D01E
:107D4000FB68B3E07B68DB6B0021184602F06EF93C
:107D5000F860FB68002B01D0FB68A7E03C2003F033
:107D6000C6FB7B68DB6B0121184602F05FF9F86007
:107D7000FB68002B01D0FB6898E04FF42F7003F0F4
:107D8000B6FB7B681B6C07F10B021146184602F02C
:107D900073F9F860FB68002B01D0FB6886E07B6814
:107DA0005B6C07F10A021146184602F065F9F860AB
:107DB000FB68002B01D0FB6878E0FB7A002B6DD0CC
:107DC000BB7A012B6AD04FF42F7003F090FB7B68D5
:107DD0001B6C07F10B021146184602F04DF9F860D2
:107DE000FB68002B01D0FB6860E07B685B6C07F1EF
:107DF0000A021146184602F03FF9F860FB68002BB2
:107E000001D0FB6852E0FB7A002B49D0BB7A002BF3
:107E100046D04FF4347003F06AFB7B681B6C07F1AB
:107E20000B021146184602F027F9F860FB68002B98
:107E300001D0FB683AE07B685B6C07F10A021146EF
:107E4000184602F019F9F860FB68002B01D0FB68B6
:107E50002CE0FB7A012B25D0BB7A012B22D07B684A
:107E60001B68DB691B21184602F02CFBF860FB68DD
:107E7000002B01D0FB6819E07B681B68DB691A21C5
:107E8000184602F01FFBF860FB68002B01D0FB686E
:107E90000CE0084808F0A4FD002307E000BF02E062
:107EA00000BF00E000BF0623FB60FB6818461037E8
:107EB000BD4680BD4467011080B586B000AFF86054
:107EC0000B467A607B810023FB740023BB747B68C4
:107ED00006221A707B89002B28D1724808F080FD99
:107EE000FB681B68DB691B21184602F00DFB7861FB
:107EF0007B69002B01D07B69CFE0FB681B68DB69E5
:107F00001A21184602F000FB78617B69002B01D032
:107F10007B69C2E0FB68DB6B0021184602F086F843
:107F200078617B69002B01D07B69B6E07B89032BEC
:107F30000ED15D4808F054FDFB68DB6B012118464B
:107F400002F074F878617B69002B01D07B69A4E0B2
:107F50007B89252B24D1554808F042FDFB681B6C1A
:107F600007F113021146184602F086F878617B6922
:107F7000002B01D07B6990E0FB685B6C07F112027B
:107F80001146184602F078F878617B69002B01D021
:107F90007B6982E0FB7C002B74D0BB7C012B71D011
:107FA0007B89482B24D1424808F01AFDFB681B6CE2
:107FB00007F113021146184602F05EF878617B69FA
:107FC000002B01D07B6968E0FB685B6C07F1120253
:107FD0001146184602F050F878617B69002B01D0F9
:107FE0007B695AE0FB7C002B4ED0BB7C002B4BD036
:107FF0007B896C2B44D12F4808F0F2FCFB681B6C8A
:1080000007F113021146184602F036F878617B69D1
:10801000002B01D07B6940E0FB685B6C07F112022A
:108020001146184602F028F878617B69002B01D0D0
:108030007B6932E0FB7C012B28D0BB7C012B25D057
:10804000FB681B68DB691B21184602F03BFA78616C
:108050007B69002B01D07B691FE0FB681B68DB6933
:108060001A21184602F02EFA78617B69002B01D0A4
:108070007B6912E07B6807221A700F4808F0B0FC99
:1080800000230AE000BF02E000BF00E000BF7B6801
:1080900008221A7006237B617B6918461837BD4693
:1080A00080BD00BF5C67011084670110B0670110DC
:1080B000D8670110006801104467011080B584B0D2
:1080C00000AF78603960114808F08AFC7B685B6813
:1080D00007F10B0211461846FFF7F6FBF860FB6844
:1080E000002B01D0FB680CE0FB7A002B05D03B682D
:1080F000B3F5FA6F01DD012303E0054808F070FCD9
:10810000002318461037BD4680BD00BF2C68011003
:10811000D866011090B583B000AF7860FFF7C6F85D
:1081200003461846FFF7ECF90446FFF7B3F8034699
:108130001846FFF7E5F903461A462146104808F0AD
:1081400007FCFFF7B3F803461846FFF7D9F90246D4
:1081500040F261739A420ED8FFF7A8F8034618461A
:10816000FFF7CEF90346B3F5C86F04D9054808F008
:1081700037FC002300E0072318460C37BD4690BDAE
:10818000546801108068011080B584B000AF786039
:108190007868FFF7BFFBF860FB68002B1AD140F24C
:1081A000E7317868FFF74CF9C82003F0A0F9786848
:1081B000FFF7A6FDF860FB68002B0DD17868FFF78C
:1081C000A9FFF860FB68002B08D1094808F008FCFB
:1081D000002308E000BF02E000BF00E000BF054848
:1081E00008F0FEFBFB6818461037BD4680BD00BF97
:1081F0009C680110BC68011080B584B000AF786045
:108200000123FB727B685B6807F10B02114618467D
:10821000FFF75AFBF860FB68002B12D1FB7A002BAA
:1082200011D17B685B6AB3F5FA6F04DB7B685B6A2C
:10823000094A934203DD094808F0D2FB04E0002319
:1082400005E000BF00E000BF0123FB60FB681846AB
:108250001037BD4680BD00BF40070400DC68011038
:1082600090B5A7B002AF0023C7F88C300023C7F841
:1082700088300023C7F884300023C7F880304FF0DF
:1082800000034FF00004C7E912344FF000034FF031
:108290000004C7E910340B2387F82B304FF48573A3
:1082A000FB674FF48573BB67002387F877300023A3
:1082B00087F87630002387F87530002387F874300C
:1082C00007F12003184603F023F93B6A3B673B6A3A
:1082D000FB663B6ABB660023FB630023BB63002392
:1082E0007B637B6A7B6600233B66002387F85F30F5
:1082F000002387F85E30002387F85D30002387F87D
:108300005C30002387F85B30002387F85A30002365
:1083100087F859300023FB610023BB6100237B6198
:1083200000233B616FF015037B654A2300933223E2
:108330005B221B21A04808F00BFB052003F0D7F8B7
:108340009E499F4808F004FB4C21012006F094F957
:1083500038633B6B002B03D16FF00B0300F088BE3A
:1083600007F10C039749184606F035F978657B6DDF
:10837000002B05D0386B06F08DF97B6D00F078BED0
:108380003B6B08331846FEF7B9FC78657B6D002B14
:1083900009D0386B06F07EF9FB68184606F043F901
:1083A0007B6D00F065BE3B6B184601F0E5FB786520
:1083B0007B6D002B40F038863B6B04331846FFF78B
:1083C00045FA78657B6D002B40F030863B6B1B686F
:1083D000D8693B6B03F13C013B6B03F140023B6B03
:1083E0004433FFF771F978657B6D002B40F02086F0
:1083F000386BFEF773FF78657B6D002B40F01A86B3
:108400003B6B5B681846FFF745FA78657B6D002B80
:1084100040F01286FFF772FA01F014FB3B6B1B6809
:10842000184603F035F878657B6D002B40F0068622
:108430003B6BC8221A87386BFFF7A6FE78657B6D09
:10844000022B54D1386BFEF7F9FC002387F82B3050
:108450003B6B93F83530002B1CD0D7F88C305A4A40
:10846000934202DC03237B6531E0D7F88C30574A16
:1084700093422CDD04237B653B6B08221A767B6DCF
:10848000DAB23B6B83F848200121386BFEF7D8FF46
:1084900000F0DDBDD7F88C304D4A934202DC032357
:1084A0007B6514E0D7F88C304A4A93420FDD0423F1
:1084B0007B653B6B08221A767B6DDAB23B6B83F8E7
:1084C00048200121386BFEF7BBFF00F0C0BD7B6D7B
:1084D000DAB23B6B83F84820386BFFF71BFA7865FC
:1084E0007B6D032BF8D0386BFFF74EFE78657B6D04
:1084F000002B0DD03B6B08221A767B6DDAB23B6BFA
:1085000083F848200121386BFEF79AFF00F09FBDE9
:1085100000BF01F08BFA0346002BFAD001F092FA6B
:108520003B6B1B68DB690E21184601F0EDFF786597
:108530007B6D002B09D03B6B08221A767B6DDAB27B
:108540003B6B83F8482000F082BD40F2E731386B86
:10855000FEF776FFFFF7ACF83B6B01225A763B6BD8
:1085600000221A763B6B002283F848200C2387F800
:108570002B30FEF783FE0346002B00F08D80FFF7C3
:1085800023F8386BFFF70AF83B46184602F0C0FFA5
:1085900007F120033A4692E8030083E803007B6A70
:1085A0007A6E9A4218D97A6A7B6ED31A03F57423CD
:1085B00003F510733B6613E00469011010690110A4
:1085C00018690110300100206F8E0100101B02009D
:1085D000B7F90200400704007A6A7B6ED31A3B6643
:1085E0003B6E44F6206293422AD93B46184602F07D
:1085F0008FFF07F120033A4692E8030083E8030067
:108600007B6A7B6697F82B30172B14D097F82B30AA
:108610001A2B10D097F82B30062B0CD097F82B3054
:10862000002B08D097F82B301946386B00F032FD3C
:10863000034687F82B3001F0B5F9012387F85A304B
:108640003A6A3B6FD31AFB63FB6B0A2B06D997F888
:108650007730012B02D1002387F877303A6AFB6E1E
:10866000D31ABB63BB6B042B06D997F87630002B6B
:1086700002D1012387F876303A6ABB6ED31A7B6346
:108680007B6B032B06D997F87530002B02D10123A1
:1086900087F87530FEF716FE07F1100307F1140294
:1086A00007F11801386B01F0F3FB78657B6D002B47
:1086B00040F0C6847B69184601F052FB03464FEA3E
:1086C000E374C7E912343B69184601F095FB034691
:1086D0004FEAE374C7E91034BB6CD7F88C2093429F
:1086E000B8BF1346C7F88C303B6CD7F8882093424C
:1086F000B8BF1346C7F88830BB69D7F880209342CB
:10870000B8BF1346C7F8803097F85A30012B7AD19A
:1087100097F85F30013387F85F3097F85D300133A9
:1087200087F85D3097F85F30042B46D997F85E30B4
:10873000092B42D83B6BD7F88C209A623B6BD7F859
:108740008020DA6297F87630012B0CD13B6BD96A26
:108750003B6B9B6A1A46BD4808F0FAF83B6AFB6619
:10876000002387F8763097F82B301946386B00F0E5
:10877000E1FF034687F82B3097F85B30002B0AD0D7
:1087800097F85E30002B06D0D7F88420D7F88830D1
:108790001344C7F884300023C7F88C300023C7F88F
:1087A00080300023C7F88830002387F85F3097F8BF
:1087B0005E30013387F85E3022E097F85E30092B97
:1087C0001ED997F85B30002B0ED097F85E30013B36
:1087D000D7F8842092FBF3F23B6B5A62002387F8B0
:1087E0005F30012387F85C30002387F85E30002378
:1087F000C7F888300023C7F88C300023C7F88030D2
:10880000002387F85A3097F85D30F92B4BD9FB6875
:1088100007F11C020021184605F08CFE78657B6D7F
:10882000002B40F00F844FF0FF33FB62FB6A1B0507
:10883000FB62FB6A1B0CFB62FB6AFA691146184675
:1088400006F097FD0346FB61FB690B21184606F015
:10885000E5FD02463B6B1A633B6B1B6B1A461346E6
:108860005B019B1A5B001A463B6B1A633B6B1B6BED
:10887000184606F0DDFF4FF00002754B07F06CF96B
:1088800003460C461A462346724808F061F897F8EA
:108890002B301946386B00F0FBFE034687F82B306F
:1088A000002387F85D30FEF7F7FE0346002B19DD45
:1088B0003B6B5B7E062B06D1FEF7FAFE3B6B00227C
:1088C00083F848200AE03B6B1A7E3B6B5A763B6B81
:1088D00008221A763B6B052283F848203B6B1A7EF0
:1088E0003B6B5A7601F052F80346B3F57A7F40F0BD
:1088F0008C8301F065F83B6B1B7E082B3FF639AE8D
:1089000001A252F823F000BFAB8B0010DB890010EE
:10891000C38B0010158C0010418C0010538D00107B
:108920002D8900105D890010098E00103B6B1A7EA6
:108930003B6B5B7E9A4202D0474808F051F83B6B94
:108940005B681846FEF7A6FFFEF7D8FF01F050F867
:10895000152387F82B30FEF781FE63E397F85B3031
:10896000002B10D1012387F85B30002387F85E309D
:108970000023C7F884300023C7F8883040F2E7317D
:10898000386BFEF75DFD97F82B30172B40F04083D6
:1089900097F85C30002B00F03B83386BFFF72CFC22
:1089A0000346002B0AD03B6B08221A763B6B012250
:1089B00083F84820002387F85B300AE0182387F803
:1089C0002B30FB6F1946386BFEF73AFD002387F812
:1089D0005B30002387F85C301AE397F87730012B7F
:1089E00003D1072387F82B30D2E097F87730002B9C
:1089F00040F0CE8097F82B30132B2FD1002387F82F
:108A0000743007F12B031A460021386BFFF754FA34
:108A100078657B6D002B09D0082387F82B303B6BE2
:108A200008221A763B6B052283F848203B461846FD
:108A300002F06EFD07F120033A4692E8030083E856
:108A400003003B6A3B67FEF709FEA1E044690110A1
:108A500000408F40646901108469011097F82B3041
:108A6000062B40F09580FEF7EDFD0346B3F5076F4A
:108A700021D397F87430032B1DD107F12B031A462D
:108A80006C21386BFFF718FA78657B6D002B09D0E5
:108A9000082387F82B303B6B08221A763B6B0522A4
:108AA00083F84820012387F8773097F87430013332
:108AB00087F874306CE0FEF7C5FD0346B3F5B46F7C
:108AC0001ED397F87430022B1AD107F12B031A46E4
:108AD0004821386BFFF7F0F978657B6D002B09D0E2
:108AE000082387F82B303B6B08221A763B6B052254
:108AF00083F8482097F87430013387F8743047E0E2
:108B0000FEF7A0FD0346B3F5397F1ED397F8743006
:108B1000012B1AD107F12B031A462521386BFFF7D9
:108B2000CBF978657B6D002B09D0082387F82B30B3
:108B30003B6B08221A763B6B052283F8482097F896
:108B40007430013387F8743022E0FEF77BFD034672
:108B50003B2B1DD997F87430002B19D107F12B034B
:108B60001A460321386BFFF7A7F978657B6D002B58
:108B700009D0082387F82B303B6B08221A763B6B11
:108B8000052283F8482097F87430013387F8743051
:108B900097F82B30082B40F03E823B6B08221A7668
:108BA0003B6B052283F8482035E23B6B1A7E3B6B1A
:108BB0005B7E9A4202D0BB4807F012FFFEF74EFDE3
:108BC00030E23B6B1A7E3B6B5B7E9A4202D0B6482A
:108BD00007F006FF40F2E731386BFEF731FC97F8FB
:108BE0002B300F2B03D097F82B30102B09D13B6B78
:108BF0005B681846FEF74EFEFEF780FE00F0F8FEBA
:108C00000CE297F82B300D2B40F00882386BFEF702
:108C100015F903E297F82B30122B08D1A34807F07F
:108C2000DFFEFB6F1946386BFEF70AFCF9E197F897
:108C30002B30192B40F0F581386BFEF7FFF8F0E18F
:108C40003B6B1A7E3B6B5B7E9A4202D0984807F0E2
:108C5000C7FE97F82B301E2B02D1A623BB6702E07C
:108C60004FF48573BB67BB6FFB67FB6F1946386BAF
:108C7000FEF7E6FB97F82B301A2B16D1FEF7E2FC35
:108C80000346132B5FD93B6BDB69962B06D9042374
:108C900087F82B30874807F0A3FE54E01B2387F8A2
:108CA0002B30854807F09CFE4DE097F82B30142BB5
:108CB00014D1824807F094FE3B6B5B681846FEF7C0
:108CC000F6FD78657B6D002B40F0BE8100F084FEE0
:108CD000FEF708FE002387F8593034E097F82B3070
:108CE0000F2B16D197F85930032B12D9386BFEF79A
:108CF000A5F897F87530012B07D1714807F070FE81
:108D00003B6ABB66002387F87530002387F859302B
:108D100019E097F82B301E2B15D197F85930072BF7
:108D200011D9386BFEF78AF897F87530012B07D107
:108D3000644807F055FE3B6ABB66002387F8753030
:108D4000002387F8593097F85930013387F85930A4
:108D500068E1BB6FFB67FB6F1946386BFEF770FB72
:108D600097F82B301A2B16D1FEF76CFC0346132B09
:108D700044D93B6BDB69962B06D9042387F82B304B
:108D80004C4807F02DFE39E01B2387F82B304A486A
:108D900007F026FE32E097F82B30142B14D14A4806
:108DA00007F01EFE3B6B5B681846FEF780FD78659A
:108DB0007B6D002B40F04A8100F00EFEFEF792FD25
:108DC000002387F8593019E097F82B30102B15D174
:108DD00097F85930072B11D9386BFEF72FF897F811
:108DE0007530012B07D1394807F0FAFD3B6ABB66A5
:108DF000002387F87530002387F8593097F85930E9
:108E0000013387F859300DE13B6B1A7E3B6B5B7E7B
:108E10009A4202D02E4807F0E3FD3B6B93F84830AE
:108E2000033B082B00F2EB8001A252F823F000BFB5
:108E3000DD8E0010118F0010758F0010FF8F001055
:108E4000818E0010558E00103B8F0010A18F0010F6
:108E5000D38F00101F4807F0C3FD40F2E731386B95
:108E6000FEF7EEFA3B6B5B681846FEF713FDFEF764
:108E700045FD00F0BDFD0121386BFEF7E1FAE6E0AB
:108E8000154807F0ADFD0121386BFEF7D9FA3B6BB1
:108E90005B681846FEF7FEFCFEF730FD00F0A8FD0B
:108EA000D5E000BF9C690110B4690110C4690110CC
:108EB000DC690110EC690110286A01103C6A01109C
:108EC0005C6A0110706A0110946A0110B46A0110A2
:108ED000D86A0110EC6A0110006B011097F82B3072
:108EE000002B40F08E803B6B9B6A1946624807F06E
:108EF0002FFD40F2E731386BFEF7A2FA3B6B5B685F
:108F00001846FEF7C7FCFEF7F9FC00F071FD78E0AB
:108F10003B6B9B6A1946594807F01AFD40F2E7314E
:108F2000386BFEF78DFA3B6B5B681846FEF7B2FCB8
:108F3000FEF7E4FC00F05CFD89E097F82B300A2B8B
:108F400061D03B6BDB6A19464D4807F001FD40F2EA
:108F5000E731386BFEF774FA3B6B5B681846FEF737
:108F600099FCFEF7CBFC00F043FD0121386BFEF7C6
:108F700067FA6CE0434807F033FD40F2E731386BA5
:108F8000FEF75EFA3B6B5B681846FEF783FCFEF764
:108F9000B5FC00F02DFD0121386BFEF751FA56E0CB
:108FA0003B6B1B6B1946384807F0D2FC40F2E731A7
:108FB000386BFEF745FA3B6B5B681846FEF76AFCB8
:108FC000FEF79CFC00F014FD0121386BFEF738FA27
:108FD0003DE02E4807F004FD40F2E731386BFEF724
:108FE0002FFA3B6B5B681846FEF754FCFEF786FCD5
:108FF00000F0FEFC0121386BFEF722FA27E000BFEB
:1090000010E000BF0EE000BF0CE000BFFFF7B1BAF8
:1090100000BFFFF7AEBA00BFFFF7ABBA00BFFFF764
:10902000A8BA00BFFFF7A5BA00BF10E000BF0EE06E
:1090300000BF0CE000BF0AE000BF08E000BF06E090
:1090400000BF04E000BF02E000BF00E000BF796D98
:109050000F4807F07DFC386BFDF7F0FE78657B6DFF
:10906000002B01D07B6D03E0322002F040FAF2E7E2
:1090700018469437BD4690BD1C6B01104C6B011017
:109080007C6B0110B06B0110C46B0110F46B01100C
:10909000086C011080B584B000AF78600B46FB709F
:1090A000FB78FB737B681B6A40F24B4293421AD8F1
:1090B000FB7B0C2B17D00523FB737B681A7E7B6828
:1090C0005A767B6808221A767B68072283F8482044
:1090D000FEF7C4FAFA7BFB789A4200F0BF82A148FF
:1090E00007F07EFCBAE27B68DB69962B25D9FB7B17
:1090F0001A2B22D07B6893F83430002B1DD1FB7BD8
:109100000F2B02D0FB7B102B17D10423FB737B6842
:109110001A7E7B685A767B6808221A767B6808225A
:1091200083F84820FEF79AFA7B68196A7B68DB6946
:109130001A468D4807F00CFC90E27B681B6AB3F579
:10914000E16F40F29F807B681B6A40F2617293423C
:1091500000F29880FB7B0C2B02D0FB7B1C2B14D1E4
:109160000D23FB737B681A7E7B685A767B6802222C
:109170001A767B68002283F84820FA7BFB789A42B3
:109180007FD07A4807F02CFC7BE0FB7B0D2B2CD0AA
:10919000FB7B032B29D0FB7B0F2B26D0FB7B102BDB
:1091A00023D0FB7B192B20D0FB7B122B1DD0FB7B0C
:1091B000152B1AD0FB7B182B17D0FB7B212B14D03F
:1091C0000323FB737B681A7E7B685A767B680222D6
:1091D0001A767B68002283F84820FA7BFB789A4253
:1091E0004FD0634807F0FCFB4BE0FB7B0F2B02D01A
:1091F000FB7B102B14D11623FB737B681A7E7B68D4
:109200005A767B6806221A767B68002283F848200B
:10921000FA7BFB789A4234D0564807F0E1FB30E005
:10922000FB7B152B15D12123FB737B681A7E7B6892
:109230005A767B6808221A767B680B2283F84820CE
:10924000FA7BFB789A4200F004824A4807F0C8FB98
:10925000FFE10D23FB737B681A7E7B685A767B687F
:1092600002221A767B68002283F84820FEF7F6F97E
:10927000FA7BFB789A4200F0EC813F4807F0B0FBA4
:10928000E7E1E6E17B681B6AB3F5C86F40F2DE8078
:109290007B681B6A40F28562934200F2D780FB7BB9
:1092A0000D2B05D0FB7B0C2B02D0FB7B1C2B1DD187
:1092B000FEF7C8F90346B3F57A7F17D20E23FB7386
:1092C0007B681A7E7B685A767B6803221A767B68F5
:1092D000002283F84820FEF7C1F9FA7BFB789A4216
:1092E00000F0B380254807F07BFBAEE0FB7B0E2B44
:1092F0001DD1FEF7A7F90346B3F5FA6F17D3122372
:10930000FB737B681A7E7B685A767B6803221A7629
:109310007B68002283F84820FEF7A0F9FA7BFB78EF
:109320009A4200F09280164807F05AFB8DE0FB7BD2
:109330000F2B02D0FB7B102B26D11523FB737B68F0
:109340001A7E7B685A767B6806221A767B68002232
:1093500083F84820FA7BFB789A4276D0094807F0D8
:109360003FFB72E0246C0110406C0110786C01101E
:10937000A86C0110C86C0110F86C0110246D01106C
:109380005C6D01108C6D0110FB7B152B15D1172323
:10939000FB737B681A7E7B685A767B6807221A7695
:1093A0007B68002283F84820FA7BFB789A4200F021
:1093B0005281AD4807F014FB4DE1FB7B182B15D112
:1093C0001123FB737B681A7E7B685A767B680322C5
:1093D0001A767B68002283F84820FA7BFB789A4251
:1093E00000F03981A14807F0FBFA34E1FB7B112B37
:1093F00002D0FB7B122B16D11923FB737B681A7EDC
:109400007B685A767B6803221A767B68002283F891
:109410004820FEF723F9FA7BFB789A4215D094484E
:1094200007F0DEFA11E0FB7B042B40F014810423EB
:10943000FB737B681A7E7B685A767B6808221A76F3
:109440007B68082283F8482005E104E17B681B6AF9
:1094500040F26E5293427DD97B681B6A40F2A9525A
:10946000934277D8FB7B192B15D11323FB737B68B1
:109470001A7E7B685A767B6801221A767B68002206
:1094800083F84820FA7BFB789A4200F0E68079481E
:1094900007F0A6FAE1E0FB7B072B17D11A23FB7339
:1094A0007B681A7E7B685A767B6804221A767B6812
:1094B000002283F84820FEF7D1F8FA7BFB789A4225
:1094C00000F0CB806C4807F08BFAC6E0FB7B1B2BCF
:1094D00015D11423FB737B681A7E7B685A767B68F0
:1094E00004221A767B68002283F84820FA7BFB78F6
:1094F0009A4200F0B280614807F072FAADE0FB7B5F
:10950000142B15D10F23FB737B681A7E7B685A7668
:109510007B6804221A767B68002283F84820FA7B55
:10952000FB789A4200F09980554807F059FA94E088
:10953000FB7B042B40F091800423FB737B681A7E35
:109540007B685A767B6808221A767B68082283F843
:10955000482082E07B681B6A40F29C4293427DD99E
:109560007B681B6A40F2C942934277D8FB7B192B78
:1095700014D11323FB737B681A7E7B685A767B6851
:1095800001221A767B68002283F84820FA7BFB7858
:109590009A4263D03B4807F023FA5FE0FB7B072B3E
:1095A00016D11A23FB737B681A7E7B685A767B6818
:1095B00005221A767B68002283F84820FEF74EF8D1
:1095C000FA7BFB789A4249D02B4807F009FA45E02C
:1095D000FB7B1B2B14D11423FB737B681A7E7B68E7
:1095E0005A767B6805221A767B68002283F8482029
:1095F000FA7BFB789A4231D0234807F0F1F92DE04D
:10960000FB7B142B14D11023FB737B681A7E7B68C1
:109610005A767B6805221A767B68002283F84820F8
:10962000FA7BFB789A4219D0184807F0D9F915E06F
:10963000FB7B042B12D10423FB737B681A7E7B68AF
:109640005A767B6808221A767B68082283F84820BD
:1096500004E000BF02E000BF00E000BFFB7B184653
:109660001037BD4680BD00BFC06D0110046E0110F3
:10967000486E01106C6E01109C6E0110D46E0110CA
:10968000046F0110306F0110646F01108C6F0110B6
:1096900080B584B000AF78600B46FB70FB78FB733D
:1096A0007B681B6B4CF25032934217DD1F23FB7318
:1096B0007B681A7E7B685A767B6808221A767B68FC
:1096C0000A2283F84820FA7BFB789A4229D07B68EB
:1096D0001B6B1946154807F03BF922E07B681B6BB2
:1096E0004AF6C87293421CDDFB7B0F2B05D0FB7B37
:1096F000102B02D0FB7B1E2B13D11E23FB737B6828
:109700001A7E7B685A767B68002283F84820FA7BB1
:10971000FB789A4205D07B681B6B1946044807F01A
:1097200017F9FB7B18461037BD4680BDAC6F0110A2
:10973000E86F011080B584B000AF78600B46FB7015
:10974000FB78FB737B689B6A894A934207DD7B68E1
:1097500093F83530002B02D0FB7B172B0CD17B68A4
:109760009B6A844A934215DD7B6893F83530002B61
:1097700010D1FB7B172B0DD02023FB737B681A7E47
:109780007B685A767B6808221A767B68042283F805
:10979000482083E07B689B6A774A93420ADCFB7B24
:1097A000002B07D0FB7B172B04D07B6893F8353058
:1097B000002B0FD17B689B6A704A934218DCFB7BBD
:1097C000002B15D0FB7B172B12D07B6893F835301C
:1097D000002B0DD10023FB737B681A7E7B685A76C1
:1097E0007B6808221A767B68032283F8482055E0BC
:1097F0007B689B6A604A93420ADCFB7B002B07D1A3
:10980000FB7B172B04D07B6893F83530002B0FD1EE
:109810007B689B6A594A934218DCFB7B002B15D16D
:10982000FB7B172B12D07B6893F83530002B0DD1C2
:109830001D23FB737B681A7E7B685A767B6808223F
:109840001A767B68032283F8482027E07B689B6AAE
:109850004B4A93420ADDFB7B002B02D0FB7B1D2B86
:1098600004D17B6893F83530002B0FD17B689B6A5D
:10987000444A934212DDFB7B002B02D0FB7B1D2B65
:109880000CD17B6893F83530002B07D11C23FB7378
:109890007B68002283F84820FDF7E0FEFB7B0F2B5E
:1098A0000BD0FB7B102B08D0FB7B0A2B05D0FB7B5E
:1098B000112B02D0FB7B152B39D17B68DB6A7A68D0
:1098C000D28E93420BDDFB7B0A2B08D00A23FB735D
:1098D000FDF7C4FE7B681A7E7B685A7641E0FDF78F
:1098E000B1FE024641F287339A423AD9FB7B0A2BFA
:1098F00037D17B68DB6A7A68D28E934210DD2248CA
:1099000007F026F80223FB737B681A7E7B685A7681
:109910007B6808221A767B68092283F8482020E0B9
:109920001423FB737B68002283F8482019E07B68CE
:10993000DB6A7A68128F934214DDFB7B172B11D000
:10994000FB7B052B0ED00223FB737B681A7E7B68A2
:109950005A767B6808221A767B68092283F84820A9
:1099600000E000BFFB7B18461037BD4680BD00BF3E
:10997000101B0200400704006F8E0100B7F90200BF
:10998000708E0100B8F902003870011080B400AF89
:10999000034B1B881846BD465DF8047B704700BF2B
:1099A0007C18002080B400AF044B4FF47A721A8008
:1099B00000BFBD465DF8047B704700BF7C180020E7
:1099C00080B400AF034B00221A8000BFBD465DF893
:1099D000047B70477C18002080B400AF034B012249
:1099E0001A7000BFBD465DF8047B70477E180020EA
:1099F00080B400AF034B00221A7000BFBD465DF873
:109A0000047B70477E18002080B483B000AF78607C
:109A1000054B1B680133044A136000BF0C37BD4679
:109A20005DF8047B704700BF8014002080B400AF55
:109A3000034B1B681846BD465DF8047B704700BFAA
:109A40008014002080B400AF034B00221A6000BFD6
:109A5000BD465DF8047B70478014002080B594B04B
:109A600000AF786007F1400300221A605A609A60E4
:109A7000DA60C02387F84C30D82387F84F3007F1DD
:109A8000300300221A605A609A60DA60234BBB6090
:109A90000023FB6007F140037B6107F13003BB61EA
:109AA00000237B620023BB6201233B611023FB6127
:109AB00010233B6207F108031846F9F71DFA07F176
:109AC00030030133184605F091FC03461721184670
:109AD00005F0A4FC02467B689A6007F13003053369
:109AE000184605F083FC03461721184605F096FC3E
:109AF00002467B68DA6007F130030933184605F047
:109B000075FC03461721184605F088FC02467B6861
:109B10001A61002318465037BD4680BD00E00B4057
:109B200080B584B000AF78607B68FB607B68002BF9
:109B30001BD0FB68DA69FB685B695B6819461046F5
:109B400000F0E2FCB860BB68002B10D1F868FFF7AA
:109B500085FFFB68DA69FB685B695B68194610463C
:109B600000F0B0FCB86000BF02E000BF00E000BF42
:109B70001037BD4680BD000090B58DB002AF786053
:109B80006E4BFB6000233B6100233B7500237B751C
:109B90000023BB6107F11C036949184600F0A5F9D1
:109BA00078627B6A002B01D07B6AC3E0FB69002BE3
:109BB00009D0FB69184600F0F1F978627B6A002B46
:109BC00001D07B6AB6E007F120035E49184600F039
:109BD000BFFB78627B6A002B01D07B6AAAE03B6AFC
:109BE000594AD360584B594A1A61574B6C4603F196
:109BF0000C0292E8030084E803000ECB786801F0C1
:109C00007FF878627B6A002B40F08C807B681B6851
:109C10001B79012B07D0032B09D0002B0BD14C480B
:109C200006F0DEFE0BE04B4806F0DAFE07E04A489D
:109C300006F0D6FE03E0494806F0D2FE00BF7B687E
:109C40001B68184601F0DEFA78627B6A002B56D159
:109C50007B681B680221184601F057FB78627B6A1B
:109C6000002B4ED17B681B680021184601F015FBC4
:109C700078627B6A002B46D17B681B6800211846FE
:109C800001F09AFA78627B6A002B3ED17B681B68F0
:109C90000521184601F0C9FA78627B681B68DB6908
:109CA00007F10C020E21184600F09FFB78627B6AD8
:109CB000002B2CD17B681B68DB6902220E21184621
:109CC00000F0DBFB78627B6A002B22D17B681B688B
:109CD000DB6904220E21184600F038FC78627B6AAA
:109CE000002B18D17B681B68DB690E21184600F039
:109CF000E9FB78627B6A002B0FD100231AE000BFDA
:109D00000CE000BF0AE000BF08E000BF06E000BFB3
:109D100004E000BF02E000BF00E000BF786801F08F
:109D20003FF900E000BF3B6A184600F03EFB00230D
:109D30003B627B6A18462C37BD4690BD099A0010DD
:109D4000AC0000202401002000140020219B001002
:109D5000587001108C700110C0700110F870011063
:109D60002DE9F04385B000AF78607B684FEAE3747B
:109D7000C7E90234D7E902562B4634464FF00001BA
:109D80004FF00002620142EAD36259010B461446C9
:109D90005B1B64EB06044FF000014FF0000262020F
:109DA00042EAD35259020B4614465B1946EB0404AF
:109DB0004FF000014FF00002A20142EA93629901C4
:109DC000C91A62EB040211EB050842EB0609084AC6
:109DD0004FF000034046494605F0A6FF03460C46F7
:109DE000C7E90234BB6818461437BD46BDE8F083A6
:109DF00069441400000000002DE9F04385B000AF75
:109E000078607B684FEAE374C7E90234D7E9025609
:109E10002B4634464FF000014FF00002620142EA47
:109E2000D36259010B4614465B1B64EB06044FF0EA
:109E300000014FF00002620242EAD35259020B467F
:109E400014465B1946EB04044FF000014FF000028A
:109E5000A20142EA93629901C91A62EB040211EB72
:109E6000050842EB060908A3D3E90023404649460A
:109E700005F05AFF03460C46C7E90234BB68184692
:109E80001437BD46BDE8F083E7741E0000000000F3
:109E900080B586B000AFF860B9607A603B60FB685F
:109EA0001B68BA680021184601F0B8F878617B6930
:109EB000002B01D07B6914E0FB681B687A680121E4
:109EC000184601F0ABF878617B69002B01D07B6903
:109ED00007E0FB681B683A680221184601F09EF80B
:109EE000034618461837BD4680BD80B584B000AF24
:109EF000786039603B68002B04D03B685B68B3F145
:109F0000FF3F04D17B6800221A60002320E03B68F9
:109F1000DB68002B02D16FF0150319E03B68DB68AA
:109F20005B68002B02D16FF0570311E03B68DB68E0
:109F30005B68396878689847F860FB68002B01D047
:109F4000FB6805E07B681B683A68D268DA6000232A
:109F500018461037BD4680BD80B582B000AF78602E
:109F60007B68002B15D07B68DB68002B02D16FF07B
:109F700015030FE07B68DB689B68002B02D16FF054
:109F8000570307E07B68DB689B687868984703465F
:109F900000E0002318460837BD4680BD80B582B07A
:109FA00000AF78607B68002B15D07B68DB68002BE6
:109FB00002D16FF015030FE07B68DB68DB68002BD4
:109FC00002D16FF0570307E07B68DB68DB687868D5
:109FD0009847034600E0002318460837BD4680BD79
:109FE00080B582B000AF78600B46FB707B68002BB9
:109FF00017D07B68DB68002B02D16FF0150311E0EE
:10A000007B68DB681B69002B02D16FF0570309E006
:10A010007B68DB681B69FA781146786898470346C5
:10A0200000E0002318460837BD4680BD80B582B0E9
:10A0300000AF78600B46FB707B68002B17D07B6805
:10A04000DB68002B02D16FF0150311E07B68DB6841
:10A050009B69002B02D16FF0570309E07B68DB6836
:10A060009B69FA78114678689847034600E0002318
:10A0700018460837BD4680BD80B582B000AF786015
:10A0800039607B68002B16D07B68DB68002B02D11F
:10A090006FF0150310E07B68DB689B69002B02D131
:10A0A0006FF0570308E07B68DB68DB693968786824
:10A0B0009847034600E0002318460837BD4680BD98
:10A0C00080B584B000AF786039603B68002B03D066
:10A0D0003B68DB68002B02D16FF015033FE03B6863
:10A0E000DB681B68002B02D16FF0570337E03B6839
:10A0F0001B68042B02D96FF0150330E03B681B6826
:10A10000194A52F82330002B08D1386800F02EF895
:10A11000F860FB68002B01D0FB6820E03B68DB683F
:10A120001B68396878689847F860FB68002B01D095
:10A13000FB6814E03B681A687B681B680A4951F8A1
:10A1400022201A607B681B681B681A790132D2B220
:10A150001A717B681B683A68D2681A610023184636
:10A160001037BD4680BD00BF8414002080B584B088
:10A1700000AF78601821012004F07EFAF860FB68D7
:10A18000002B02D16FF00B031DE0FB68184605F0B1
:10A190007FF8FB6800221A717B681A68FB689A6076
:10A1A0007B685A68FB68DA607B68DA68FB681A616A
:10A1B0007B681A69FB685A617B681B680449FA6806
:10A1C00041F82320002318461037BD4680BD00BF4C
:10A1D0008414002080B582B000AF78607B681B6873
:10A1E0009B68184600F01CF87B68002B03D07B6846
:10A1F0001B69002B02D16FF015030DE07B681B6912
:10A20000DB68002B02D16FF0570305E07B681B6908
:10A21000DB6878689847034618460837BD4680BD16
:10A2200080B584B000AF7860114A7B6852F8233063
:10A23000FB60FB681B79002B05D0FB681B79013B99
:10A24000DAB2FB681A71FB681B79002B0CD1FB6832
:10A250001B68184605F03AF8FB68002B04D0F86834
:10A2600004F018FA0023FB6000BF1037BD4680BD24
:10A270008414002090B587B000AFF860B960114633
:10A280001A460B46FB711346BB71FB68002B03D0CB
:10A29000FB681B69002B02D16FF015031DE0FB6802
:10A2A0001B695B68002B02D16FF0570315E0FB6858
:10A2B0001B681B68184604F0F5FFFB681B695C68A7
:10A2C000BB79FA79B968F868A0477861FB681B68C0
:10A2D0001B68184604F0F0FF7B6918461C37BD4622
:10A2E00090BD90B587B000AFF860B96011461A46CE
:10A2F0000B46FB711346BB71FB68002B03D0FB6858
:10A300001B69002B02D16FF015031DE0FB681B6970
:10A310009B68002B02D16FF0570315E0FB681B68A8
:10A320001B68184604F0BEFFFB681B699C68BB797C
:10A33000FA79B968F868A0477861FB681B681B6800
:10A34000184604F0B9FF7B6918461C37BD4690BD1E
:10A3500080B584B000AF786039603B68002B03D0D3
:10A360003B685B68002B02D16FF0150319E03B6876
:10A370005B681B68002B02D16FF0570311E03B684C
:10A380005B681B68396878689847F860FB68002B41
:10A3900001D0FB6805E07B681B683A6852685A6028
:10A3A000002318461037BD4680BD80B582B000AF8F
:10A3B00078607B68002B03D07B685B68002B02D140
:10A3C0006FF015030DE07B685B685B6A002B02D1C0
:10A3D0006FF0570305E07B685B685B6A78689847B5
:10A3E000034618460837BD4680BD80B584B000AF2F
:10A3F000F860B9607A60FB68002B03D0FB685B688B
:10A40000002B02D16FF015030FE0FB685B685B68FF
:10A41000002B02D16FF0570307E0FB685B685B68B5
:10A420007A68B968F8689847034618461037BD46F9
:10A4300080BD80B584B000AFF860B9607A60FB6819
:10A44000002B03D0FB685B68002B02D16FF0150373
:10A450000FE0FB685B689B68002B02D16FF057032D
:10A4600007E0FB685B689B687A68B968F86898479A
:10A47000034618461037BD4680BD80B584B000AF96
:10A48000F860B9601346FB71FB68002B03D0FB68D2
:10A490005B68002B02D16FF015030FE0FB685B686F
:10A4A0005B69002B02D16FF0570307E0FB685B6824
:10A4B0005B69FA79B968F868984703461846103717
:10A4C000BD4680BD80B582B000AF786039607B68E2
:10A4D000002B03D07B685B68002B02D16FF0150363
:10A4E0000EE07B685B689B69002B02D16FF057031D
:10A4F00006E07B685B689B69396878689847034623
:10A5000018460837BD4680BD80B582B000AF786080
:10A5100039607B68002B03D07B685B68002B02D11D
:10A520006FF015030EE07B685B68DB69002B02D1DE
:10A530006FF0570306E07B685B68DB693968786811
:10A540009847034618460837BD4680BD80B584B09D
:10A5500000AFF860B9607A60FB68002B03D0FB683D
:10A560005B68002B02D16FF015030FE0FB685B689E
:10A570001B6A002B02D16FF0570307E0FB685B6892
:10A580001B6A7A68B968F868984703461846103716
:10A59000BD4680BD80B584B000AF786039603B684F
:10A5A000002B03D03B68DB68002B02D16FF0150352
:10A5B0004DE03B68DB681B68002B02D16FF057034E
:10A5C00045E03B681B68082B02D96FF015033EE09D
:10A5D0003B681B68204A52F82330002B08D13868AA
:10A5E00000F03CF8F860FB68002B01D0FB682EE01F
:10A5F0003B68DB681B68396878689847F860FB68D7
:10A60000002B01D0FB6822E03B681A687B681B685E
:10A61000114951F822201A607B681B681B681A795F
:10A620000132D2B21A717B681B683A68D2681A612B
:10A630007B681B683A68D2691A627B681B683A6853
:10A640001433103292E8030083E803000023184615
:10A650001037BD4680BD00BF9814002080B584B07F
:10A6600000AF78601C21012004F006F8F860FB6858
:10A67000002B02D16FF00B0325E0FB68184604F0B5
:10A6800007FEFB6800221A717B681A68FB689A60F3
:10A690007B685A68FB68DA607B685A7AFB681A74D0
:10A6A0007B689A7AFB685A747B68DA68FB685A613F
:10A6B0007B689A69FB689A617B681B680449FA6841
:10A6C00041F82320002318461037BD4680BD00BF47
:10A6D0009814002080B582B000AF78607B681B685A
:10A6E0009B68184600F01CF87B68002B03D07B6841
:10A6F0001B69002B02D16FF015030DE07B681B690D
:10A70000DB68002B02D16FF0570305E07B681B6903
:10A71000DB6878689847034618460837BD4680BD11
:10A7200080B584B000AF7860144A7B6852F823305B
:10A73000FB60FB681B79002B05D0FB681B79013B94
:10A74000DAB2FB681A71FB681B79002B11D1FB6828
:10A750001B68184604F0BAFDFB68002B09D0F868A6
:10A7600003F098FF0023FB60044A7B68002142F855
:10A77000231000BF1037BD4680BD00BF98140020D5
:10A7800080B586B000AFF860B9601346FB80FB6807
:10A79000002B03D0FB681B69002B02D16FF015035F
:10A7A0001CE0FB681B695B68002B02D16FF057034C
:10A7B00014E0FB681B681B68184604F073FDFB6817
:10A7C0001B695B68FA88B968F86898477861FB6824
:10A7D0001B681B68184604F06FFD7B691846183724
:10A7E000BD4680BD80B584B000AF786039603B68FD
:10A7F000002B07D03B685B69002B03D03B681B78BC
:10A800000A2B02D96FF015032AE03B685B691B68CD
:10A81000002B02D16FF0570322E03B685B691B6895
:10A82000396878689847F860FB68002B01D0FB68AE
:10A8300016E07B681B683A6852695A613B681B786E
:10A840009B00094A1344184604F022FD3B681B781C
:10A8500019467B681B68044A52F821201A600023BD
:10A8600018461037BD4680BDBC14002080B582B0AC
:10A8700000AF78607B68002B03D07B685B69002B9E
:10A8800002D16FF0150319E07B685B695B69002BEF
:10A8900002D16FF0570311E07B681B68184604F083
:10A8A00015FD7B681B791946064B002243F82120D1
:10A8B0007B685B695B697868984703461846083788
:10A8C000BD4680BDBC14002080B586B000AFF860E6
:10A8D000B9607A60FB68002B06D0FB685B69002BCF
:10A8E00002D0BB68002B02D16FF015031AE0FB68A1
:10A8F0005B695B68002B02D16FF0570312E0FB68C5
:10A900001B68184604F0CEFCFB685B695B687A68DC
:10A91000B968F86898477861FB681B68184604F0C6
:10A92000CBFC7B6918461837BD4680BD80B586B024
:10A9300000AFF860B9607A60FB68002B06D0FB6856
:10A940005B69002B02D0BB68002B02D16FF01503AE
:10A950001AE0FB685B699B68002B02D16FF057031C
:10A9600012E0FB681B68184604F09CFCFB685B69FE
:10A970009B687A68B968F86898477861FB681B68D3
:10A98000184604F099FC7B6918461837BD4680BD0F
:10A9900080B58CB000AFF8607A601A460B46FB7247
:10A9A0001346BB72042387F82F30032387F82E3019
:10A9B0000C2387F82D3007F1100300221A605A602B
:10A9C0009A60DA6080233B77BB7A002B04D13B7F0F
:10A9D00043F04003DBB23B77FB7A7B7707F1100350
:10A9E00003F10C0100230322724803F006FF034623
:10A9F00087F82B3097F82B3083F0550387F82B30EE
:10AA000097F82B30FB77062387F82F300A2387F837
:10AA10002D30BB7A002B08D1102387F82F3000236C
:10AA200087F82D300D2387F82E30FB68186897F8CB
:10AA30002D3007F11002134497F82F2092B21946D7
:10AA4000FFF79EFE78627B6A002B01D07B6AADE047
:10AA5000002387F82C300CE097F82C3007F13002F7
:10AA60001344002203F8202C97F82C30013387F888
:10AA70002C3097F82C300F2BEED9BB7A002B04D159
:10AA80003B7F43F04003DBB23B7707F1100303F158
:10AA90000C0100230322474803F0AFFE034687F86A
:10AAA0002B3097F82B3083F0550387F82B3097F82D
:10AAB0002B30FB77FB68186897F82D3007F11002F0
:10AAC000134497F82F2092B21946FFF759FE786287
:10AAD0007B6A002B01D07B6A68E0FB685B79002B06
:10AAE0002AD097F82D3007F11002D11897F82F309F
:10AAF000023B1A464FF6FF732F4803F015FE03463C
:10AB00007B8497F82D2097F82F301344023B07F1F0
:10AB100010021344184604F054FC03463B843A8C5C
:10AB20007B8C9A4208D03B8C002B02D16FF0120331
:10AB30003CE06FF0460339E0BB7A002B29D107F1E6
:10AB400010030133184604F051FC03461721184640
:10AB500004F064FC0246FB689A6007F110030533B9
:10AB6000184604F043FC03461721184604F056FC2F
:10AB70000246FB68DA6007F110030933184604F057
:10AB800035FC03461721184604F048FC0246FB68D2
:10AB90001A6197F82D2097F82E30134407F13002F0
:10ABA000134413F8202C7B681A70002318463037A2
:10ABB000BD4680BDE8140020E815002080B584B0B3
:10ABC00000AF7860084611461A460346FB700B46F4
:10ABD000BB7013467B700023BB607B78002B04D1D5
:10ABE0003B7A43F04003DBB23B72FB787B72BB786D
:10ABF000BB7207F10801002303220C4803F0FDFD9E
:10AC00000346FB73FB7B83F05503FB73FB7BFB72FB
:10AC10007B681B6807F1080104221846FFF7B0FDA6
:10AC2000034618461037BD4680BD00BFE81400201B
:10AC300080B584B000AF7860084611461A460346D6
:10AC4000FB700B46BB7013467B7007F10B02F97863
:10AC500001237868FFF79CFEF860FB68002B01D0A9
:10AC6000FB6818E097F90230DB435AB2FB7A5BB21B
:10AC700013405BB2DBB2FB727A78BB781340DAB276
:10AC8000FB7A1343DBB2FB72FA7AF9780123786816
:10AC9000FFF794FF034618461037BD4680BD80B5C8
:10ACA00086B000AF78607B687B617B69DA697B691D
:10ACB0005B695B6819461046FFF726FC38613B6903
:10ACC000002B16D107F10F02002302217868FFF74D
:10ACD0005FFE38613B69002B0DD17B69DA697B69C6
:10ACE0005B695B6819461046FFF7ECFB386100BFF3
:10ACF00002E000BF00E000BF1837BD4680BD000085
:10AD000084B090B58BB000AF786007F13C0080E86C
:10AD10000E0000233B62BB6C002B02D16FF01503C9
:10AD200030E13021012003F0A7FCF861FB69002B22
:10AD300002D16FF00B0325E107F1080300221A602E
:10AD40005A609A60DA60934BBB60FB69FB60FB6CF6
:10AD5000002B01D0FB6CBB60FB69FA6B11461846F7
:10AD6000FFF718FC78627B6A002B40F00681FB69D4
:10AD700014333A6C11461846FFF7B7F878627B6ACD
:10AD8000002B40F0F180FB695B69002B09D0FB6967
:10AD90005B691846FFF702F978627B6A002B40F086
:10ADA000CE80B86CFB695B695B68194607F10803E4
:10ADB0001A46FFF71AFB78627B6A002B40F0C180CD
:10ADC000FB6903F1200407F108030FCB84E80F00AF
:10ADD000B86CFB695B695B6802221946FFF74DFBA3
:10ADE00078627B6A002B40F09A80B86CFB695B69E3
:10ADF0005B6803221946FFF7A9FB78627B6A002B88
:10AE000040F08F80BA6CFB695B695B68194610463D
:10AE1000FFF77AFB78627B6A002B40F08480BA6C83
:10AE2000FB69DA61FB6918337A6C11461846FFF743
:10AE30005CF878627B6A002B40F09880FB699B6924
:10AE4000002B09D0FB699B6901211846FFF7C8F860
:10AE500078627B6A002B76D107214F4803F090FC83
:10AE600041F221014D4803F020FCFB6901225A7197
:10AE7000FB699B6900211846FFF7D8F878627B6A66
:10AE8000002B62D10A2000F032FBFB699B69012193
:10AE90001846FFF7CBF878627B6A002B57D1322037
:10AEA00000F025FB07F11B031946F86900F096FA3C
:10AEB00078627B6A002B4CD1052000F018FB3B6ABE
:10AEC00001333B623B6A142B03D16FF07F037B623B
:10AED00044E0FB7E002BE5D007F11B031946F8691F
:10AEE00000F0A2FA78627B6A002B34D1FA7EFB690B
:10AEF0001A7107F11B031946F86900F07FFA7862AE
:10AF00007B6A002B29D1FB7E122B03D06FF012033A
:10AF10007B6223E07B68FA691A60002332E000BF9D
:10AF200002E000BF00E000BFB86CFB695B695B68D2
:10AF3000194607F108031A46FFF77BFA0EE000BF37
:10AF40000CE000BF0AE000BF08E000BF06E000BF61
:10AF500004E000BF02E000BF00E000BFFB695B69E6
:10AF60001846FEF7F9FF02E000BF00E000BFFB69F2
:10AF70001B681846FFF7AEFB00E000BFF86903F05E
:10AF800089FB7B6A18462C37BD46BDE8904004B06B
:10AF9000704700BF9FAC0010E8140020E8150020A7
:10AFA00080B584B000AF78607B681B681846FFF7F7
:10AFB00091FBF860FB68002B01D0FB682AE07B68FE
:10AFC0005B691846FEF7C8FFF860FB68002B01D0EC
:10AFD000FB681FE07B689B691846FEF7BDFFF860C1
:10AFE000FB68002B01D0FB6814E07B68D8697B68A4
:10AFF0005B695B6819467B6820331A46FFF719FACC
:10B00000F860FB68002B01D0FB6803E0786803F070
:10B0100041FB002318461037BD4680BD90B486B072
:10B0200000AFF8600B467A60FB724FF000034FF000
:10B030000004C7E90434FB68002B02D16FF012034F
:10B040007FE0FB7A022B02D96FF0150379E0FB7ADF
:10B05000002B02D0012B26D04AE0FB689B684FEA08
:10B06000E3743A4A02FB04F1002202FB03F20A44B1
:10B070003649A3FB013422441446002B74F100022C
:10B0800006DA6FF070414FF000025B1842EB0404E7
:10B090004FF000014FF00002190F41EA041122178E
:10B0A000C7E9041249E0FB68DB684FEAE374274A0A
:10B0B00002FB04F1002202FB03F20A442349A3FB32
:10B0C000013422441446002B74F1000205DA2049B1
:10B0D0004FF000025B1842EB04044FF000014FF008
:10B0E0000002D90D41EA4421E215C7E9041224E027
:10B0F000FB681B694FEAE374144A02FB04F1002267
:10B1000002FB03F20A441149A3FB01342244144612
:10B11000002B74F1000205DA0D494FF000025B18B4
:10B1200042EB04044FF000014FF00002D90D41EA58
:10B130004421E215C7E9041200BF3A697B681A602E
:10B14000002318461837BD4690BC7047AB7C0D00F5
:10B15000FFFF7F0090B585B000AF78600B46FB70B5
:10B16000FB78032B02D96FF0150321E04FF0FF337A
:10B17000FB60FB689B07FB60FB681B0FFB60FB68C9
:10B18000DCB24FF0FF33BB60BB689B07BB60BB68A2
:10B190001B0FBB60BB68FA781146184604F0D7F85D
:10B1A0000346DBB2224602217868FFF741FD0346E1
:10B1B00018461437BD4690BD80B584B000AF7860A6
:10B1C0000B46FB70FB78012B02D96FF0150315E0DD
:10B1D000FB781946022004F0BAF80346DBB20222DB
:10B1E00002217868FFF724FDF860FB68002B01D08E
:10B1F000FB6803E07B68FA785A7100231846103721
:10B20000BD4680BD80B582B000AF78607B68002B02
:10B2100002D16FF0120304E000217868FFF79AFF73
:10B22000034618460837BD4680BD90B585B000AFCF
:10B2300078600B46FB70FB78072B02D96FF0150383
:10B2400027E0FB78072B02D96FF0150321E04FF0C0
:10B25000FF33FB60FB685B07FB60FB685B0FFB6019
:10B26000FB68DCB24FF0FF33BB60BB685B07BB60C1
:10B27000BB685B0FBB60BB68FA781146184604F0E8
:10B2800066F80346DBB2224603217868FFF7D0FC5C
:10B29000034618461437BD4690BD90B585B000AF43
:10B2A00078600B46FB707B68002B02D16FF01203B5
:10B2B00027E0FB78032B02D96FF0150321E04FF054
:10B2C000FF33FB60FB689B07FB60FB681B0FFB60A9
:10B2D000FB68DCB24FF0FF33BB60BB689B07BB6011
:10B2E000BB681B0FBB60BB68FA781146184604F0B8
:10B2F0002EF80346DBB2224612217868FFF798FC4D
:10B30000034618461437BD4690BD90B585B000AFD2
:10B3100078600B46FB707B68002B02D16FF0120344
:10B3200027E0FB78032B02D96FF0150321E04FF0E3
:10B33000FF33FB60FB689B07FB60FB689B0FFB60B8
:10B34000FB68DCB24FF0FF33BB60BB689B07BB60A0
:10B35000BB689B0FBB60BB68FA781146184603F0C8
:10B36000F6FF0346DBB2224612217868FFF760FC45
:10B37000034618461437BD4690BD80B586B000AF71
:10B38000F8607B600B46FB721346BB727B68002B38
:10B3900002D16FF015031DE007F11302F97A0123C2
:10B3A000F868FFF7F5FA78617B69002B01D07B69BB
:10B3B00010E0BB7A184603F0ACFF03461A4607F1CB
:10B3C00013031946104603F08BFF0346DAB27B687D
:10B3D0001A70002318461837BD4680BD80B582B06C
:10B3E00000AF786039603B68102220217868FFF751
:10B3F000C4FF034618460837BD4680BD80B582B0FD
:10B4000000AF786039603B68002B02D16FF0150304
:10B4100006E001233A687D217868FFF7B9FA034610
:10B4200018460837BD4680BD80B584B000AF78604F
:10B4300039603B68002B02D16FF0150324E007F15F
:10B440000B0201237E217868FFF7A2FAF860FB68FF
:10B45000002B01D0FB6817E0FB7A012B07D0032BF0
:10B4600009D0002B0BD13B6800221A700BE03B681F
:10B4700001221A7007E03B6803221A7003E06FF0A4
:10B480001203FB6000BFFB6818461037BD4680BD45
:10B4900080B582B000AF78607B68DA697B685B69F1
:10B4A0005B6819461046FFF70DF803461846083743
:10B4B000BD4680BDF8B500AFF8F702FD054BD3E9F6
:10B4C00000345D1C44F10006024BC3E9005600BF86
:10B4D000F8BD00BFE817002080B582B000AF7860EB
:10B4E0007868F8F711FE00BF0837BD4680BD80B50B
:10B4F00082B000AF78607B684FF47A7202FB03F38E
:10B500001846F8F701FE00BF0837BD4680BD0000B1
:10B51000F0B585B000AF78601A4BD3E900014FF465
:10B520007A724FF0000304F04FFC03460C46BB60F8
:10B53000144BD3E90012BB684FF47A7000FB03F39D
:10B540004FF00004CD1A62EB04062A464FF47A73DA
:10B5500003FB02F20C4B99680C4B1B680C48A0FBD8
:10B5600003039B0CB1FBF3F31344FB607B681A46A7
:10B5700007F1080393E8030082E8030078681437B2
:10B58000BD46F0BDE817002010E000E000000020FC
:10B5900083DE1B4380B485B000AFF860B96013460A
:10B5A000FB71FB79002B06D0FB681A68BB681A4355
:10B5B000FB681A6006E0FB681A68BB68DB431A4048
:10B5C000FB681A6000BF1437BD465DF8047B704706
:10B5D00080B588B000AF786039603B68002B07D039
:10B5E0003B681B69002B03D03B685B681F2B02DDA7
:10B5F0006FF0150391E01421012003F03DF878610C
:10B600007B69002B02D16FF00B0386E00C21012037
:10B6100003F032F838613B69002B03D16FF00B0364
:10B62000FB6176E03B681B69FB603B681B7A012B82
:10B6300006D0022B07D0002B08D10023BB6109E004
:10B640000123BB6106E00223BB6103E06FF0150339
:10B65000FB615BE03B681B68032B03DD6FF01503A8
:10B66000FB6153E03B681B68002B13D03B681B68F1
:10B67000012B0DD03B681B68022B07D03B681B6871
:10B68000032B01D1274B06E0002304E0264B02E008
:10B69000264B00E0264B3A6913603B685B68012249
:10B6A00002FA03F31A463B695A60BB69DAB23B6996
:10B6B0005A723B6900221A72FB681A783B699A72C7
:10B6C0003B681A687B691A603B685A687B695A60F4
:10B6D0003B681A7A7B691A727B693A691A613B681E
:10B6E0001B681846F5F7D4F97B691B691846F5F70E
:10B6F000EBF9F861FB69002B03D06FF01503FB61D8
:10B7000004E07B687A691A60002306E0386902F079
:10B71000C1FF786902F0BEFFFB6918462037BD46BD
:10B7200080BD00BF000608400004084000900040B3
:10B730000080004080B582B000AF786039603B681F
:10B74000002B04D17B6800221A60002304E03968D2
:10B750007868FFF73DFF034618460837BD4680BDB1
:10B7600080B582B000AF78607B68002B02D16FF0AB
:10B77000150308E07B681B69184602F08BFF7868A8
:10B7800002F088FF002318460837BD4680BD80B50B
:10B7900084B000AF78607B68002B03D07B685B6867
:10B7A0001F2B02DD6FF0150309E07B681B69FB604E
:10B7B000FB6800221A72F868F5F786F9002318462C
:10B7C0001037BD4680BD80B584B000AF78600B46B1
:10B7D000FB707B68002B06D07B685B681F2B02DC4C
:10B7E000FB78012B02D96FF0150330E07B681B69F1
:10B7F000FB60FB681B68BB60FB6801221A72F8687B
:10B80000F5F762F97B685B68012202FA03F3012213
:10B810001946B868FFF7BEFEFB78002B02D0012B5B
:10B820000AD013E07B685B68012202FA03F3194631
:10B83000B868F5F71DFB09E07B685B68012202FA36
:10B8400003F31946B868F5F7E5FA00BF0023184678
:10B850001037BD4680BD80B485B000AF78603960D8
:10B860007B68002B03D07B685B681F2B02DD6FF0C9
:10B8700015030EE07B681B69FB60FB681B7A012BDC
:10B8800003D13B6801221A7002E03B6800221A7063
:10B89000002318461437BD465DF8047B704780B519
:10B8A00084B000AF78600B46FB707B68002B03D040
:10B8B0007B685B681F2B02DD6FF0150339E07B6846
:10B8C0001B69FB60FB681B68BB607B685B680122CF
:10B8D00002FA03F301221946B868FFF75BFEFB7812
:10B8E000012B0DD0022B15D0002B1ED17B685B687D
:10B8F000012202FA03F31946B868F5F7B9FA17E01E
:10B900007B685B68012202FA03F31946B868F5F711
:10B9100081FA0DE07B685B68012202FA03F30022E2
:10B920001946B868FFF736FE02E06FF0150300E035
:10B93000002318461037BD4680BD80B584B000AFE7
:10B94000786039607B68002B03D07B685B681F2BB5
:10B9500002DD6FF0150337E07B681B69FB60FB6855
:10B960001B68BB607B685B68012202FA03F301225B
:10B970001946B868FFF70EFEFB681B7A002B11D141
:10B980007B685B68012202FA03F31946B868F5F791
:10B99000EFF902467B685B6822FA03F3DAB23B6890
:10B9A0001A7010E07B685B68012202FA03F3194603
:10B9B000B868F5F78BFA02467B685B6822FA03F3F6
:10B9C000DAB23B681A70002318461037BD4680BDB6
:10B9D00080B483B000AF03463960FB7197F907303C
:10B9E000002B0BDA3B68DAB20C49FB7903F00F034A
:10B9F000043B5201D2B20B441A7609E03B68DAB23A
:10BA0000074997F907305201D2B20B4483F800235B
:10BA100000BF0C37BD465DF8047B704700ED00E0C9
:10BA200000E100E080B586B000AF78607B687B61A4
:10BA30007B695B681C4A934217D07B695B681B4A31
:10BA4000934210D07B695B68194A934209D07B69A5
:10BA50005B68184A934201D1032307E04FF0FF339C
:10BA600004E0022302E0012300E000233B61124ACC
:10BA70003B6952F8233007F108017A69184603F050
:10BA8000FBF9F860FB68002B0AD1BB689B68002BB0
:10BA900007D0BB689B68BA68D2681046984700E038
:10BAA00000BF1837BD4680BD0080004000900040B8
:10BAB0000004084000060840F017002080B500AFE1
:10BAC0000020F5F78AFA00BF80BD80B500AF0120E5
:10BAD000F5F783FA00BF80BD80B500AF0220F5F70F
:10BAE0007CFA00BF80BD000080B584B000AF7860F4
:10BAF00039603B68002B02D16FF0150331E00C2157
:10BB0000012002F0B9FDF860FB68002B02D16FF054
:10BB10000B0326E03B681A68FB681A603B689A686A
:10BB2000FB689A603B681B68104A52F82330002B70
:10BB30000DD13B681B689B000C4A13440C4A03213F
:10BB4000184602F0FDFFB860BB68002B04D17B688B
:10BB5000FA681A60002304E000BFF86802F09AFD5A
:10BB6000BB6818461037BD4680BD00BFF0170020E7
:10BB7000BDC7001080B584B000AF78607B68002B33
:10BB800006D16FF015031DE0FB68184602F082FD38
:10BB90007B681B680D4A52F8233007F10C021146EE
:10BBA000184603F0A2F90346002BEDD07B681B6812
:10BBB000064A52F82330184603F006F8786802F077
:10BBC00069FD002318461037BD4680BDF0170020E0
:10BBD00080B58EB000AFF860B9607A6007F12003DD
:10BBE00000221A605A609A60DA60BB683B62FB68A8
:10BBF000002B02D07B68002B02D16FF01503AAE066
:10BC0000FB681B68564A52F8233007F1200207F1FF
:10BC10003001184603F030F978637B6B002B40D07D
:10BC20001021012002F028FD03463B633B6B002BF3
:10BC300002D16FF00B038EE03B6BBA681A60FB68B1
:10BC40001B68002B13D0FB681B68012B0DD0FB6811
:10BC50001B68022B07D0FB681B68032B01D1414BEB
:10BC600006E0002304E0404B02E0404B00E0404B84
:10BC70003A6B53603B6B7A685268DA603B6B7A6868
:10BC800012689A60FB681B68354A52F823303A6B99
:10BC90001146184602F0F8FF78637B6B002B26D024
:10BCA00054E03B6BBA681A60FB681B68002B13D02A
:10BCB000FB681B68012B0DD0FB681B68022B07D0AB
:10BCC000FB681B68032B01D1264B06E0002304E030
:10BCD000254B02E0254B00E0254B3A6B53603B6B54
:10BCE0007A685268DA603B6B7A6812689A60FB681F
:10BCF0001B68002B13D0FB681B68012B0DD0FB6861
:10BD00001B68022B07D0FB681B68032B01D1154A67
:10BD100006E0002204E0144A02E0144A00E0144A5B
:10BD20000121BB6801FA03F3184607F1140300214F
:10BD30001960596099607A61B8613A6B07F1140330
:10BD40000C491846F5F73AF9002304E03B6B184616
:10BD500002F0A0FC7B6B18463837BD4680BD00BFA3
:10BD6000F017002000060840000408400090004042
:10BD70000080004025BA001080B58EB000AFF8609A
:10BD8000B9607A6000233B6307F1200300221A6048
:10BD90005A609A60DA60BB683B62FB68002B05D092
:10BDA0007B68002B02D0BB681F2B02D96FF01503F4
:10BDB00044E0FB681B68234A52F8233007F1200255
:10BDC00007F13001184603F057F878637B6B002BBE
:10BDD00002D06FF0120331E0FB681B68002B13D018
:10BDE000FB681B68012B0DD0FB681B68022B07D07A
:10BDF000FB681B68032B01D1134A06E0002204E014
:10BE0000124A02E0124A00E0124A0121BB6801FA1C
:10BE100003F3184607F11403002119605960996073
:10BE20007A61B86107F11403002200211846F5F782
:10BE3000C5F83B6B184602F02DFC00231846383736
:10BE4000BD4680BDF01700200006084000040840F1
:10BE50000090004000800040B0B58CB000AFF860AA
:10BE6000B9601346FB71254B07F110041D460FCD39
:10BE70000FC42B682360FB68002B02D0BB681F2B0C
:10BE800002D96FF0150334E0FB681B68002B13D058
:10BE9000FB681B68012B0DD0FB681B68022B07D0C9
:10BEA000FB681B68032B01D1154A06E0002204E061
:10BEB000144A02E0144A00E0144A0121BB6801FA66
:10BEC00003F3184607F124030021196059609960B3
:10BED0007A62B862FB799B0007F13002134453F891
:10BEE000203CDAB207F1240311461846F5F73CF876
:10BEF000002318463037BD46B0BD00BF3871011071
:10BF00000006084000040840009000400080004007
:10BF100080B582B000AF786039603B681F2B02D9D2
:10BF20006FF0150321E07B681B68002B13D07B6842
:10BF30001B68012B0DD07B681B68022B07D07B6828
:10BF40001B68032B01D10B4B06E0002304E00A4BD6
:10BF500002E00A4B00E00A4B01213A6801FA02F2C2
:10BF600011461846F5F710F8002318460837BD4665
:10BF700080BD00BF0006084000040840009000405B
:10BF80000080004080B582B000AF786039603B68C7
:10BF90001F2B02D96FF0150321E07B681B68002B73
:10BFA00013D07B681B68012B0DD07B681B68022BAC
:10BFB00007D07B681B68032B01D10B4B06E00023E5
:10BFC00004E00A4B02E00A4B00E00A4B01213A6808
:10BFD00001FA02F211461846F4F7E3FF002318466F
:10BFE0000837BD4680BD00BF000608400004084079
:10BFF000009000400080004080B584B000AF7860C1
:10C000007B681B68002B13D07B681B68012B0DD04D
:10C010007B681B68022B07D07B681B68032B01D150
:10C020000A4B06E0002304E0094B02E0094B00E064
:10C03000094B4FF0FF32FA60FA6811461846F4F7E0
:10C04000A3FF002318461037BD4680BD00060840F8
:10C0500000040840009000400080004080B584B09B
:10C0600000AF78607B681B68002B13D07B681B686F
:10C07000012B0DD07B681B68022B07D07B681B68E7
:10C08000032B01D10A4B06E0002304E0094B02E038
:10C09000094B00E0094B4FF0FF32FA60FA68114695
:10C0A0001846F4F77EFF002318461037BD4680BDC2
:10C0B0000006084000040840009000400080004056
:10C0C00080B586B000AFF860B9607A60FB681B6825
:10C0D000002B0DD0FB681B68012B07D0FB681B6889
:10C0E000022B01D11A2304E0002302E0192300E00F
:10C0F00018237B617B695BB279681846FFF768FC9F
:10C10000002318461837BD4680BD000080B483B0B8
:10C1100000AF0346FB71FB7903F01F03012202FA13
:10C1200003F1064A97F907305B09203342F82310E0
:10C1300000BF0C37BD465DF8047B704700E100E0AE
:10C1400080B500AF0248F5F777FA00BF80BD00BFA9
:10C1500000D0014080B500AF0248F5F76DFA00BF8E
:10C1600080BD00BF00E0014080B500AF0248F5F798
:10C1700063FA00BF80BD00BF00F0014080B586B00B
:10C1800000AF78600B46FB707B68012B0DD07B689D
:10C19000002B03D07B68022B0ED014E0114A07F16C
:10C1A0000C0307CA83E8070010E00F4A07F10C03ED
:10C1B00007CA83E8070009E00C4A07F10C0307CA25
:10C1C00083E8070002E06FF0150307E0FB78BB751A
:10C1D00007F10C031846F4F777FC002318461837CC
:10C1E000BD4680BD506501105C6501106865011099
:10C1F00080B588B000AF786039607B68002B06D0CE
:10C200003B68002B03D03B681B69002B02D16FF009
:10C210001503C7E03B681B68022B02D96FF01503BA
:10C22000C0E01821012002F027FA02467B681A605C
:10C230007B681B68002B02D16FF00B03B2E00C216E
:10C24000012002F019FAB861BB69002B03D16FF02D
:10C250000B03FB61A0E03B681B697B613B681B68CB
:10C26000002B0DD03B681B68012B07D03B681B6877
:10C27000022B01D14D4B04E0002302E04C4B00E0C7
:10C280004C4B3B61BB693A691A607B681B683A6832
:10C2900012685A603B685B68474A934204D87B68DF
:10C2A0001B68454A9A6021E03B685B68434A9342B9
:10C2B00004D87B681B68414A9A6017E03B685B685A
:10C2C0003F4A934204D87B681B683D4A9A600DE060
:10C2D0003B685B683B4A934204D87B681B68394AD9
:10C2E0009A6003E06FF01503FB6152E07B681B6806
:10C2F0003A68127A1A737B681B68BA695A613B689C
:10C300001B68314A52F82330002B10D1BB691B68DF
:10C310001846F5F7A5F8002201213869F5F746F827
:10C320000346002B03D04FF0FF33FB6131E07B6805
:10C330001B685A687B691B7819461046FFF71EFF79
:10C34000F861FB69002B01D0FB692BE03869F5F738
:10C35000D3F80346FB607B681B689B68FA689342CE
:10C3600028BF1346FB60F9683869F5F7ADF8F86146
:10C37000FB69002B02DA6FF0150313E03B681B68C2
:10C38000114A52F8232001320F4941F8232000239B
:10C3900008E0B86902F07EF97B681B68184602F075
:10C3A00079F9FB6918462037BD4680BD00F0014091
:10C3B00000E0014000D00140A0860100801A060084
:10C3C00040420F0040E133000018002080B584B0E7
:10C3D00000AF78607B685B69FB607B68002B02D1F3
:10C3E0006FF0150337E07B685B681D4A52F8232025
:10C3F000013A1B4941F823207B685B68184A52F8D0
:10C400002330002B20D1FB681B681846F5F728F86D
:10C41000B860BB68002B01D0BB681CE07B685B6820
:10C42000002B0DD07B685B68012B07D07B685B68B5
:10C43000022B01D13E2304E0002302E0242300E08C
:10C440000D231846FFF762FEF86802F023F97868BA
:10C4500002F020F9002318461037BD4680BD00BF0A
:10C460000018002080B590B000AFF860B9601146A8
:10C470001A460B46FB711346BB71FB68002B03D0B9
:10C48000FB685B69002B02D16FF0150358E0FB6875
:10C490005B68002B0DD0FB685B68012B07D0FB6845
:10C4A0005B68022B01D1284B04E0002302E0274BFC
:10C4B00000E0274BFB63FB685B69BB63BB79002B28
:10C4C00029D1BB6BFA791A72BB6B5B68002B0BD05E
:10C4D000BB6B5B68FA791146184604F089FA7863F9
:10C4E000BB6B7A6B5A600DE0FB79184602F0B8F826
:10C4F0000246BB6B5A60BB6B5B68002B02D16FF0CE
:10C500000B031DE0BB6B5B68FA79B968184604F051
:10C5100021F9002314E0FB6B7B61FB681B7BBB6193
:10C52000BB68FB61FB793B620023BB62BB687B623B
:10C530000023FB6207F114031846F5F754F803468D
:10C5400018464037BD4680BD00F0014000E0014084
:10C5500000D0014080B590B000AFF860B9601146DE
:10C560001A460B46FB711346BB71FB68002B03D0C8
:10C57000FB685B69002B02D16FF015034CE0FB6890
:10C580005B69FB63FB685B68002B0DD0FB685B6835
:10C59000012B07D0FB685B68022B01D1204B04E024
:10C5A000002302E01F4B00E01F4BBB63BB6B7B61B2
:10C5B000FB681B7BBB6100233B620023FB61BB6804
:10C5C0007B62FB79BB62BB79002B0CBF012300238C
:10C5D000DBB2FB62FB6B1B7A002B07D00023FB62F4
:10C5E000FB6B1B7A3B62FB6B5B68FB6107F114031F
:10C5F0001846F4F7F8FF7863FB6B1B7A002B0AD020
:10C60000FB6B5B68184602F045F8FB6B00221A7260
:10C61000FB6B00225A607B6B18464037BD4680BDDD
:10C6200000F0014000E0014000D0014080B483B040
:10C6300000AF03463960FB7197F90730002B0BDA26
:10C640003B68DAB20C49FB7903F00F03043B52015B
:10C65000D2B20B441A7609E03B68DAB2074997F97F
:10C6600007305201D2B20B4483F8002300BF0C37CD
:10C67000BD465DF8047B704700ED00E000E100E09E
:10C6800080B582B000AF78607B68013BB3F1807FFA
:10C6900001D301230FE00A4A7B68013B5360072165
:10C6A0004FF0FF30FFF7C2FF054B00229A60044BAA
:10C6B00007221A60002318460837BD4680BD00BF18
:10C6C00010E000E080B500AF074B1B68074AA2FBF3
:10C6D00003239B091846FFF7D3FF0120F7F714FD4A
:10C6E0000346184680BD00BF00000020D34D6210F5
:10C6F00080B500AFFFF7E6FF0346184680BD000097
:10C7000080B483B000AF0346FB71FB7903F01F03D5
:10C71000012202FA03F1064A97F907305B0942F851
:10C72000231000BF0C37BD465DF8047B704700BF87
:10C7300000E100E080B483B000AF0346FB71FB79F9
:10C7400003F01F03012202FA03F1064A97F90730AA
:10C750005B09203342F8231000BF0C37BD465DF85B
:10C76000047B704700E100E080B483B000AF034673
:10C770003960FB7197F90730002B0BDA3B68DAB2AE
:10C780000C49FB7903F00F03043B5201D2B20B4476
:10C790001A7609E03B68DAB2074997F90730520187
:10C7A000D2B20B4483F8002300BF0C37BD465DF8BE
:10C7B000047B704700ED00E000E100E080B483B04E
:10C7C00000AF786039607B681A683B681B68D31AD1
:10C7D00018460C37BD465DF8047B704780B485B0C1
:10C7E00000AF78600023FB6017E0FB68002B0BD0E4
:10C7F000FB68012B06D0FB68022B01D11A2304E051
:10C80000002302E0192300E018237A68934201D143
:10C81000012306E0FB680133FB60FB68032BE4D9CE
:10C82000002318461437BD465DF8047B70470000AE
:10C8300080B58AB000AF786007F1100300221A605B
:10C840005A609A60DA607B68404A93425BD07B68AA
:10C850003E4A934203D07B683D4A934251D07B6865
:10C860003A4A934207D07B68394A934203D07B68A7
:10C87000384A934243D07B68344A93420BD07B685A
:10C88000334A934207D07B68324A934203D07B6895
:10C89000314A934231D07B682C4A93420FD07B6857
:10C8A0002B4A93420BD07B682A4A934207D07B687D
:10C8B000294A934203D07B68284A93421BD07B6865
:10C8C000224A934215D07B68214A934211D07B685B
:10C8D000204A93420DD07B681F4A934209D07B685F
:10C8E0001E4A934205D07B681D4A934201D10A2318
:10C8F0000AE0002308E0092306E0082304E00723F8
:10C9000002E0062300E005233B61164B7B627B6A55
:10C910005B6807F1100207F10C01184602F0ACFA4F
:10C9200038623B6A002B0DD1FB689B68002B05D059
:10C93000FB689B68FA68D268104698477868F8F7F1
:10C94000B9F800E000BF2837BD4680BD00000140B7
:10C95000001001400020014000300140000C084060
:10C96000001008408401002080B584B000AF7860DA
:10C970007B681B4A934214D07B681A4A93420ED0BC
:10C980007B68194A934208D07B68184A934201D1C8
:10C99000032307E04FF0FF3304E0022302E001230A
:10C9A00000E000235B01124A1344FB607868F9F74A
:10C9B00021F9FB681B68002B0ED0FB689B69002BDC
:10C9C00003D1FB681B69002B03D1FB68DB68002BDC
:10C9D00002D0F868F9F7F6F800BF1037BD4680BD01
:10C9E000002004400030044000400440001408408F
:10C9F0008418002080B500AF0248FFF7B5FF00BFE4
:10CA000080BD00BF0020044080B500AF0248FFF7A2
:10CA1000ABFF00BF80BD00BF0030044080B500AF59
:10CA20000248FFF7A1FF00BF80BD00BF00400440E7
:10CA300080B500AF0248FFF797FF00BF80BD00BF81
:10CA40000014084080B500AF0248FFF7F1FE00BFB8
:10CA500080BD00BF0000014080B500AF0248FFF775
:10CA6000E7FE00BF80BD00BF0010014080B500AFF1
:10CA70000248FFF7DDFE00BF80BD00BF002001407F
:10CA800080B584B000AFF5F703FE0346FB60124BA0
:10CA9000BB60FB6803F04003002B19D04020F5F782
:10CAA00001FEBB685B683A461146184602F096F9EB
:10CAB00078607B68002B0ADB3B689B68002B07D003
:10CAC0003B689B683A68D2681046984700E000BF10
:10CAD0001037BD4680BD00BF7401002080B58AB00C
:10CAE00000AF786039607B681B68414A934217D079
:10CAF0007B681B683F4A934210D07B681B683E4AA4
:10CB0000934209D07B681B683C4A934201D10323BE
:10CB100007E04FF0FF3304E0022302E0012300E0CE
:10CB200000233B6207F1080300221A605A609A60F2
:10CB3000DA603B6A002B10D03B6A012B0BD03B6ABA
:10CB4000022B06D03B6A032B01D1582306E00023B9
:10CB500004E0222302E00F2300E00E23BB603B68C9
:10CB6000002B02D0264B7B6218E07B68DA687B687A
:10CB70005B699A4206D17B68DB68002B02D0214BAF
:10CB80007B620BE07B681A697B689B699A4229D1BA
:10CB90007B681B69002B25D01B4B7B627B6A5B6823
:10CBA00007F1080207F11801184602F065F9F8616B
:10CBB000FB69002B18D1154A3B6A5B011344002224
:10CBC0001A60BB699B68002B0FD0114B01221A70B1
:10CBD000BB699B68BA69D268104698470C4B002223
:10CBE0001A7002E000BF00E000BF2837BD4680BDDC
:10CBF000002004400030044000400440001408407D
:10CC00006C0100205C0100206401002084180020D9
:10CC10008018002080B584B000AF786039603B6830
:10CC2000002B02D16FF0150316E00C21012001F05A
:10CC300023FDF860FB68002B02D16FF00B030BE0C3
:10CC40003B681A68FB681A603B689A68FB689A60E0
:10CC50007B68FA681A60002318461037BD4680BD0D
:10CC600080B584B000AF78607B68002B02D16FF094
:10CC7000150326E00023FB601CE0BB68184601F0AA
:10CC800009FD124AFB68DB0013445B6807F10802E8
:10CC90001146184602F029F90346002BEDD00B4A45
:10CCA000FB68DB0013445B68184601F08DFFFB68EE
:10CCB0000133FB60FB68062BE3D9786801F0EAFCDE
:10CCC000002318461037BD4680BD00BF5401002028
:10CCD00080B58AB000AFF860B9607A6007F11003E0
:10CCE00000221A605A609A60DA60BB683B61B868DB
:10CCF000FFF774FD0346002B02D06FF0570340E1AD
:10CD0000FB68002B02D07B68002B02D16FF015036B
:10CD100037E17B685B7A022B6BD0032B00F0C48079
:10CD2000012B40F021817B681B7A984ADB00134479
:10CD30005B68002B10D17B681B7ADB00934A13449D
:10CD40000433934A0321184601F0FAFE78627B6AA5
:10CD5000002B01D07B6A14E17B681B7A8B4ADB00D5
:10CD600013445B6807F1100207F12001184602F036
:10CD700083F878627B6A002B2BD01021012001F010
:10CD80007BFC03463B623B6A002B02D16FF00B0336
:10CD9000F7E03B6ABA681A603B6A7A68D2685A6000
:10CDA0003B6A7A6812689A603B6A7A685268DA600D
:10CDB0007B681B7A754ADB0013445B683A6A11464C
:10CDC000184601F061FF78627B6A002B00F0CF808B
:10CDD000D2E03B6ABA681A603B6A7A68D2685A60E5
:10CDE0003B6A7A6812689A603B6A7A685268DA60CD
:10CDF000BDE0664B5B6A002B0AD1654A032165489A
:10CE000001F09EFE78627B6A002B01D07B6AB8E05D
:10CE10005E4B5B6A07F120021146184601F0DEFF07
:10CE200078627B6A002B26D01021012001F024FCBF
:10CE300003463B623B6A002B02D16FF00B03A0E07C
:10CE40003B6ABA681A603B6A7A68D2685A603B6A81
:10CE50007A6812689A603B6A7A685268DA604B4B6B
:10CE60005B6A3A6A1146184601F0D9FE78627B6A1D
:10CE7000002B0FD080E03B6ABA681A603B6A7A6880
:10CE8000D2685A603B6A7A6812689A603B6A7A682C
:10CE90005268DA600220F5F7DBFB78627B6A002BD0
:10CEA00067D06FF00F036CE0384B5B6B002B0AD13F
:10CEB000374A0321384801F043FE78627B6A002B31
:10CEC00001D07B6A5DE07B681B7A304ADB0013444B
:10CED0005B6807F1100207F12001184601F0CCFF52
:10CEE00078627B6A002B2AD01021012001F0C4FB5C
:10CEF00003463B623B6A002B02D16FF00B0340E01C
:10CF00003B6ABA681A603B6A7A68D2685A603B6AC0
:10CF10007A6812689A603B6A7A685268DA607B685D
:10CF20001B7A1A4ADB0013445B683A6A11461846BA
:10CF300001F0AAFE78627B6A002B0FD01CE03B6AEE
:10CF4000BA681A603B6A7A68D2685A603B6A7A6843
:10CF500012689A603B6A7A685268DA607B68DB68BC
:10CF60001846F7F7B2FD05E06FF0150309E000BFC2
:10CF700000E000BF002304E03B6A184601F08AFB92
:10CF80007B6A18462837BD4680BD00BF540100208B
:10CF9000BDC70010780100208801002080B58AB04C
:10CFA00000AFF860B9607A6000233B6207F11003BC
:10CFB00000221A605A609A60DA60BB683B61B86808
:10CFC000FFF70CFC0346002B02D06FF057033AE04A
:10CFD000FB68002B02D07B68002B02D16FF0150399
:10CFE00031E07B685B7A022B07D0032B0BD0012B3F
:10CFF0000FD17B68DB687B610CE0154B7B61022005
:10D00000F5F736FB06E07B68DB681846F7F768FD46
:10D0100000E000BF7B681B7A0E4ADB0013445B68AC
:10D0200007F1100207F12001184601F0E0FF7862D5
:10D030007B6A002B02D06FF0120304E03B6A1846B3
:10D0400001F028FB7B6A18462837BD4680BD00BF2B
:10D05000006000405401002080B485B000AFF8604B
:10D06000B9601346FB716FF0570318461437BD467D
:10D070005DF8047B704780B483B000AF786062B61F
:10D08000002318460C37BD465DF8047B704780B41A
:10D0900083B000AF786072B6002318460C37BD46E7
:10D0A0005DF8047B704780B582B000AF786039606E
:10D0B0003B68672B02D96FF0150305E03B685BB254
:10D0C0001846FFF71DFB002318460837BD4680BDF4
:10D0D00080B582B000AF786039603B68672B02D9B9
:10D0E0006FF0150305E03B685BB21846FFF722FBC3
:10D0F000002318460837BD4680BD80B584B000AF18
:10D10000F860B9607A60BB68672B02D96FF01503CD
:10D1100006E0BB685BB279681846FFF725FB002381
:10D1200018461037BD4680BD80B58AB000AF786024
:10D1300039607B68DB693B623B685B694FF47A72FC
:10D1400002FB03F27B685B691344FB613B689B69EC
:10D150004FF47A7202FB03F27B689B691344BB6154
:10D160003B6A5B68FA699A4204D13B6A9B68BA6978
:10D170009A4277D07B685B68002B07D07B685B683E
:10D18000012B01D1394B02E0002300E0384B7B61D9
:10D190007B691B693B617869F5F77AFD0346FB60A3
:10D1A000FB685A08334B1344FA68B3FBF2F3BB60D5
:10D1B0003B6A5B68FA699A4221D0FB69002B02D175
:10D1C00001237B6204E0FA69BB68B2FBF3F37B6284
:10D1D0007B6AFF2B03D9284803F002FC3EE07B6901
:10D1E0001B6923F0FF027B691A61796AFF2002F054
:10D1F000AEF802467B691B691A437B691A613B6A78
:10D200009B68BA699A4222D0BB69002B02D10123E4
:10D210007B6204E0BA69BB68B2FBF3F37B627B6AB2
:10D22000FF2B03D9154803F0DBFB17E07B691B6973
:10D2300023F47F427B691A61796A4FF47F4002F0E0
:10D2400086F802467B691B691A437B691A613B6A4F
:10D25000FA695A603B6ABA699A6004E07B693A6984
:10D260001A6100E000BF2837BD4680BD00E00B40DA
:10D270000060044000CA9A3BAC710110D8710110E3
:10D28000F0B591B006AF78607B68DB69FB61FB6944
:10D290001B68BB6101233B737B681B7B002B0CBFAE
:10D2A00001230023DBB27B737B681B7B012B0CBF4C
:10D2B00001230023DBB2BB737B681B7B022B0CBFFB
:10D2C00001230023DBB2FB7301233B7401237B7436
:10D2D0000023BB740023FB74FB691B685B79002B84
:10D2E00014BF01230023DBB23B757B685B68002B16
:10D2F00007D07B685B68012B01D1534C02E000240E
:10D3000000E0524CBB691B689C46BB691B791E46FA
:10D310007B689D6802AB07F10C0207CA03C31A7051
:10D32000019500966346002201212046F5F768FB2F
:10D3300038623B6A002B03D06FF015033B626EE04E
:10D340007B685B7B032B18D801A252F823F000BF47
:10D3500071D3001061D3001069D3001071D3001095
:10D36000022387F827300BE0012387F8273007E0F6
:10D370007B685B7B87F8273002E06FF015035FE086
:10D380007B685B68002B07D07B685B68012B01D151
:10D390002D4B02E0002300E02C4B97F8272011468C
:10D3A0001846F5F72DFD38623B6A002B03D06FF06D
:10D3B00015033B6233E07B685B68002B07D07B681A
:10D3C0005B68012B01D1204B02E0002300E01F4BE2
:10D3D00001211846F5F7F8FC38623B6A002B03D0B0
:10D3E0006FF015033B621AE07B685B68002B07D087
:10D3F0007B685B68012B01D1134B02E0002300E046
:10D40000124B08211846F5F7B7FC38623B6A002B2F
:10D4100003D06FF015033B6201E0002310E07B684E
:10D420005B68002B07D07B685B68012B01D1064B42
:10D4300002E0002300E0054B1846F5F7F7FB3B6AD6
:10D4400018462C37BD46F0BD00E00B40006004409C
:10D4500080B586B000AF786039603B68002B03D0A0
:10D460003B689B69002B02D16FF015035FE024211C
:10D47000012001F001F938613B69002B02D16FF006
:10D480000B0354E00C21012001F0F6F8F860FB6872
:10D49000002B03D16FF00B037B6141E03B689B697C
:10D4A000BB603B681A683B695A603B685A683B69D5
:10D4B0009A603B681A7A3B691A733B685A7A3B69EF
:10D4C0005A733B689A7A3B699A73FB68BA681A6028
:10D4D0003B69FA68DA613B695B68012B03D96FF03D
:10D4E00015037B611CE03869FFF7CAFE78617B6930
:10D4F000002B04D17B683A691A60002317E000BF53
:10D500003B695B68002B07D03B695B68012B01D14D
:10D51000094B02E0002300E0084B1846F5F786FBB4
:10D52000F86801F0B7F8386901F0B4F87B6918467B
:10D530001837BD4680BD00BF00E00B4000600440CE
:10D5400080B582B000AF78607B68002B02D16FF0AD
:10D55000150318E07B685B68002B07D07B685B686D
:10D56000012B01D10A4B02E0002300E0094B1846D1
:10D57000F5F75CFB7B68DB69184601F08BF878688F
:10D5800001F088F8002318460837BD4680BD00BF6B
:10D5900000E00B400060044080B58CB000AFF86044
:10D5A000B9607A60FB685B68002B07D0FB685B683A
:10D5B000012B01D1764B02E0002300E0754BFB61AB
:10D5C000012387F82730012387F8263000233B62A8
:10D5D000FB68002B02D0BB68002B02D16FF0150353
:10D5E000A0E1FB681B7BBB61FB685B686A4A52F881
:10D5F0002330BA699A420ED0F868FFF741FE78618D
:10D600007B69002B01D07B698CE1FB685B68624918
:10D61000BA6941F82320FB695B6823F47022FB6937
:10D620005A60FB681B7B1A460123934019464FF44E
:10D63000702001F08CFE0246FB695B681A43FB69AF
:10D640005A6000233B6267E1FB69DB6943F08012AB
:10D65000FB69DA61FB691B6A43F40062FB691A62C9
:10D66000FB6900229A600023BB620023FB623A6AD6
:10D670001346DB009B1A9B001A46BB6813441B7BB6
:10D68000002B06D0FB695B6823F48072FB695A604B
:10D6900005E0FB695B6843F48072FB695A603A6A93
:10D6A0001346DB009B1A9B001A46BB6813441946BD
:10D6B000F868FFF739FD3A6A1346DB009B1A9B00B6
:10D6C0001A46BB6813441B68002B3AD0BB689A68A3
:10D6D000FB699A60002387F82630FB69DB6943F019
:10D6E0004002FB69DA613A6A1346DB009B1A9B0031
:10D6F0001A46BB6813441A68FB6AD1183A6A134683
:10D70000DB009B1A9B001A46BB6813449A68FB6AAD
:10D71000D31A1A46F869F5F7B7FB0246FB6A1344B9
:10D72000FB623A6A1346DB009B1A9B001A46BB68F1
:10D7300013449B68FA6A9A420CBF0123002387F8BE
:10D7400026303A6A1346DB009B1A9B001A46BB68D8
:10D7500013445B68002B14D0BB689B6819460F48C4
:10D7600001F0F5FD0246FB699B681A43FB699A606C
:10D77000FB69DB6943F48002FB69DA61002387F807
:10D780002730FB695B6843F02002FB695A6091E037
:10D7900000E00B40006004400C1800200000FFFF78
:10D7A0003A6A1346DB009B1A9B001A46BB68134477
:10D7B0001B68002B39D03A6A1346DB009B1A9B008A
:10D7C0001A46BB6813449B68FA6A9A422DD23A6A99
:10D7D0001346DB009B1A9B001A46BB6813441A6869
:10D7E000FB6AD1183A6A1346DB009B1A9B001A4663
:10D7F000BB6813449A68FB6AD31A1A46F869F5F7AE
:10D8000043FB0246FB6A1344FB623A6A1346DB00A1
:10D810009B1A9B001A46BB6813449B68FA6A9A429B
:10D820000CBF0123002387F826303A6A1346DB0039
:10D830009B1A9B001A46BB6813445B68002B39D0C7
:10D840003A6A1346DB009B1A9B001A46BB681344D6
:10D850009B68BA6A9A422DD23A6A1346DB009B1A39
:10D860009B001A46BB6813445A68BB6AD1183A6ACF
:10D870001346DB009B1A9B001A46BB6813449A6848
:10D88000BB6AD31A1A46F869F5F7E2FA0246BB6A90
:10D890001344BB623A6A1346DB009B1A9B001A468C
:10D8A000BB6813449B68BA6A9A420CBF01230023E9
:10D8B00087F8273097F8273083F00103DBB2002B7D
:10D8C0007FF46EAF97F8263083F00103DBB2002BB4
:10D8D0007FF466AF00BFFB691B6A03F40063002B93
:10D8E000F9D0FB695B6823F02002FB695A60FB6991
:10D8F000DB6923F04012FB69DA613A6A1346DB0008
:10D900009B1A9B001A46BB6813441B691846FDF717
:10D91000E3FD3B6A01333B623A6A7B689A42FFF45B
:10D9200093AE002318463037BD4680BD80B58CB01D
:10D9300000AFF860B9601346FB8007F114030022C2
:10D940001A605A609A60DA601A615A619A61BB681B
:10D950007B61BB68BB61FB88FB61012387F82030DA
:10D9600007F1140301221946F868FFF715FE034674
:10D9700018463037BD4680BD80B483B000AF7860B4
:10D98000396000BF0C37BD465DF8047B704700006E
:10D9900080B586B000AF78600B46FB707B68012BCA
:10D9A0000DD07B68002B03D07B68022B0ED014E0D7
:10D9B000114A07F10C0307CA83E8070010E00F4A79
:10D9C00007F10C0307CA83E8070009E00C4A07F1D6
:10D9D0000C0307CA83E8070002E06FF0150307E0B5
:10D9E000FB78BB7507F10C031846F3F76DF80023BD
:10D9F00018461837BD4680BD746501109865011042
:10DA0000BC65011080B586B000AFF860B9607A607F
:10DA100000237B61FB68002B05D0BB68002B02D084
:10DA20007B68002B02D16FF0150349E0FB68DB68CF
:10DA3000002B1FD000237B6116E0FB68D868BA6812
:10DA40007B691344194600F050FF38613B69002B95
:10DA500007D07B69002B01D07B6931E06FF00A03AE
:10DA60002EE07B6901337B617B687A699A42E4D35B
:10DA70007B6925E0FB681B79002B13D0FB681B79C1
:10DA8000012B0DD0FB681B79022B07D0FB681B799B
:10DA9000032B01D10C4B06E0002304E00B4B02E00A
:10DAA0000B4B00E00B4B3A1DB9681846F7F7CAFF5D
:10DAB00038613B69002B02D06FF0040300E07B6803
:10DAC00018461837BD4680BD001408400040044089
:10DAD000003004400020044080B588B000AFF860FA
:10DAE000B9607A600023FB61FB68002B05D0BB683E
:10DAF000002B02D07B68002B5AD16FF015035BE03E
:10DB00007B68082B28BF08237B6100BFFB681B795B
:10DB1000002B13D0FB681B79012B0DD0FB681B7900
:10DB2000022B07D0FB681B79032B01D1244B06E0A5
:10DB3000002304E0234B02E0234B00E0234B184674
:10DB4000F8F734F8034603F04003002BDED0FB68FF
:10DB50001B79002B13D0FB681B79012B0DD0FB68C0
:10DB60001B79022B07D0FB681B79032B01D1144BC7
:10DB700006E0002304E0134B02E0134B00E0134BDC
:10DB8000FA69B968114407F114021846F7F76AFFF9
:10DB9000B8617B69FA691344FB617B691A467B684B
:10DBA0009B1A7B60BB69002B02D06FF0040303E07B
:10DBB0007B68002BA4D1FB6918462037BD4680BD89
:10DBC000001408400040044000300440002004409D
:10DBD00080B586B000AFF860B9607A60FB68002B52
:10DBE00005D0BB68002B02D07B68002B02D16FF000
:10DBF00015035DE0FB681B797B617B69002B10D00E
:10DC00007B69012B0BD07B69022B06D07B69032B30
:10DC100001D1294B06E0002304E0284B02E0284B09
:10DC200000E0284B28497A6952010A441360264AC9
:10DC30007B695B0113440833BA681A60224A7B6926
:10DC40005B01134410337A681A601F4A7B695B01D9
:10DC50001344043300221A601B4A7B695B0113449E
:10DC60000C3300221A60184A7B695B011344183395
:10DC700000221A60144A7B695B0113441C33134A67
:10DC80001A60134B1B7883F00103DBB2002B0ED01C
:10DC90007B695B010C4A13441846F7F793FF386120
:10DCA0003B6913F1060F02D16FF00F0300E0002370
:10DCB00018461837BD4680BD001408400040044097
:10DCC000003004400020044084180020DDCA001009
:10DCD0008018002080B586B000AFF860B9607A6027
:10DCE000FB68002B05D0BB68002B02D07B68002BA3
:10DCF00002D16FF015035DE0FB681B797B617B69E6
:10DD0000002B10D07B69012B0BD07B69022B06D036
:10DD10007B69032B01D1294B06E0002304E0284B4B
:10DD200002E0284B00E0284B28497A6952010A4456
:10DD30001360264A7B695B0113440433BA681A6096
:10DD4000224A7B695B0113440C337A681A601F4ACC
:10DD50007B695B011344083300221A601B4A7B690C
:10DD60005B011344103300221A60184A7B695B017F
:10DD70001344143300221A60144A7B695B01134474
:10DD80001C33134A1A60134B1B7883F00103DBB278
:10DD9000002B0ED07B695B010C4A13441846F7F741
:10DDA00011FF38613B6913F1060F02D16FF00F03C9
:10DDB00000E0002318461837BD4680BD0014084017
:10DDC000004004400030044000200440841800203B
:10DDD000DDCA00108018002080B584B000AF7860E4
:10DDE0007B68FB60FB68DA68074B1B7819461046B6
:10DDF00000F09CFD01220449F868FFF7E9FE00BF2E
:10DE00001037BD4680BD00BF1418002080B592B009
:10DE100000AF786039603B68002B03D03B689B699A
:10DE2000002B02D16FF01503AAE11C21012000F0A4
:10DE300023FCF862FB6A002B02D16FF00B039FE119
:10DE40000421012000F018FCB862FB6A002B03D10A
:10DE50006FF00B037B6489E1FB6ABA6A9A613B68E5
:10DE60001B78002B13D03B681B78012B0DD03B682F
:10DE70001B78022B07D03B681B78032B01D1924BF8
:10DE800006E0002304E0914B02E0914B00E0914B4F
:10DE90003B633B689B697B623B681A78FB6A1A713B
:10DEA0003B68DA68FB6A1A613B685B7C032B06D02F
:10DEB000042B07D0002B08D100237B6309E0042347
:10DEC0007B6306E002237B6303E06FF015037B6452
:10DED0004CE13B681B7C032B16D801A252F823F0BF
:10DEE000F1DE0010F7DE0010FDDE001003DF001091
:10DEF0000523FB630CE00623FB6309E00723FB63B8
:10DF000006E00823FB6303E06FF015037B642DE15B
:10DF10003B689B7C002B02D0012B03D005E0002343
:10DF20003B6406E001233B6403E06FF015037B6470
:10DF30001CE17B6A1B78002B04D0002B08DB022B32
:10DF400006DC02E00023BB6306E00123BB6303E0C1
:10DF50006FF015037B6409E1FB6A1B690022194617
:10DF6000386BF7F7E9F978647B6C002B03D06FF01E
:10DF700015037B64FAE0FB6A1B791A467B6A5B78BF
:10DF800019461046FFF704FD78647B6C002B01D026
:10DF90007B6CF5E0F96B386BF7F766FC78647B6CAB
:10DFA000002B03D06FF015037B64DFE07B6BDBB2EB
:10DFB0001946386BF7F776FC78647B6C002B03D03E
:10DFC0006FF015037B64D1E03B6CDBB21946386B14
:10DFD000F7F758FC78647B6C002B03D06FF01503C7
:10DFE0007B64C3E0BB6BDBB208221946386BF7F7E2
:10DFF00069FC78647B6C002B03D06FF015037B64A5
:10E00000B4E07B68FA6A1A603B681B7A002B00F068
:10E010009D80FB6A0C33184600F011FC78647B6C21
:10E02000002B40F0A08007F1180300221A605A600C
:10E030009A60294BFB61BB6A07F11802114618462A
:10E04000FCF786F978647B6C002B40F08E80234BC4
:10E05000BB60FB6AFB6002233B7401237B74FB6A99
:10E060001B79002B13D0FB6A1B79012B0DD0FB6AA7
:10E070001B79022B07D0FB6A1B79032B01D1124BB2
:10E0800006E0002304E0114B02E0114B00E0114BCD
:10E090007B61BB6A1868FB6A1B79002B20D0FB6A86
:10E0A0001B79012B0DD0FB6A1B79022B07D0FB6A71
:10E0B0001B79032B01D1582313E0002311E0222305
:10E0C0000FE00F230DE000BF0014084000400440A3
:10E0D000003004400020044084710110D9DD00109C
:10E0E0000E2307F108021946FCF77FF978647B6C70
:10E0F000002B2DD1BB6A1A68FB6A1B79002B13D049
:10E10000FB6A1B79012B0DD0FB6A1B79022B07D010
:10E11000FB6A1B79032B01D1582306E0002304E09E
:10E12000222302E00F2300E00E2319461046FCF7DD
:10E13000C9F978647B6C002B0CD101221249F86A72
:10E14000FFF746FD78647B6C002B05D1002317E0B8
:10E1500000BF02E000BF00E000BFBB6A1B681846BA
:10E16000FCF723F902E000BF00E000BFB86A00F04E
:10E1700091FAF86A00F08EFA386BF7F75DF97B6C6C
:10E1800018464837BD4680BD1418002080B588B0B9
:10E1900000AF786007F1080300221A605A609A60A5
:10E1A000DA6002233B7401237B747B681B79002BAC
:10E1B00013D07B681B79012B0DD07B681B79022B58
:10E1C00007D07B681B79032B01D1654B06E0002348
:10E1D00004E0644B02E0644B00E0644B7B617B68CD
:10E1E000002B02D16FF01503B5E07B681B79FB6152
:10E1F0007B689B69BB617B68DB68002B4DD0BB698A
:10E200001A687B681B79002B13D07B681B79012B64
:10E210000DD07B681B79022B07D07B681B79032B01
:10E2200001D1582306E0002304E0222302E00F235B
:10E2300000E00E2319461046FCF766F9BB69186822
:10E240007B681B79002B13D07B681B79012B0DD0C9
:10E250007B681B79022B07D07B681B79032B01D1CC
:10E26000582306E0002304E0222302E00F2300E00D
:10E270000E2307F108021946FCF7DBF8BB691B689F
:10E280001846FCF792F87B68DB68184600F06FFBD5
:10E290007B68DB68184600F0FDF9FB69002B10D0A5
:10E2A000FB69012B0BD0FB69022B06D0FB69032B0A
:10E2B00001D12B4B06E0002304E02A4B02E02A4B5D
:10E2C00000E02A4B2A49FA6952010A441360284A9D
:10E2D000FB695B0113441C33264A1A60FB69002B5F
:10E2E00010D0FB69012B0BD0FB69022B06D0FB6918
:10E2F000032B01D11A4B06E0002304E0194B02E086
:10E30000194B00E0194B1846F7F768FC7B681B793E
:10E31000002B13D07B681B79012B0DD07B681B79F8
:10E32000022B07D07B681B79032B01D10C4B06E035
:10E33000002304E00B4B02E00B4B00E00B4B1846B4
:10E34000F7F77AF87B689B69184600F0A3F97868BC
:10E3500000F0A0F9002318462037BD4680BD00BF5D
:10E3600000140840004004400030044000200440F5
:10E370008418002079D9001080B483B000AF786091
:10E380006FF0570318460C37BD465DF8047B7047A5
:10E3900080B582B000AF78607B68002B0BD0084A54
:10E3A0007B681360074B1B689868002302220021DA
:10E3B00002F0EEFC00E000BF0837BD4680BD00BFA4
:10E3C000181800209001002080B582B000AF78605E
:10E3D0007B68002B04DB7B68022B01DC002306E05A
:10E3E00001F0B2FE0246092313604FF0FF331846D6
:10E3F0000837BD4680BD80B582B000AF78607B68CD
:10E40000002B04DB7B68022B01DC012305E001F01B
:10E410009BFE024609231360002318460837BD46B9
:10E4200080BD80B584B000AFF860B9607A6001F05B
:10E430008BFE0246092313604FF0FF331846103756
:10E44000BD4680BD80B582B000AF786039607B6822
:10E45000002B08DB7B68022B05DC3B684FF4005285
:10E460005A60002305E001F06FFE024609231360A5
:10E47000002318460837BD4680BD000080B586B031
:10E4800000AFF860B9607A60FB68002B15D1104BC3
:10E490001B687A68B9681846FCF716FA78617B69D8
:10E4A000002B08DA01F050FE02467B695B421360E4
:10E4B0004FF0FF3308E07B6906E001F045FE0246BD
:10E4C000092313604FF0FF3318461837BD4680BD4F
:10E4D0001818002080B586B000AFF860B9607A6087
:10E4E000FB68012B02D0FB68022B15D1104B1B6877
:10E4F0007A68B9681846FCF719FA78617B69002BCD
:10E5000008DA01F021FE02467B695B4213604FF09E
:10E51000FF3308E07B6906E001F016FE024609239E
:10E5200013604FF0FF3318461837BD4680BD00BF5B
:10E530001818002080B588B000AFF860B9607A6024
:10E54000BB68012B01D1012300E00223FB614FF0E6
:10E55000FF33BB61BB695B07BB61BB695B0FBB6121
:10E56000BB69B968184600F004FF0346DBB23B7490
:10E57000FB68186807F1100100230122FBF77AFEFF
:10E5800078617B69002B01D07B6920E0FB6818680B
:10E59000FB69DAB207F110010123FBF7A2FE7861F3
:10E5A0007B69002B01D07B6911E0FB69022B09D14B
:10E5B00007F11003184600F0EFFE03461A467B6889
:10E5C0001A8003E03B7C9AB27B681A8000231846CD
:10E5D0002037BD4680BD80B584B000AF786039601B
:10E5E0000421012000F048F8F860FB68002B02D1FC
:10E5F0006FF00B0313E0FB683A6811461846FBF70F
:10E600005FFDB860BB68002B04D17B68FA681A60B4
:10E61000002304E000BFF86800F03CF8BB6818462F
:10E620001037BD4680BD80B584B000AF78607B6890
:10E63000002B02D16FF015030EE07B681B681846B3
:10E64000FBF7C8FDF860FB68002B01D0FB6803E016
:10E65000786800F01FF8002318461037BD4680BDCB
:10E6600080B582B000AF7860786801F0B1FD0346F4
:10E6700018460837BD4680BD80B582B000AF7860CF
:10E6800039603968786801F027FD03461846083775
:10E69000BD4680BD80B582B000AF7860786801F07B
:10E6A0009FFD00BF0837BD4680BD80B485B000AF78
:10E6B00078600B467B807B68002B2FD00023FB818A
:10E6C00027E0FB891B02BB810023FB7211E0B7F935
:10E6D0000C30002B07DABB895B00BB81BA897B88D1
:10E6E0005340BB8102E0BB895B00BB81FB7A0133F5
:10E6F000FB72FB7A072BEAD9B7F90E305B007A6818
:10E700001344BA891A80B7F90E309BB201339BB219
:10E71000FB81B7F90E30FF2BD3DD00E000BF1437CB
:10E72000BD465DF8047B704780B487B000AFF860E9
:10E73000B9607A607B8017E07B881B0A9BB21A461F
:10E74000BB681B785340DBB27B617B695B00FA6876
:10E7500013441B881AB27B881B021BB253401BB2A6
:10E760007B80BB680133BB607B685A1E7A60002BDC
:10E77000E2D17B8818461C37BD465DF8047B7047A4
:10E7800080B485B000AF78600B46FB707B68002BCF
:10E790002DD00023FB8125E0FB897B7300233B7395
:10E7A00011E097F90D30002B07DA7B7B5B007B7360
:10E7B0007A7BFB7853407B7302E07B7B5B007B734F
:10E7C0003B7B01333B733B7B072BEAD9B7F90E3018
:10E7D0007A6813447A7B1A70B7F90E309BB2013312
:10E7E0009BB2FB81B7F90E30FF2BD5DD00E000BFF7
:10E7F0001437BD465DF8047B704780B487B000AF26
:10E80000F860B9607A60FB700DE0BB681A78FB783D
:10E810005340DBB27B61FA687B6913441B78FB7061
:10E82000BB680133BB607B685A1E7A60002BECD159
:10E83000FB7818461C37BD465DF8047B704780B5F1
:10E8400084B000AF78607B68002B02D16FF01503B5
:10E8500020E008210120FFF70FFFF860FB68002B84
:10E8600002D16FF00B0315E04FF480710120FFF728
:10E8700003FF0246FB681A60FB681B68002B05D18A
:10E88000F868FFF707FF6FF00B0303E07B68FA6897
:10E890001A60002318461037BD4680BD80B483B08F
:10E8A00000AF78607B685B7901337A6812799342B4
:10E8B0000CBF01230023DBB218460C37BD465DF8C0
:10E8C000047B704780B483B000AF78607B685A796E
:10E8D0007B681B799A420CBF01230023DBB21846E8
:10E8E0000C37BD465DF8047B704780B582B000AF41
:10E8F000786039607868FFF7E5FF0346002B02D0A7
:10E900004FF0FF330EE07B681B687A68127913447E
:10E910001A783B681A707B681B790133DAB27B681E
:10E920001A71002318460837BD4680BD80B582B0F5
:10E9300000AF78600B46FB707868FFF7AFFF0346C7
:10E94000002B02D04FF0FF330DE07B681B687A6824
:10E9500052791344FA781A707B685B790133DAB222
:10E960007B685A71002318460837BD4680BD80B5C4
:10E9700082B000AF78607B68002B08D07B681B6892
:10E98000002B04D07B681B681846FFF783FE00BF8E
:10E990000837BD4680BD80B483B000AF7860396071
:10E9A0007A683B68D31A9B1018460C37BD465DF851
:10E9B000047B704780B586B000AFF860B9607A60BC
:10E9C0000C210120FFF758FE78617B69002B01D1F3
:10E9D000002309E07B69FA681A607B69BA685A60AB
:10E9E0007B697A689A607B6918461837BD4680BD96
:10E9F00080B485B000AFF860B9607A60FB68002B26
:10EA000007D0BB68002B01D0BB6800E07B68FA68C8
:10EA10009360BB68002B05D0BB68FA685A60BB687E
:10EA20007A689A607B68002B07D0BB68002B01D006
:10EA3000BB6800E0FB687A68536000BF1437BD46CE
:10EA40005DF8047B704780B485B000AFF860B960B2
:10EA50007A60FB681B68BA689A420CD1FB687A68D6
:10EA60005A60BB68002B02D07B68002B0FD1FB687B
:10EA70007A681A600BE0FB68BA681A607B68002B42
:10EA800002D0BB68002B02D1FB68BA685A6000BF95
:10EA90001437BD465DF8047B7047000080B483B036
:10EAA00000AF78600B46FB70FB78012B11D0032B75
:10EAB0001FD17B681A4A1A607B681A4A5A607B68C1
:10EAC000194A9A607B68194ADA607B68184A1A61A9
:10EAD0001FE07B68174A1A607B68124A5A607B689D
:10EAE000114A9A607B68114ADA607B68104A1A61A1
:10EAF0000FE07B680F4A1A607B680F4A5A607B6898
:10EB00000A4A9A607B68084ADA607B680B4A1A6195
:10EB100000BF00BF0C37BD465DF8047B704700BFE7
:10EB2000F3EC0010EBEE0010DDED00102BEE00100A
:10EB300079ED001089EC00106DEF0010ABED0010C6
:10EB400080B586B000AFF8600B467A60FB72FB6858
:10EB5000002B02D14FF0FF332FE018210120FFF7E7
:10EB60008BFD78617B69002B02D14FF0FF3324E0ED
:10EB70001C210120FFF780FD38613B69002B05D186
:10EB80007869FFF787FD4FF0FF3316E0FB687A697D
:10EB90001A607B693A695A617B68002B01D07B68F7
:10EBA00000E0084B3A69D360FB7A19467869FFF7B1
:10EBB00075FF3B693A695A61002318461837BD460C
:10EBC00080BD00BF97E9001080B584B000AF7860C9
:10EBD0007B68002B02D14FF0FF331CE07B685B6940
:10EBE000FB60FB681B69002B02D04FF0FF3312E083
:10EBF00000BF07F108031946786800F076F903466C
:10EC0000002BF6D07B685B691846FFF743FD7868F8
:10EC1000FFF740FD002318461037BD4680BD80B584
:10EC200086B000AF786039607B68002B02D14FF06E
:10EC3000FF3325E07B685B697B6100233B617B6977
:10EC40001B68FB60FA6839693868FFF7B3FEB86083
:10EC5000BB68002B02D14FF0FF3311E0FA68B968AE
:10EC60003869FFF7C5FE7B695B681A46B968786941
:10EC7000FFF7E9FE7B699B685A1C7B699A60002359
:10EC800018461837BD4680BD80B586B000AF7860A5
:10EC900039607B68002B02D14FF0FF3325E07B68A1
:10ECA0005B697B617B695B683B610023FB60FA68A1
:10ECB00039693868FFF77EFEB860BB68002B02D167
:10ECC0004FF0FF3311E0FA68B9683869FFF790FE3A
:10ECD0007B691B68BA6819467869FFF7B4FE7B69DF
:10ECE0009B685A1C7B699A60002318461837BD46FA
:10ECF00080BD80B584B000AF786039607B68002B40
:10ED000002D14FF0FF3333E07B685B69BB60BB68C7
:10ED10001B68FB600CE0BB68DB68FA681268396846
:10ED2000104698470346002B06DCFB689B68FB6097
:10ED3000FB68002BEFD100E000BFFB68002B0CD17B
:10ED4000BB685A68BB689A61BB6814330122396892
:10ED5000184600F034FA03460AE0BB68FA689A6184
:10ED6000BB68143300223968184600F028FA0346BD
:10ED700018461037BD4680BD80B485B000AF7860BE
:10ED800039607B68002B02D14FF0FF3307E07B68CE
:10ED90005B69FB60FB681B683A681A6000231846D1
:10EDA0001437BD465DF8047B704780B485B000AF72
:10EDB000786039607B68002B02D14FF0FF3307E0A9
:10EDC0007B685B69FB60FB685B683A681A600023DC
:10EDD00018461437BD465DF8047B704780B485B093
:10EDE00000AF786039607B68002B02D03B68002B55
:10EDF00002D14FF0FF3312E03B6800221A607B68BB
:10EE00005B69FB60FB681B68002B02D14FF0FF338E
:10EE100005E0FB681B681A683B681A600023184607
:10EE20001437BD465DF8047B704780B485B000AFF1
:10EE3000786039607B68002B02D03B68002B02D1E0
:10EE40004FF0FF3312E03B6800221A607B685B6979
:10EE5000FB60FB685B68002B02D14FF0FF3305E0DD
:10EE6000FB685B681A683B681A6000231846143711
:10EE7000BD465DF8047B704780B586B000AFF86092
:10EE8000B9607A60FB68002B02D0BB68002B02D10E
:10EE90004FF0FF3325E0BB6800221A60FB685B6916
:10EEA0007B617B69002B02D14FF0FF3319E0FB68D7
:10EEB0005B697B617B691A687B699A617B69143342
:10EEC0007968184600F0C3F80346002B02D04FF0D3
:10EED000FF3306E07B691433B968184600F04FF938
:10EEE000034618461837BD4680BD80B586B000AFD2
:10EEF000786039607B68002B02D03B68002B02D120
:10EF00004FF0FF332EE03B6800221A607B685B699C
:10EF10007B617B699B68002B02D14FF0FF3321E0BE
:10EF20007B691B683B613B695B68FB603B699B6875
:10EF3000BB60BA680021F868FFF75AFD7B695B681F
:10EF40001A46B9687869FFF77EFD7B699B685A1E8F
:10EF50007B699A603B691A683B681A603869FFF7F9
:10EF600099FB002318461837BD4680BD80B586B092
:10EF700000AF786039607B68002B02D03B68002BC3
:10EF800002D14FF0FF332EE03B6800221A607B680D
:10EF90005B697B617B699B68002B02D14FF0FF337B
:10EFA00021E07B695B683B613B695B68FB603B69B7
:10EFB0009B68BB60BA680021F868FFF719FD7B69A0
:10EFC0001B68FA6819467869FFF73DFD7B699B6805
:10EFD0005A1E7B699A603B691A683B681A603869F7
:10EFE000FFF758FB002318461837BD4680BD80B593
:10EFF00086B000AFF860B9607A60FB68002B02D081
:10F00000BB68002B02D14FF0FF331CE0BB6800222D
:10F010001A60FB685B697B617B691A687B699A612E
:10F020007B6914337968184600F011F80346002B09
:10F0300002D04FF0FF3306E07B691433B9681846FD
:10F0400000F033F8034618461837BD4680BD80B53A
:10F0500084B000AF786039607B68BB60BB68002B10
:10F0600002D14FF0FF331CE0BB681B681B68FB60DC
:10F0700012E0BB681B68DB68FA68126839681046E2
:10F0800098470346002B04D1BB68FA685A600023F6
:10F0900007E0FB689B68FB60FB68002BE9D14FF041
:10F0A000FF3318461037BD4680BD80B584B000AF31
:10F0B000786039607B68BB60BB68002B06D0BB689A
:10F0C0005B68002B02D03B68002B02D14FF0FF336E
:10F0D00051E0BB685B685868BB685B689B681A4610
:10F0E0000021FFF785FCBB685A68BB681B681B687A
:10F0F0009A420BD1BB681868BB685B689968BB68AB
:10F100001B685B681A46FFF79EFC11E0BB685A68F3
:10F11000BB681B685B689A420AD1BB681868BB6809
:10F120001B681968BB685B685B681A46FFF78BFC55
:10F13000BB681B689A68013A9A60BB685B681A688A
:10F140003B681A60BB685A68BB681B685B689A4278
:10F1500004D1BB685B685B68FB6003E0BB685B680D
:10F160009B68FB60BB685B681846FFF793FABB6857
:10F17000FA685A60002318461037BD4680BD80B437
:10F1800085B000AF786039607B68FB60FB68002B5E
:10F1900006D0FB685B68002B02D03B68002B02D1D5
:10F1A0004FF0FF3305E0FB685B681A683B681A6044
:10F1B000002318461437BD465DF8047B704780B5C0
:10F1C0008CB000AFF860B9601346FB71FB68BB629E
:10F1D000BB6A002B02D14FF0FF3355E0FB681B6880
:10F1E0007B62FB79002B0ED0BB6A5A68BB6A1B6836
:10F1F0005B689A4207D107F11003B9681846FFF718
:10F2000043FD034640E0FB7983F00103DBB2002BB2
:10F210000ED0BB6A5A68BB6A1B681B689A4207D14A
:10F2200007F11003B9681846FFF7F9FC03462BE015
:10F23000FB79002B0AD0BB6A5968BB6A5B689B6884
:10F240001A46B868FFF7B6FBF86209E0BB6A5B686C
:10F250005968BB6A5B681A46B868FFF7ABFBF8628F
:10F26000FB6A002B02D14FF0FF330DE0FB6A5868B8
:10F27000FB6A9B681A46F96AFFF7BAFBBB6A1B6810
:10F280009A6801329A60002318463037BD4680BD27
:10F2900080B483B000AF786000BF0C37BD465DF826
:10F2A000047B704780B483B000AF786000BF0C3738
:10F2B000BD465DF8047B704780B483B000AF7860D2
:10F2C00000BF0C37BD465DF8047B704780B483B047
:10F2D00000AF786000BF0C37BD465DF8047B704717
:10F2E00080B483B000AF786039607B68002B00DAAF
:10F2F0001F335B119B003A6813441A687B6842FA1B
:10F3000003F303F0010318460C37BD465DF8047B98
:10F31000704780B485B000AF78600023FB600CE0DC
:10F320007B6803F00103002B01D0FB6809E07B68D8
:10F330005B087B60FB680133FB607B68002BEFD1CF
:10F34000202318461437BD465DF8047B704780B50E
:10F3500082B000AF786039607868FFF7DAFF024664
:10F360003B6803FA02F27B68134018460837BD4633
:10F3700080BD90B583B000AF786039603A687B6833
:10F3800002EA03047868FFF7C4FF034624FA03F394
:10F3900018460C37BD4690BD80B483B000AF78608E
:10F3A0007B6801331B781AB27B681B781B021BB287
:10F3B00013431BB29BB218460C37BD465DF8047B65
:10F3C000704780B483B000AF78607B681B781AB256
:10F3D0007B6801331B781B021BB213431BB29BB229
:10F3E00018460C37BD465DF8047B704780B483B087
:10F3F00000AF78607B681B781A467B6801331B7806
:10F400001B0213431A467B6802331B781B04134309
:10F4100018460C37BD465DF8047B704780B485B054
:10F4200000AF786039603B68DBB2C3F11F03FB7348
:10F43000FB7B7A6802FA03F31A46FB7B42FA03F37A
:10F4400018461437BD465DF8047B7047454885462D
:10F450004548804780B94549454A464B9B1A03DDDC
:10F46000043BC858D050FBDC4349444A0020914239
:10F47000BCBF41F8040BFAE7414880474148804748
:10F4800041488047FFF7FEFFFEE7FEE7FEE7FEE7A5
:10F49000FEE7FEE7FEE7FEE7FEE7FEE7FEE7FEE744
:10F4A000FEE7FEE7FEE7FEE7FEE7FEE7FEE7FEE734
:10F4B000FEE7FEE7FEE7FEE7FEE7FEE7FEE7FEE724
:10F4C000FEE7FEE7FEE7FEE7FEE7FEE7FEE7FEE714
:10F4D000FEE7FEE7FEE7FEE7FEE7FEE7FEE7FEE704
:10F4E000FEE7FEE7FEE7FEE7FEE7FEE7FEE7FEE7F4
:10F4F000FEE7FEE7FEE7FEE7FEE7FEE7FEE7FEE7E4
:10F50000FEE7FEE7FEE7FEE7FEE7FEE7FEE7FEE7D3
:10F51000FEE7FEE7FEE7FEE7FEE7FEE7FEE7FEE7C3
:10F52000FEE7FEE7FEE7FEE7FEE7FEE7FEE7FEE7B3
:10F53000FEE7FEE7FEE7FEE7FEE7FEE7FEE7FEE7A3
:10F54000FEE7FEE7FEE7FEE7FEE7FEE7FEE7FEE793
:10F55000FEE7FEE7FEE7FEE7FEE7FEE7FEE7FEE783
:10F56000FEE7FEE7000002207D030010E8750110B1
:10F5700000000020480B0020000C0020081900208B
:10F5800001040010890101108D70001081F000410C
:10F5900002E000BF83F0004330B54FEA41044FEA78
:10F5A000430594EA050F08BF90EA020F1FBF54EA13
:10F5B000000C55EA020C7FEA645C7FEA655C00F0AF
:10F5C000E2804FEA5454D4EB5555B8BF6D420CDD80
:10F5D0002C4480EA020281EA030382EA000083EA03
:10F5E000010180EA020281EA0303362D88BF30BDA3
:10F5F00011F0004F4FEA01314FF4801C4CEA1131F9
:10F6000002D0404261EB410113F0004F4FEA033357
:10F610004CEA133302D0524263EB430394EA050FE2
:10F6200000F0A780A4F10104D5F1200E0DDB02FA51
:10F630000EFC22FA05F2801841F1000103FA0EF2E5
:10F64000801843FA05F359410EE0A5F120050EF1AB
:10F65000200E012A03FA0EFC28BF4CF0020C43FADC
:10F6600005F3C01851EBE37101F0004507D54FF0E9
:10F67000000EDCF1000C7EEB00006EEB0101B1F539
:10F68000801F1BD3B1F5001F0CD349085FEA30007F
:10F690004FEA3C0C04F101044FEA445212F5800F8A
:10F6A00080F09A80BCF1004F08BF5FEA500C50F127
:10F6B000000041EB045141EA050130BD5FEA4C0C0A
:10F6C000404141EB010111F4801FA4F10104E9D193
:10F6D00091F0000F04BF01460020B1FA81F308BF8A
:10F6E0002033A3F10B03B3F120020CDA0C3208DD56
:10F6F00002F1140CC2F10C0201FA0CF021FA02F131
:10F700000CE002F11402D8BFC2F1200C01FA02F1A0
:10F7100020FA0CFCDCBF41EA0C019040E41AA2BFC5
:10F7200001EB0451294330BD6FEA04041F3C1CDA8D
:10F730000C340EDC04F11404C4F1200220FA04F0AD
:10F7400001FA02F340EA030021FA04F345EA030157
:10F7500030BDC4F10C04C4F1200220FA02F001FA19
:10F7600004F340EA0300294630BD21FA04F029469B
:10F7700030BD94F0000F83F4801306BF81F4801134
:10F780000134013D4EE77FEA645C18BF7FEA655CA7
:10F7900029D094EA050F08BF90EA020F05D054EA79
:10F7A000000C04BF1946104630BD91EA030F1EBF7E
:10F7B0000021002030BD5FEA545C05D14000494182
:10F7C00028BF41F0004130BD14F580043CBF01F575
:10F7D000801130BD01F0004545F0FE4141F470015B
:10F7E0004FF0000030BD7FEA645C1ABF1946104636
:10F7F0007FEA655C1CBF0B46024650EA013406BF37
:10F8000052EA033591EA030F41F4002130BD00BFF5
:10F8100090F0000F04BF0021704730B54FF48064B2
:10F8200004F132044FF000054FF0000150E700BF33
:10F8300090F0000F04BF0021704730B54FF4806492
:10F8400004F1320410F0004548BF40424FF000017F
:10F850003EE700BF42004FEAE2014FEA31014FEAC2
:10F8600002701FBF12F07F4393F07F4F81F0605111
:10F87000704732F07F4208BF704793F07F4F04BF5C
:10F8800041F40021704730B54FF4607401F0004539
:10F8900021F000411CE700BF50EA010208BF704799
:10F8A00030B54FF000050AE050EA010208BF70478A
:10F8B00030B511F0004502D5404261EB41014FF4F3
:10F8C000806404F132045FEA915C3FF4D8AE4FF0FB
:10F8D00003025FEADC0C18BF03325FEADC0C18BFDE
:10F8E000033202EBDC02C2F1200300FA03FC20FA2F
:10F8F00002F001FA03FE40EA0E0021FA02F114447C
:10F90000BDE600BF70B54FF0FF0C4CF4E06C1CEA94
:10F9100011541DBF1CEA135594EA0C0F95EA0C0F05
:10F9200000F0DEF82C4481EA030621EA4C5123EA78
:10F930004C5350EA013518BF52EA033541F48011A7
:10F9400043F4801338D0A0FB02CE4FF00005E1FB5A
:10F9500002E506F00042E0FB03E54FF00006E1FBA4
:10F9600003569CF0000F18BF4EF0010EA4F1FF04E7
:10F97000B6F5007F64F5407404D25FEA4E0E6D4127
:10F9800046EB060642EAC62141EA55514FEAC52038
:10F9900040EA5E504FEACE2EB4F1FD0C88BFBCF5B4
:10F9A000E06F1ED8BEF1004F08BF5FEA500E50F165
:10F9B000000041EB045170BD06F0004646EA01012B
:10F9C00040EA020081EA0301B4EB5C04C2BFD4EB5D
:10F9D0000C0541EA045170BD41F480114FF0000E56
:10F9E000013C00F3AB8014F1360FDEBF002001F0C4
:10F9F000004170BDC4F10004203C35DA0C341BDC3E
:10FA000004F11404C4F1200500FA05F320FA04F00F
:10FA100001FA05F240EA020001F0004221F0004143
:10FA200010EBD37021FA04F642EB06015EEA430EB6
:10FA300008BF20EAD37070BDC4F10C04C4F12005E6
:10FA400000FA04F320FA05F001FA04F240EA020099
:10FA500001F0004110EBD37041F100015EEA430E6A
:10FA600008BF20EAD37070BDC4F1200500FA05F28A
:10FA70004EEA020E20FA04F301FA05F243EA020309
:10FA800021FA04F001F0004121FA04F220EA020018
:10FA900000EBD3705EEA430E08BF20EAD37070BD5E
:10FAA00094F0000F0FD101F00046400041EB01013E
:10FAB00011F4801F08BF013CF7D041EA060195F020
:10FAC000000F18BF704703F00046520043EB0303DA
:10FAD00013F4801F08BF013DF7D043EA06037047C7
:10FAE00094EA0C0F0CEA135518BF95EA0C0F0CD0D2
:10FAF00050EA410618BF52EA4306D1D181EA030118
:10FB000001F000414FF0000070BD50EA410606BF11
:10FB10001046194652EA430619D094EA0C0F02D156
:10FB200050EA013613D195EA0C0F05D152EA03369B
:10FB30001CBF104619460AD181EA030101F00041B9
:10FB400041F0FE4141F470014FF0000070BD41F002
:10FB5000FE4141F4780170BD70B54FF0FF0C4CF4DC
:10FB6000E06C1CEA11541DBF1CEA135594EA0C0FFB
:10FB700095EA0C0F00F0A7F8A4EB050481EA030E48
:10FB800052EA03354FEA013100F088804FEA03332F
:10FB90004FF0805545EA131343EA12634FEA0222FD
:10FBA00045EA111545EA10654FEA00260EF00041BE
:10FBB0009D4208BF964244F1FD0404F5407402D210
:10FBC0005B084FEA3202B61A65EB03055B084FEAA1
:10FBD00032024FF480104FF4002CB6EB020E75EB9E
:10FBE000030E22BFB61A754640EA0C005B084FEAC6
:10FBF0003202B6EB020E75EB030E22BFB61A754643
:10FC000040EA5C005B084FEA3202B6EB020E75EB8D
:10FC1000030E22BFB61A754640EA9C005B084FEA05
:10FC20003202B6EB020E75EB030E22BFB61A754612
:10FC300040EADC0055EA060E18D04FEA051545EA01
:10FC400016754FEA06164FEAC30343EA52734FEAAA
:10FC5000C2025FEA1C1CC0D111F4801F0BD141EA23
:10FC600000014FF000004FF0004CB6E711F4801F88
:10FC700004BF01430020B4F1FD0C88BFBCF5E06F68
:10FC80003FF6AFAEB5EB030C04BFB6EB020C5FEA78
:10FC9000500C50F1000041EB045170BD0EF0004ECD
:10FCA0004EEA113114EB5C04C2BFD4EB0C0541EAFF
:10FCB000045170BD41F480114FF0000E013C90E6FC
:10FCC00045EA060E8DE60CEA135594EA0C0F08BFC0
:10FCD00095EA0C0F3FF43BAF94EA0C0F0AD150EABF
:10FCE00001347FF434AF95EA0C0F7FF425AF104652
:10FCF00019462CE795EA0C0F06D152EA03353FF47A
:10FD0000FDAE1046194622E750EA410618BF52EAF6
:10FD100043067FF4C5AE50EA41047FF40DAF52EACA
:10FD200043057FF4EBAE12E77BB972B90029BEBF81
:10FD300000204FF0004106E008BF00281CBF6FF014
:10FD400000414FF0FF3000F0BFB9ADF1080C6DE994
:10FD500004CE002909DB002B1ADB00F04DF8DDF89A
:10FD600004E0DDE9022304B07047404261EB410149
:10FD7000002B1BDB00F040F8DDF804E0DDE9022396
:10FD800004B0404261EB4101524263EB43037047D0
:10FD9000524263EB430300F02FF8DDF804E0DDE9A5
:10FDA000022304B0404261EB41017047524263EBD1
:10FDB000430300F021F8DDF804E0DDE9022304B09C
:10FDC000524263EB4303704753B94AB9002908BF55
:10FDD00000281CBF4FF0FF314FF0FF3000F074B926
:10FDE000ADF1080C6DE904CE00F006F8DDF804E092
:10FDF000DDE9022304B070472DE9F047089E044670
:10FE00008846002B40F085808A42154648D9B2FAD0
:10FE100082F24AB1C2F1200701FA02F320FA07F791
:10FE2000954047EA030894404FEA154E230CB8FB6F
:10FE3000FEF71FFA85FC0EFB178843EA084307FB11
:10FE40000CF1994209D9EB1807F1FF3080F0E380FB
:10FE5000994240F2E080023F2B445B1AA4B2B3FB0C
:10FE6000FEF00EFB103344EA034400FB0CFCA445F7
:10FE700009D92C1900F1FF3380F0CB80A44540F262
:10FE8000C88002382C4440EA0740A4EB0C04002749
:10FE90001EB1D4400023C6E900433946BDE8F087CF
:10FEA000002A53D0B2FA82F2002A40F0B680491BF1
:10FEB0004FEA154E1FFA85F80127B1FBFEFC230C13
:10FEC0000EFB1C1143EA014308FB0CF1994207D9D0
:10FED000EB180CF1FF3002D2994200F2EC8084461C
:10FEE000591AA3B2B1FBFEF00EFB101443EA04440E
:10FEF00008FB00F8A04507D92C1900F1FF3302D206
:10FF0000A04500F2DC801846A4EB080440EA0C404F
:10FF1000BEE78B4208D9002E78D00027C6E9000141
:10FF200038463946BDE8F087B3FA83F77FB98B428C
:10FF300002D3824200F2BD80841A61EB03030120E8
:10FF40009846002EA9D0C6E90048A6E7FFDEC7F113
:10FF50002005BB4022FA05FC4CEA030C01FA07F429
:10FF600020FA05F821FA05F34FEA1C4E48EA04048A
:10FF7000B3FBFEF9210C0EFB19331FFA8CF841EA92
:10FF8000034309FB08FA9A4502FA07F200FA07F15F
:10FF90000BD91CEB030309F1FF3080F088809A45F0
:10FFA00040F28580A9F102096344A3EB0A03A4B2DD
:10FFB000B3FBFEF00EFB103344EA034400FB08F8E9
:10FFC000A04508D91CEB040400F1FF336BD2A04517
:10FFD00069D90238644440EA0940A4EB0804A0FB54
:10FFE00002894C45C6464B4654D351D0002E69D0A9
:10FFF000B1EB0E0264EB030404FA05F522FA07F3F1
:020000041001E9
:10000000FC401D43C6E90054002746E7374630460A
:1000100043E7184637E707461FE7C2F1200320FAF7
:1000200003F7954001FA02F021FA03F34FEA154E67
:100030003843010CB3FBFEF71FFA85F80EFB1733AC
:1000400041EA034107FB08F38B4204FA02F407D9A3
:10005000691807F1FF3C28D28B4226D9023F294478
:10006000CB1A81B2B3FBFEF00EFB103341EA034121
:1000700000FB08F38B4207D9691800F1FF3C10D24E
:100080008B420ED902382944C91A40EA074714E7BF
:100090004145ABD2B8EB020E69EB0C0201381346B6
:1000A000A4E76046F0E7184695E76746D8E781463B
:1000B0007BE7384645E7ACF1020C2B4410E70238E9
:1000C0002C4421E73746E8E6704700BF002301468D
:1000D0001A46184602F0ACBA024B0A4601461868A6
:1000E00000F002B89001002010B502FB01F100F011
:1000F0007FF8044668B150F8042C22F00302043A59
:10010000242A18D8132A06D802460023C2E900334D
:100110009360204610BD00231B2AC0E900330FD98D
:10012000242AC0E9023312BF00F11002C0E90433EF
:1001300000F11802E9E7002100F0A6FB204610BDFF
:1001400000F10802E1E700BF014B1868704700BFEB
:100150009001002038B50A4C0A4D641BA4100AD047
:1001600004F18043013B05EB8305013C55F804395C
:100170009847002CF9D1BDE8384007F029BA00BFF4
:10018000480B0020440B002070B50D4E0D4D761B22
:10019000B61006D00024013455F8043B9847A64217
:1001A000F9D1094E094D761B07F00CFAB61006D0AE
:1001B0000024013455F8043B9847A642F9D170BD9C
:1001C0003C0B00203C0B0020440B00203C0B00208B
:1001D000024B0146186800F00BB800BF90010020E8
:1001E000024B0146186803F05FBC00BF900100207D
:1001F0002DE9F04F01F10B05162D83B0064623D8EB
:10020000102900F2B98000F08FFB1025182302207E
:10021000CD4F3B44A3F108025C68944200F0B980E2
:10022000636823F003032344D4E902515A68E96068
:1002300042F0010230468D605A6000F077FB0834CE
:10024000204603B0BDE8F08F35F0070500F194803B
:10025000A94200F2918000F067FBB5F5FC7FC0F089
:100260009D816B0A00F08F80042B00F27381AB0933
:1002700003F1390003F1380CC300B34F3B44A3F141
:1002800008015C68A14206D10CE0002A80F22B81B3
:10029000E468A14206D0636823F003035A1B0F2AC7
:1002A000F3DD60463C69DFF8A4C264457CD0636836
:1002B00023F003035A1B0F2A00F37E81002AC7E9AB
:1002C00004CC80F26F81B3F5007F80F01A81DB08E7
:1002D000591C7A6857F83180C4F808804FF0010E35
:1002E0009B100EFA03F307EBC10E1343AEF10802A5
:1002F000E2607B6047F83140C8F80C40821001246E
:1003000094409C4256D81C4206D120F00300640061
:100310001C4200F10400FAD007EBC009CE4680462B
:10032000DEF80C309E4507D120E1002A80F22781BB
:10033000DB689E4500F01A81596821F003014A1BD1
:100340000F2AF2DDD3E9028E5C1945F001055D60EC
:1003500042F00105C8F80CE03046CEF80880C7E945
:100360000444C4E902CC65605A50009300F0DEFA00
:10037000009B03F1080402E00C23336000242046B4
:1003800003B0BDE8F08F4FF4007340204FF03F0CF6
:1003900073E7DC68A34208BF02307FF441AF3C69D9
:1003A000DFF8A8C1644582D17B68821001249440A3
:1003B0009C42A8D9BC68636823F00308A84503D30E
:1003C000A8EB05030F2B7EDCDFF88491D7F8082417
:1003D000D9F80030013204EB080A2B4400F03781D1
:1003E00003F580530F3323F47F6B2BF00F0B59462B
:1003F000304600F0BBFC411C024600F0F78082450D
:1004000000F2F280D9F804105944C9F804100B46E0
:1004100000F05381D7F8081401311BBFA2EB0A0A80
:100420005344C7F80824C9F8043012F0070300F059
:100430001A81C3F108010A44C3F58051934408317D
:10044000A1EB0B01C1F30B0A514630460193009218
:1004500000F08CFC421CDDE9002300F05381831A7C
:1004600003EB0A0BD9F80410BA604BF001035144B6
:10047000BC425360C9F8041000F02B81B8F10F0F93
:1004800040F229816368A8F10C0020F0070003F016
:10049000010304EB000C03434FF0050E0F286360CB
:1004A000CCE901EE00F2358153681446D9F82C20CE
:1004B0008A42D9F8302038BFC9F82C108A4238BF98
:1004C000C9F8301094E0621943F0010345F00105CA
:1004D00065603046BA60536000F028FA0834204660
:1004E00003B0BDE8F08F2344E1685A68A56842F084
:1004F0000102E96030468D605A6000F017FA083456
:100500003DE75A0A042A69D9142A00F2BE8002F192
:100510005C01C9005B3207EB010E7958AEF1080EA1
:100520008E4500F097804A6822F003029A4202D971
:1005300089688E45F7D1D1F80CE07B68C4E9021ECA
:10054000CEF80840CC60D9E6C0050020C8050020E0
:100550001C180020142B59D9542B00F29E802B0B11
:1005600003F16F0003F16E0CC30086E608F1010889
:1005700018F0030F0EF1080E7FF4D2AE51E01944CB
:100580001C464A68DB6854F8085F42F001024A6082
:100590003046EB609D6000F0C9F9F0E6E80805F12F
:1005A000080335E6234430465A6842F001025A6097
:1005B000083400F0BBF9E2E6611945F0010E42F0A3
:1005C0000105C4F804E03046C7E90411C1E902CCD2
:1005D0004D60E25000F0AAF90834D0E69A0902F121
:1005E0003901C900383296E7BC4260D0BC68636804
:1005F00023F0030BAB45ABEB050302D30F2B3FF707
:1006000062AF304600F092F90024B8E603F15C00D6
:1006100003F15B0CC30030E659F808394B4540F054
:10062000968010F0030F00F1FF30F5D17B6823EACC
:1006300004037B6064009C423FF6BCAE1CB9B9E683
:10064000640008F104081C42FAD0404664E603F155
:10065000100BCCE67B6892104FF0010808FA02F20A
:1006600013437B606AE702EB0B014942C1F30B0ABB
:10067000514630460193009200F078FB431CDDE9BF
:1006800000237FF4ECAE9A46ECE6542A26D81A0BE7
:1006900002F16F01C9006E323DE7B3F5AA7F26D89B
:1006A000EB0B03F1780003F1770CC300E5E5D9F813
:1006B00004305B44C9F80430ACE6CAF30B000028F0
:1006C0007FF4A8AE08EB0B03BC6843F00103636042
:1006D000ECE61446EAE60123536092E7B2F5AA7FFE
:1006E00021D8DA0B02F17801C900773213E740F222
:1006F0005452934221D8AB0C03F17D0003F17C0CE2
:10070000C300BAE5083B9B44ABEB020B4FF0000A79
:10071000A8E604F10801304603F0C6F9BC68D9F830
:1007200004106368C2E640F254518A420BD89A0C16
:1007300002F17D01C9007C32EDE64FF47E737F202B
:100740004FF07E0C99E54FF47E717E22E3E67B68E4
:1007500070E700BF844641EA000313F003036DD144
:10076000403A41D351F8043B40F8043B51F8043B74
:1007700040F8043B51F8043B40F8043B51F8043B7B
:1007800040F8043B51F8043B40F8043B51F8043B6B
:1007900040F8043B51F8043B40F8043B51F8043B5B
:1007A00040F8043B51F8043B40F8043B51F8043B4B
:1007B00040F8043B51F8043B40F8043B51F8043B3B
:1007C00040F8043B51F8043B40F8043B51F8043B2B
:1007D00040F8043B51F8043B40F8043B51F8043B1B
:1007E00040F8043B403ABDD2303211D351F8043BBB
:1007F00040F8043B51F8043B40F8043B51F8043BFB
:1008000040F8043B51F8043B40F8043B103AEDD269
:100810000C3205D351F8043B40F8043B043AF9D2BA
:10082000043208D0D2071CBF11F8013B00F8013B8D
:1008300001D30B8803806046704700BF082A13D39A
:100840008B078DD010F003038AD0C3F10403D21AB2
:10085000DB071CBF11F8013B00F8013B80D331F8E6
:10086000023B20F8023B7BE7043AD9D3013A11F866
:10087000013B00F8013BF9D20B7803704B784370D1
:100880008B78837060467047F0B4860746D0541E5C
:10089000002A3CD0CAB2034602E014F1FF3436D33A
:1008A00003F8012B9D07F8D1032C29D9CDB245EAD5
:1008B00005250F2C45EA054533D9A4F11006360964
:1008C00003F1200707EB061703F1100242E9045574
:1008D00042E902551032BA42F8D1721C14F00C0FE2
:1008E00003EB021204F00F0613D0331F23F00303AF
:1008F0000433134442F8045B9342FBD106F0030433
:100900002CB1C9B21C4403F8011B9C42FBD1F0BCC2
:10091000704734461346002CF3D1F8E714460346DB
:10092000C2E71A462646E0E7704700BF704700BF9F
:100930000EB400B582B003AB816853F8042B019369
:1009400000F04EFB02B05DF804EB03B0704700BF4F
:100950000FB400B5074983B004AB086853F8042B03
:100960008168019300F03CFB03B05DF804EB04B038
:10097000704700BF9001002070B5054688B008465A
:100980000C4600F0BDFA154AAB6B04940126441CDA
:1009900004A90692022203940590AC680796CDE95B
:1009A0000112B3B1B4F90C309A0406D4626E43F468
:1009B000005322F40052A38162662146284601AA10
:1009C00003F06CF9002814BF4FF0FF300A2008B084
:1009D00070BD284602F0F8FFE4E700BF3472011052
:1009E000024B01461868FFF7C7BF00BF9001002007
:1009F000024B0A460146186800F002B89001002038
:100A00002DE9F84F1746002900F0BB8007F10B04D1
:100A100081460D46FFF788FF162C5ED8102422462B
:100A2000A7425FD855F804EC2EF00306A5F108089C
:100A3000964208EB060A80F28180CB4BDAF804007C
:100A40009968514500F0B58020F0010353445B687C
:100A5000DB0700F18A8020F003003318934280F214
:100A600012811EF0010F0FD155F8083CA8EB030BC3
:100A7000DBF8041021F0030108448319934280F24B
:100A800016817318934234DA39464846FFF7B0FBB3
:100A90000746E0B155F8043C23F001034344A0F1BC
:100AA0000802934200F0F780321F242A00F2FB80F4
:100AB000132A296800F2C98003462A461960516842
:100AC000596092689A602946484602F0EDFF484610
:100AD000FFF72CFF3846BDE8F88F24F00704002C00
:100AE00022469DDA0C23C9F8003000273846BDE8BD
:100AF000F88F5F46DBF80C1057F8080F321F242AD6
:100B0000C1600BEB030A886000F2D980132A2968C0
:100B100040F2D380CBF808106968CBF80C101B2A80
:100B2000A96800F2E0800BF11002083511606968D5
:100B30005160A96891601E46D8463D46D8F80430F9
:100B4000321B0F2A03F0010320D83343C8F80430C6
:100B5000DAF8043043F00103CAF8043048462F465F
:100B6000FFF7E4FE3846BDE8F88F1EF0010F8BD189
:100B700055F8083CA8EB030BDBF8041021F0030147
:100B80007FE71146BDE8F84FFFF732BB08EB0401E1
:100B9000234342F00102C8F804304A60DAF8043016
:100BA00043F001030831CAF80430484602F07CFFE4
:100BB000D4E720F00300311804F1100C61454FDA3E
:100BC0001EF0010F7FF460AF55F8081CA8EB010B75
:100BD000DBF8041021F00301084400EB060AD445B9
:100BE0003FF74FAF5F46DBF80C1057F8080F321F86
:100BF000242AC160886000F29980132A296840F293
:100C00009380CBF808106968CBF80C101B2AA968F0
:100C100000F292800BF11002083511606968516092
:100C2000A96891600BEB0401AAEB040242F00102F7
:100C300099604A60DBF8043003F001031C43484626
:100C4000CBF80440FFF772FE50E701606B68436029
:100C50001B2A3CD805F1080200F10803A9682DE71A
:100C600008EB04000A1B42F001029860426055F84C
:100C7000043C03F001031C43484645F8044CFFF7CD
:100C800055FE2F4632E7DAE902121E46CA6008EB2B
:100C9000030A916052E750F8043C23F003031E441A
:100CA00008EB060A4AE7294603F0A2FA0BE7DAE95D
:100CB00002125F46CA6091601CE73A4636E7294651
:100CC00038461E46D84603F093FA3D4636E7AB68F1
:100CD0008360EB68C360242A11D005F1100200F193
:100CE00010032969EAE6CBF81010E968CBF8141074
:100CF000242A0ED029690BF11802103516E72B694A
:100D000003616B694361A96905F1180200F11803D9
:100D1000D4E62A69CBF818206A69CBF81C20A969A7
:100D20000BF12002183501E73A4676E729463846A6
:100D300003F05EFA0C4B75E7CBF81010E968CBF8BE
:100D40001410242A04D029690BF11802103564E725
:100D50002A69CBF818206A69CBF81C20A9690BF125
:100D60002002183559E700BFC005002038B5074CF0
:100D70000023054608462360EFF76EFA431C00D0B7
:100D800038BD2368002BFBD02B6038BD0419002030
:100D90002DE9F043524C256883B004460F46904637
:100DA0001E4615B1AB6B002B65D0B8F1020F06D013
:100DB000B8F1010F00F29180002EC0F28E80214622
:100DC000284602F0FBFC216B41B104F1400399423B
:100DD00002D0284602F068FE00232363B4F90C30E9
:100DE0000022A26162601A064DD423F44A6323F004
:100DF0000303B8F1020FA3814CD001AB6A46214630
:100E0000284603F029F9A3891843A08116B317B324
:100E1000AB6B63B3009BB4F90C002760B3421CBFFB
:100E200040F40060A081B8F1010F08BF40F001005C
:100E300083B208BFA08113F00800C4E904761ED075
:100E400013F0010035D000207642A661A06003B007
:100E5000BDE8F083009E3046FFF7BAF9074660B35D
:100E6000A38943F08003A381AB6B002BD2D128462A
:100E700002F0AAFDCEE7284602F0A6FD95E7A060A5
:100E800003B0BDE8F0832169284602F00DFEB4F9F5
:100E90000C30AAE7002004F1430243F002030025CE
:100EA0000121A381A5602260C4E9042103B0BDE84B
:100EB000F083A66003B0BDE8F083DDF80090B14593
:100EC00006D04846FFF784F9074608B14E46C7E703
:100ED000B4F90C304FF0FF30DDE74FF0FF30CFE7D3
:100EE0009001002000000000000000000000000051
:100EF00000000000000000000000000000000000F2
:100F000090F800F06DE9024520F007016FF0000C49
:100F100010F0070491F820F040F049804FF00004F1
:100F20006FF00700D1E9002391F840F000F10800CC
:100F300082FA4CF2A4FA8CF283FA4CF3A2FA8CF304
:100F40004BBBD1E9022382FA4CF200F10800A4FA6B
:100F50008CF283FA4CF3A2FA8CF3E3B9D1E90423BF
:100F600082FA4CF200F10800A4FA8CF283FA4CF3F6
:100F7000A2FA8CF37BB9D1E9062301F1200182FAB0
:100F80004CF200F10800A4FA8CF283FA4CF3A2FAB6
:100F90008CF3002BC6D0002A04BF04301A4612BAC4
:100FA000B2FA82F2FDE8024500EBD2007047D1E9C7
:100FB000002304F00305C4F100004FEAC50514F056
:100FC000040F91F840F00CFA05F562EA05021CBF27
:100FD00063EA050362464FF00004A9E70000000041
:100FE0002DE9F04FBFB01C4604919146054608908C
:100FF00003F02AF8036811931846FFF781FF09945C
:101000000F901DB1AB6B002B00F067830499B1F911
:101010000C2093B29E04084607D4496E42F4005354
:1010200021F40051838141669BB21D0740F1D080BD
:10103000049A1269002A00F0CB8003F01A030A2BED
:1010400000F0D4809FED9A7B00238DED0C7B0E93F6
:10105000CDE922331093129305932EAB21939A4638
:1010600099F80030002B00F0DD80252B00F0BE86C3
:101070004D4603E0252B00F0C78025466B786C1C9D
:10108000002BF7D1B4EB090600F0CC80DDE9223269
:1010900001333244072BCAF80090CAF80460CDE946
:1010A000223200F3B6800AF1080A059A6B783244BE
:1010B0000592002B00F0B680002367788DF867302A
:1010C0001A46194606939B4604F101094FF0FF3674
:1010D00009F10109A7F12003582B00F20283DFE890
:1010E00013F0DA0200030003E2020003000300032E
:1010F0000003000300032902BC020003B702C1027F
:101100000003C000B100B100B100B100B100B100F6
:10111000B100B100B10000030003000300030003AD
:10112000000300030003000300039D0251020003BB
:10113000510200030003000300034C0200030003FC
:1011400068000003000300030003000359000003CC
:101150000003340200030003000300030003000344
:101160000003000300030003AE01740151025102A9
:1011700051026F01740100030003620100034C017E
:101180006A001C0117010003ED0000035B0000036F
:101190000003C5004BF0100B1BF0200F00F09282F3
:1011A000099C073424F00703F3E80245099301235F
:1011B000C3E04BF0100B1BF0200300F07982099C78
:1011C000073424F00703F3E8024509930023B4E051
:1011D0000499089801F0C4F9002841F01381049B98
:1011E0009B8903F01A030A2B7FF42CAF049BB3F9FD
:1011F0000E30002BFFF626AF23464A460499089886
:1012000001F078F9059019E0B4EB09063FF454AF0A
:101210003CE721AA0499089803F0AAFD48B90DF10A
:10122000B80A42E7239B23B10898049921AA03F046
:101230009FFD049B9B895A0601F1E48005983FB00D
:10124000BDE8F08FA7F13003002019F8017B00EB17
:10125000800003EB4000A7F13003092BF5D906907D
:1012600038E74BF0800B99F8007031E7002A41F025
:10127000B180114B10931BF0200F00F06F81099C7F
:10128000073424F00703F3E8024509931BF0010F2C
:1012900000F0388254EA050300F0348230238DF8E0
:1012A00068308DF869704BF0020B022345E000BFF7
:1012B00000000000000000007C720110099C54F83E
:1012C000043B0A9300258DF86750002B00F07F86C1
:1012D000711C00F05387324629460A9802F038FF05
:1012E000002801F059800A9BC31A07932E4623EA6F
:1012F000E3739DF867800994CDF808B003930B96CB
:10130000B8F1000F00F0AD80039B01330393A8E018
:101310004BF0200B99F80070DAE6099C54F8043B76
:10132000099447F630021C46B74B1093ADF868207D
:101330004BF0020B0025022378274FF000088DF8B0
:101340006780721C00F0E2812BF08002029254EA66
:10135000050240F0D981002E40F01284002B40F0AD
:10136000DC841BF00103079300F0498530238DF8DE
:10137000B7300DF1B7030A9359E0002A41F03280EB
:10138000099A1BF0200F52F8043B099240F03B856C
:101390001BF0100F40F054861BF0400F00F05086F9
:1013A000059A1A805CE699F800706C2F03BF99F8D3
:1013B00001704BF0200B09F101094BF0100B87E68F
:1013C0004BF0400B99F8007082E6002A41F0128041
:1013D0001BF0200F00F02B81099C073424F0070339
:1013E0001946F1E80223099114461D46002A73F1BB
:1013F0000003C0F2F184731C9DF8678008D02BF0C5
:101400008003029354EA050300F08484DDF808B0F9
:10141000002D08BF0A2C80F0548401233034079338
:101420000DF1B7038DF8B740CDF808B00A93079BCC
:10143000B342B8BF3346039300230B9360E7099C84
:10144000002354F8042B8DF890208DF8673001228A
:1014500024AB0392099407920A930026CDF808B0B2
:101460000B96029B13F0020302D0039A02320392FE
:10147000029A239C12F0840B05D1069A0399551AFF
:10148000002D00F3E8829DF8672072B1229A0132A4
:1014900001340DF167000121072ACDE92224CAE9B0
:1014A000000100F31A830AF1080A6BB1229B013391
:1014B00002341AA90222072BCDE92234CAE900120C
:1014C00000F319830AF1080ABBF1800F00F0A8812C
:1014D000079BF61A002E00F3EC81029BDB0500F15E
:1014E0004281229B0A9ACAF80020079ACAF804206F
:1014F00001331444072B2394229300F34E820AF104
:10150000080A029B590705D5069B039A9D1A002DD0
:1015100000F3FD82DDE9053203998A42ACBF9B18D6
:101520005B180593002C40F0FE81002322930DF1FF
:10153000B80A95E5099B99F8007053F8040B0690DA
:101540000028C0F216850993C2E5002A40F05687AC
:101550002E4B10931BF0200F7FF491AE099B1BF0D4
:10156000100F53F8044B099340F02B841BF0400FED
:1015700000F02784A4B2002588E64BF0080B99F808
:101580000070A5E5002A40F02987099C073424F063
:101590000703B3EC027B55EC174B099325F000438E
:1015A00015938DED147ADDE914014FF0FF32184BDD
:1015B0008DED0C7B04F07CFF002840F02B844FF075
:1015C000FF32134BDDE9140104F054FF002840F012
:1015D0002184002200232046294604F041FF0028F0
:1015E00040F03E869DF867800A4A0B4B0321002697
:1015F0002BF08000472FC8BF1A46039102900A9231
:1016000007910B967CE600BF7C7201106872011096
:10161000FFFFEF7F587201105C720110002A40F04A
:10162000E5864BF0100B1BF0200F7FF4D5AE099B25
:101630001BF0100F53F8044B099340F0C5831BF0C7
:10164000400F00F0C18324B2E51722462B46CDE6B9
:1016500099F800704BF0040B3AE599F800700122FC
:101660002B2135E5484610F8017B2A2F00F023870F
:10167000A7F13003092B81464FF000063FF62AAD53
:1016800019F8017B06EB860603EB4606A7F130034B
:10169000092BF5D91EE599F8007000297FF418ADE3
:1016A0000122202114E54BF0010B99F800700FE5A1
:1016B000099A52F8044B09921BF0100200F0518471
:1016C00000253AE6099B1BF0100F53F8044B0993D1
:1016D00000F03F84002501232FE6089802F074F9FA
:1016E00094E4002A40F0D685002F3FF49BAD002300
:1016F00001228DF8673024AB03928DF89070079229
:101700000A93AAE6022318E6DDF808B0012B3FF49D
:101710007FAE022B00F03C822EA900E01146E208C9
:1017200042EA4572E80804F00703054614463033E0
:1017300054EA050001F8013C01F1FF32EED11BF043
:10174000010F0A9200F0DF82302B00F04B840A9ADE
:10175000CDF808B03023023902F8013C2EAB5B1AF9
:1017600007930A9163E6652F40F32381002200234B
:10177000DDE90C0104F06AFE002800F02282229BC1
:10178000BC4ACAF80020013301340122072BCDE9FD
:101790002234CAF8042000F39D840AF1080A1B9B36
:1017A0000E9A239C934280F22483229B119ACAF8BA
:1017B00000200F9ACAF8042001331444072BCDE906
:1017C000223400F3F7830AF1080A0E9B5D1E002DF8
:1017D0007FF797AE102D229ADFF89CB240F3708409
:1017E0001026089FDDF8108005E00AF1080A103D78
:1017F000102D40F3658401321034072ACDE92224EC
:10180000CAE900B6F1DD21AA4146384603F0B0FA34
:1018100000287FF40EADDDE922240DF1B80AE6E7D9
:10182000069B039A9D1A002D7FF752AE102D229A27
:10183000DFF844B22DDD584653462146CA46BB4622
:10184000B1464FF01008089C049E074604E0103D86
:10185000102D03F1080315DD01321031072ACDE9FF
:101860002221C3E90078F2DD21AA3146204603F0A7
:101870007FFA00287FF4DDAC103D102DDDE9222138
:101880002EABE9DC4E46D1469A463B460C465F46B7
:101890009B4601322C44072ACDE92224CAE900B52F
:1018A00000F32484079BF61A002E0AF1080A7FF73A
:1018B00014AE102E229ADFF8C0B128DD5946234617
:1018C000BB461025DDF82080049C0F4604E0103E46
:1018D000102E0AF1080A16DD01321033072ACDE96D
:1018E0002223CAE90075F2DD21AA2146404603F011
:1018F0003FFA00287FF49DAC103E102EDDE9222334
:101900000DF1B80AE8DC1C463B465F469B460132B7
:101910003444072ACDE92224CAE900B600F3448200
:101920000AF1080AD9E521AA0499089803F020FAD7
:1019300000283FF4FAAD7CE421AA0499089803F04A
:1019400017FA00287FF475AC1B9B239C0DF1B80A95
:10195000002B40F0D883029B0E9A03F0010313433F
:101960003FF4CFAD229A119BCAF800300F9BCAF802
:10197000043001321C44072A2394229200F39E84EF
:101980000AF1080A0E9B0A9901321C44072ACDE984
:101990002224CAE900137FF7B2AD21AA049908985E
:1019A00003F0E6F900287FF444AC239C0DF1B80A5B
:1019B000A7E50E9A229B012A04F1010403F1010517
:1019C0000AF1080640F3AF8101230A9ACAF8002001
:1019D000072DCDE92254CAF8043000F345830F9B4C
:1019E000119A01351C44072DCDE92254C6E9002384
:1019F00000F32E8308366B1C1F46B8460E9F0793D4
:101A000000220023DDE90C0106F1080A013F04F081
:101A10001DFD002840F09B810A9B776001333C4408
:101A2000B8F1070F33602394CDF8888000F3B282B9
:101A300006F1100305F1020856469A46129A7260A2
:101A400014441DABB8F1070F2394CDF888803360A0
:101A50007FF757ADA1E7102D229A31DD5146204680
:101A6000CA464FF01008B14613932E46089C049DB9
:101A700009E000BF9872011048720110103E102E4C
:101A800001F1080116DD0132C54B1030072ACDE9FE
:101A90002220C1E90038F1DD21AA2946204603F0C1
:101AA00067F900287FF4C5AB103E102EDDE9222037
:101AB0002EA9E8DC139B354604464E46D1468A469D
:101AC0000132B7492C44072ACDE92224CAE900157E
:101AD00000F3D6820AF1080AD5E421AA04990898ED
:101AE000139303F045F900287FF4A3AB239C139BC9
:101AF0000DF1B80AD9E421AA0499089803F038F93D
:101B000000287FF496AB239C0DF1B80ADCE4102D7D
:101B1000229B21DD1026089FDDF8108004E0103D97
:101B2000102D0AF1080A17DD01339D4A1034072BE6
:101B3000CDE92234CAE90026F1DD21AA4146384622
:101B400003F016F900287FF474AB103D102DDDE989
:101B500022340DF1B80AE7DC0133914A2C44072BFB
:101B6000CDE92234CAE900257FF7D4AC21AA049933
:101B7000089803F0FDF800287FF45BAB239CC9E4D0
:101B8000012B00F0B583022BDDF808B07FF4C4AD63
:101B9000DDF840C02EAA230904F00F0043EA0573C4
:101BA00029091C460D461CF8003002F8013D54EA94
:101BB0000503F0D12EAB9B1A0A92CDF808B007931B
:101BC00035E41B9B002B40F36A820E9B0B9A9342D9
:101BD000A8BF1346002B1D460EDD229B0A9ACAF8A9
:101BE000002001332C44072B2394CAF8045022937D
:101BF00000F3B5830AF1080A0B9B002DA8BF5B1BFD
